:0400000057EF00F0C6
:100008002B002B002B002B002B002B002B002B0090
:1000180028762B002B002B002B002B002B002B000D
:100028002B002B002B002B002B002B002B002B0070
:100038002B002B002B002D002B002B002B0069051B
:1000480072052B00EA022B002B002B002B002B0043
:100058002B002B002B002B002B002B002B002B0040
:100068002B002B002B002B002B002B002B002B0030
:10007800717F2B002B002B002B002B002B002B005B
:100088002B002B002B002B002B002B002B002B0010
:100098002A042B002B002B002B002B002B002B00FD
:0A00A8002B002B00FF00D4EFF0F056
:1000B4003901A3A7110093A711006F00A0F712F054
:1000C4000D0E1218D8B407D00101AB5104E1800E13
:1000D400AA5DD8A016D0010E0101CF6F800EAA250B
:1000E400D96E050EAB21DA6E000EDF6EAAC1AEF139
:1000F400ABC1AFF1000EAB6F000EAA6F390193973D
:100104001100800EAA25D96E050EAB21DA6E6000AF
:100114004BF0DFFFAA4BAB2BAAC1AEF1ABC1AFF1E1
:100124001100606F3BC063F03CC064F03DC061F0FF
:100134003EC062F00001605179ECFCF00009D8B4D3
:10014400F9D7800E2B6E080E2C6E000E2D6E610EEC
:100154002E6E2F6A0AEC0CF03A0E256E266A000EFB
:10016400286E010E276E25EC0CF0000E2B6E000E8F
:100174002C6E000E2D6E000E2E6E000E2F6EFCECFB
:100184000BF0C6EC0CF06DEC0BF0E806D8A41200F2
:10019400FAD7000E2A6E26AE06D0256C261ED8B0DD
:1001A400262A010E2A6E28AE04D0276C281ED8B049
:1001B400282A27502810D8B418D0010E296E04D04C
:1001C400D89027362836292A28AEFAD72750255C16
:1001D40028502658D8A004D02750255E2850265AE7
:1001E400D89028322732292EF1D72A50D8B404D0F7
:1001F400256C261ED8B0262A25C025F026C026F058
:10020400120025C02BF026C02CF019D02906D8A046
:100214002A0660009FF0D9FF6000A3F0DAFF274AA6
:10022400282A6000AFF0E1FF6000B3F0E2FF2B4A40
:100234002C2A6F007FFFE7FFE750D8B40FD0295076
:100244002A10D8B40BD0E2D76000AFF0D9FF600019
:10025400B3F0DAFF000EDF6E2B4A2C2A2906D8A051
:100264002A062928F1E12A28D8B41200EDD7600023
:100274009FF0F6FF6000A3F0F7FF000EF86E080091
:100284006F00D4FFCEF119D060009FF0F6FF60003C
:10029400A3F0F7FF000EF86E08006F00D4FFCEF154
:1002A400600097F0D9FF60009BF0DAFF60003BF735
:1002B400DFFF254A262A274A282A0101CE51D8A43D
:1002C400E3D7600097F0D9FF60009BF0DAFF000EDF
:1002D400DF6E12003B6E000E3C6E3B5079ECFCF07E
:1002E4000009D8B4FAD7F80E2B6E120E2C6E000E3D
:1002F4002D6E3C0E2E6E2F6A0AEC0CF03A0E256E13
:10030400266A000E286E010E276E25EC0CF0000EF6
:100314002B6E000E2C6E000E2D6E000E2E6E000E37
:100324002F6EFCEC0BF0C6EC0CF06DEC0BF0E80659
:10033400D8B4FBD73C50120020C1FDF021C1FEF01F
:10034400000E0201546F000E536F15D01EC1F4F05D
:100354001FC1F5F0FD0E0001F66F22C1F7F023C1B5
:10036400F8F0D2ECC9F00001F45102015327000166
:10037400F551020154236000F7F3F6FF6000FBF32C
:10038400F7FF000EF86E0800F5500009D8A4DED778
:1003940053C21EF154C21FF1120029890ED0E6EC9B
:1003A4000CF0070E120002012529B7EC0CF0030E25
:1003B4001200E9EC0CF00A0E120012C230F013C263
:1003C40031F001D80AD00500FA6E0051FD6E0151DA
:1003D400FE6E0251FF6EFA501200326E336A3350D1
:1003E400000AD8A4E6D73250010AD8B4E2D7030AE7
:1003F400D8B4D5D7060AD8B4D6D7DBD72BC02FF0BC
:100404002CC030F029C031F02AC032F02F502D6EAC
:1004140030502E6E2F4A302A6000B7F0F6FF60008D
:10042400BBF0F7FF000EF86E6000C7F0D9FF600064
:10043400CBF0DAFF314A322A1F0EF76403D00800EA
:10044400F55007D06F00DBFFE1FF6F00DFFFE2FF35
:10045400E750DF6EDF50D8B41200D8D73901A3B704
:100464006F00A0F712F0000E266E000E256E800EAF
:100474002524D96E050E2620DA6E000EDF6E254A7D
:10048400262A265004E17F0E255CD8A0F0D73D0132
:10049400F289000EF96F000EFA6F000E0501806FED
:1004A400000E0101AF6F000EAE6F000E126E000E53
:1004B400CF6F3901938D938712003C6E3C5079ECD9
:1004C400FCF00009D8B4FAD7980E2B6E120E2C6EDD
:1004D400000E2D6E3B0E2E6E2F6A0AEC0CF03A0EB7
:1004E400256E266A000E286E010E276E25EC0CF090
:1004F400000E2B6E000E2C6E000E2D6E000E2E6E56
:10050400000E2F6EFCEC0BF0C6EC0CF06DEC0BF057
:10051400E806D8A41200FAD7D6EC0CF0020E0201B9
:10052400286F09D07EEC0CF01200EEEC0CF01200F7
:100534006FEC0CF0120014C230F015C231F020EE52
:1005440003F201D80AD00500FA6EDE50FD6EDE50CB
:10055400FE6EDE50FF6EFA501200326E336A335074
:10056400000AD8A4E5D73250020AD8B4DBD7010A6E
:10057400D8B4DBD7DDD7000E01015E6F300E5D6F9E
:1005840029ECF4F05DC170F15EC171F15FC172F1EB
:1005940060C173F1000E01015E6F340E5D6F29ECD2
:1005A400F4F05DC174F15EC175F15FC176F160C1B3
:1005B40077F1000E01015E6F380E5D6F29ECF4F0E7
:1005C4005DC178F15EC179F15FC17AF160C17BF1FF
:1005D4001200000ED2BE010E2A6E2650030B390102
:1005E400E16F600097F0E0F960009FF0E3F93F0EDF
:1005F400E517E585D29E550EE66FAA0EE66FE583F4
:1006040000F03901E5B3FCD7E5952AB002D0D29EBB
:1006140001D0D28E030E296E080E286E770EE82EB6
:10062400FED7282EFCD7292EFAD700F01200ACEC06
:1006340009F002012951030B0009D8B408D085EC54
:100644000CF00009D8B403D0100E0201276F020188
:100654002751030DEF0EF324F66ED10EF420F76E3E
:10066400F86A000EF82201D80DD00500FA6E0900D0
:10067400F550FD6E0900F550FE6E0900F550FF6E51
:10068400FA5012000201276F1200D2AE02D0010EFE
:1006940001D0000E256ED29ED28AD29ED29CD28ADE
:1006A400550ED46EAA0ED46ED490000ED76E000EE2
:1006B400D66E080ED56E550ED46EAA0ED46ED480A6
:1006C4003901838781818491839F8495879189915E
:1006D400809FD28CD28E25B002D0D29E01D0D28EF1
:1006E4001200FC0E2917020E286F299505D0ECEC98
:1006F4000CF012000F0E120016C230F017C231F0C7
:1007040020EE06F201D80AD00500FA6EDE50FD6E26
:10071400DE50FE6EDE50FF6EFA501200326E336A07
:100724003350000AD8A4E6D73250020AD8B4DFD72F
:10073400010AD8B4DCD7DED7000E2B6E000E2A6E69
:1007440027502810D8B41CD0010E296E04D0D8909C
:1007540027362836292A28AEFAD7D8902A362B36B7
:100764002750255C28502658D8A005D02750255E50
:100774002850265A2A80D89028322732292EEDD79D
:100784002AC025F02BC026F01200000E476E000E82
:10079400466E44504510D8B41CD0010E486E04D0A7
:1007A400D89044364536482A45AEFAD7D8904636CE
:1007B40047364450425C45504358D8A005D0445075
:1007C400425E4550435A4680D89045324432482EC2
:1007D400EDD746C042F047C043F01200280E4C6FDC
:1007E400010E4D6F24C14EF125C14FF1000E526F21
:1007F400000E516F000E586F000E576F4E0E1E6F95
:10080400010E1F6F26C120F127C121F14C0E226F6A
:10081400010E236F9EEC01F0010151512425D96E84
:1008240052512521DA6E000EDF6E1200000E000117
:10083400676F000E666F0ED066516325D96E6751DF
:100844006421DA6EDF509BECFFF07EEC0BF00001CC
:10085400664B672B66516325D96E67516421DA6E46
:10086400DF50D8B412005750665D6751800A656F37
:100874005850800A6559D8B01200DED720EE02F035
:100884003050D9263150DA226F0078FF25F06F00FE
:1008940074FF26F06000C3F0D9FF6000C7F0DAFFF0
:1008A4006F0078FF27F06F0074FF28F025EC0CF040
:1008B400000E2B6E000E2C6E000E2D6E000E2E6E92
:1008C400000E2F6E0AEC0CF0020E1200256E390198
:1008D4009991050E966E000E956E000E926E770E2F
:1008E400946EF40E936E0101BC9B3901A9912550BD
:1008F400D8B408D0FF0E25240201796F7A6BFF0E5D
:100904007A2305D0000E02017A6F000E796F390147
:100914009981A991948E120025C027F026C028F051
:1009240002D0254A262A600097F0F6FF60009BF06B
:10093400F7FF000EF86E1F0EF76403D00800F550A1
:1009440007D06F00DBFFE1FF6F00DFFFE2FFE7503E
:100954000009D8A4E6D72750255C256E28502658D0
:10096400266E1200266E040E1218D8A409D0112A7D
:100974002B0E3D01EA6F1150255CD8A026C011F062
:10098400080E1218D8A409D011062D0E3D01EA6FE5
:100994002650115CD8A025C011F0600093F6D9FF51
:1009A400600097F6DAFF600047F0DFFF12003E6E4A
:1009B4003E5079ECFCF00009D8B4FAD73AC025F0DF
:1009C4003BC026F03CC027F03DC028F025EC0CF0DD
:1009D400000E2B6E000E2C6E000E2D6E000E2E6E71
:1009E400000E2F6EFCEC0BF0C6EC0CF06DEC0BF073
:1009F400E806D8A41200FAD7000E3D01EC6F000EF1
:100A0400ED6F000EEE6F000EEF6F000EF06F000E34
:100A1400F16FB00EF26F800EF36F000EF46F8A0E5A
:100A2400F56F000EF66F000EF76F000EF86F000EF4
:100A3400F96F000EFA6FF28BF28939019397120065
:100A4400256EB89EB888B896B894B892B890B98E06
:100A5400B99CB98AB988B996B984B982B980670E44
:100A6400B76E440EB66E000E02017E6F000E7D6FEF
:100A74000101BC913901A39F2504D8A402D0938F0E
:100A840001D0939FB88E1200D29E2D0E0201596F91
:100A94005A6B000E326E000E316E31502B24256ECF
:100AA40032502C20266E315002015925D96E325015
:100AB4005A21DA6EDF50276EEBEC02F0314A322A0B
:100AC400325004E1040E315CD8A0E7D7D28E120074
:100AD400000E00018A1B000E8B1B000E8C1B800E67
:100AE4008D1B86C076F087C077F088C078F089C007
:100AF40079F08AC07AF08BC07BF08CC07CF08DC01A
:100B04007DF099ECE0F076C086F077C087F078C08D
:100B140088F079C089F01200286E000E0201626F1D
:100B2400000E616F0FD0520E266E2B0E256E000E36
:100B3400E82EFED7252EFCD7262EFAD700D00201A8
:100B4400614B622B2850256E266A2550615D6251E7
:100B5400800A276E2650800A2758D8B01200E3D79F
:100B6400000EAC6E050EAE6EAC8CAC9AAC88AC507C
:100B7400F00B0709AC6EC20EAB6E000EAA6E000E2F
:100B8400AF6E000E0201766F000E756F0101BC9509
:100B9400000E0201706F000E6F6F39019485A495E9
:100BA400AC8E12006F0060FF53F00201754B762B80
:100BB400000E706F010E6F6FC20EAB6E75C24EF0F9
:100BC40076C24FF0000E516E0A0E506E17EC06F00E
:100BD4004E504F10D8A402D00101BC853901A49510
:100BE40060004FF1D8FF110027502810D8B418D056
:100BF400010E296E04D0D89027362836292A28AE2B
:100C0400FAD72750255C28502658D8A004D027505E
:100C1400255E2850265AD89028322732292EF1D71B
:100C240025C025F026C026F0120050505110D8B42B
:100C340018D0010E526E04D0D89050365136522A34
:100C440051AEFAD750504E5C51504F58D8A004D0F2
:100C540050504E5E51504F5AD89051325032522E0D
:100C6400F1D74EC04EF04FC04FF0120000016E6F2E
:100C74009E0E256E030E266E8EECFBF032EC0CF00D
:100C8400020E00016E6108D0A60E6E25D96EDA6AD6
:100C9400030EDA22070EDF6E010E6A6F9E0E6B6F73
:100CA400030E6C6F0D50EEEC0BF01200000EA06EF4
:100CB400050EA26E700EA012A050F00B0709A06ED4
:100CC400F40E9F6E000E9E6E000EA36E000E0201C7
:100CD400786F000E776F000E746F000E736F010152
:100CE400BC9939019781A791A09E120011D03901B6
:100CF400A3A9FDD76000AFF0F6FF6000B3F0F7FFE3
:100D0400000EF86E08006F00D7FFEAFD2B4A2C2A6C
:100D14006000AFF0F6FF6000B3F0F7FF000EF86E6E
:100D24000800F5500009D8B41200E1D726BE11D04E
:100D3400265003E12504D8A00CD0C294CA941A0EFC
:100D4400E82EFED700D0C284C00E00D0E82EFDD716
:100D54001200C294CA94E00E00D0E82EFDD7C284DB
:100D64000A0EE82EFED700D0120026BE11D026505F
:100D740003E12504D8A00CD0C292CA921A0EE82E20
:100D8400FED700D0C282C00E00D0E82EFDD71200DC
:100D9400C292CA92E00E00D0E82EFDD7C2820A0E9B
:100DA400E82EFED700D0120026BE11D0265003E153
:100DB4002504D8A00CD0C290CA901A0EE82EFED7F3
:100DC40000D0C280C00E00D0E82EFDD71200C29021
:100DD400CA90E00E00D0E82EFDD7C2800A0EE82E9D
:100DE400FED700D01200010E2B6E200E25182610FF
:100DF400D8B414D0F70E276EFF0E286E25C029F044
:100E040026C02AF02750292628502A222A5004E1F5
:100E1400050E295CD8A002D0000E2B6E2BC025F045
:100E2400266A1200CF0E2B6EFD0E2C6E78EC06F0A7
:100E34000F50300F4AEC0CF032EC0CF0010E8EEC3B
:100E440005F0000E106E000E3A01576F000E0F6E83
:100E5400000E106E0101BC9F3901A1919181120015
:100E64003E6E3EC03AF0680E6CEC01F00201916FE8
:100E74003D04D8A410D01E0E256E030E266E91518B
:100E840050EC07F01E0E256E030E266E8EECFBF062
:100E9400090E4AEC0CF0020191511200276E27381A
:100EA4000F0B300F600097F0D9FF60009BF0DAFF62
:100EB400DF6E20EE01F02550D9262650DA22275085
:100EC4000F0B300FDF6E20EE02F02550D92626508E
:100ED400DA22000EDF6E1200386E010E396E020146
:100EE40029B516D02985000E396E2551B7EC0CF0C2
:100EF4003850D8B406D0040E0201276F5CEC0BF016
:100F040005D0030E0201276F54EC0CF05EEC0CF0DC
:100F140039501200AFD6A6D69DD694D68BD682D69B
:100F240079D670D605040306060502000000803F4A
:100F34000000003F0000003F000020C100004040CE
:0F0F4400010020203030304830304D3030530025
:100F54001004D8A41200E90E055C030E0658D8A0AC
:100F64001200000E106E000E0201A76FC0EC0BF011
:100F7400000E0D6E000E0E6E000E0F6ED00E2B6E58
:100F8400F00E2C6E78EC06F01200266E000E286E21
:100F94002550D8B415D0010E276E03D0D89025362D
:100FA400272A25AEFBD7D89028362550265CD8A012
:100FB40003D02550265E2880D8902532272EF3D7DB
:100FC40028501200BF0E2D6EFF0E2E6E2BC02FF078
:100FD4002CC030F02D502F262E50302230500AE1F4
:100FE4001A0E2F5CD8B006D0200E2B102B6E2C506E
:100FF4002C6E12002BC02BF02CC02CF012009F0E74
:101004002D6EFF0E2E6E2BC02FF02CC030F02D5005
:101014002F262E503022305009E11A0E2F5CD8B002
:1010240005D05F0E2B142B6E2C6A12002BC02BF0F4
:101034002CC02CF01200000E346E000E336E0BD058
:1010440032C025F0266A30C027F031C028F093EC76
:10105400FAF0334A342A33502E24D96E34502F20D8
:10106400DA6EDF50326E3250D8B41200E9D79F0ED8
:10107400276EFF0E286E200E2510296E000E2610F6
:101084002A6E2750292628502A222A5006E11A0EB1
:10109400295CD8B002D0010E01D0000E256E266A5C
:0210A400120038
:1010A8006F0060FF24F002017ABF09D07A5103E192
:1010B8007905D8A004D07907D8A07A0704D001010F
:1010C800BC8B3901999156803901A991600093F040
:1010D800D8FF110000D7FAD6F4D6EED6E8D6E2D675
:1010E800DCD6D6D6D0D6CAD6C4D6BED6B8D653D570
:1010F80053D48AD5E7D53CD6DCD251D2A9D300D473
:1011080098D4B9D51AD5C290CA900B0E256E620E26
:10111800E82EFED7252EFCD700D0C280C00E00D006
:10112800E82EFDD7CAB01200E40E00D000D0E82E99
:10113800FCD700D000D01200C294CA940B0E256EC2
:10114800620EE82EFED7252EFCD700D0C284C00E32
:1011580000D0E82EFDD7CAB41200E40E00D000D0AB
:10116800E82EFCD700D000D01200C292CA920B0E13
:10117800256E620EE82EFED7252EFCD700D0C2823F
:10118800C00E00D0E82EFDD7CAB21200E40E00D07F
:1011980000D0E82EFCD700D000D01200C290CA9030
:1011A8000B0E256E620EE82EFED7252EFCD700D03A
:1011B800C280C00E00D0E82EFDD7CAB01200E40EDF
:1011C80000D000D0E82EFCD700D000D01200B7BF66
:1011D80005D0B75110E1B605D8B00DD0B6C0B8F0FB
:1011E800B7C0B9F0B81FB91FB84BB92BB8C0B6F023
:1011F800B9C0B7F01200B6C0B6F0B7C0B7F0120069
:101208009F0E276EFF0E286E25C029F026C02AF0F3
:101218002750292628502A222A5006E11A0E295C2E
:10122800D8B002D0010E01D0000E256E266A120039
:10123800BF0E276EFF0E286E25C029F026C02AF0A3
:101248002750292628502A222A5006E11A0E295CFE
:10125800D8B002D0010E01D0000E256E266A120009
:10126800D00E276EFF0E286E25C029F026C02AF062
:101278002750292628502A222A5006E10A0E295CDE
:10128800D8B002D0010E01D0000E256E266A1200D9
:1012980030C025F031C026F0000E286E010E276EF2
:1012A80025EC0CF0000E2B6E000E2C6E000E2D6E31
:1012B800000E2E6E000E2F6E0AEC0CF0040E1200BB
:1012C80030C025F031C026F0000E286E020E276EC1
:1012D80025EC0CF0000E2B6E000E2C6E000E2D6E01
:1012E800000E2E6E000E2F6E0AEC0CF0020E12008D
:1012F80030C025F031C026F0000E286E010E276E92
:1013080025EC0CF0000E2B6E000E2C6E000E2D6ED0
:10131800000E2E6E000E2F6E0AEC0CF0020E12005C
:1013280030C025F031C026F0000E286E020E276E60
:1013380025EC0CF0000E2B6E000E2C6E000E2D6EA0
:10134800000E2E6E000E2F6E0AEC0CF0040E12002A
:1013580093EC0CF00009D8B403D0FAEC0CF01200AE
:10136800A6EC0CF00009D8B403D0F6EC0CF012008F
:10137800ACEC0CF00009D8B41200F8EC0CF0120038
:101388000000984100002041000070410000984191
:101398000000F0410000AA4200000C420000003F9B
:1013A800000020410000A0C00000984101473350D0
:1013B800341035103610D8B408D0000E331A000E89
:1013C800341A000E351A800E361A33C033F034C082
:1013D80034F035C035F036C036F01200266E800E77
:1013E8000ED0265027140009D8B404D02A0E4AEC8F
:1013F8000CF003D0200E4AEC0CF0D8902730276E62
:101408002750D8B41200EDD7266E080E276E000EAE
:10141800286ED89026342834286ED8902636255041
:10142800285CD8A002D02550285E272EF2D7285055
:101438001200C294CA94050EE82EFED700F0C284AA
:101448001A0EE82EFED700D0000ECAB4010E256E83
:10145800B00E00D0E82EFDD725501200C292CA92D5
:10146800050EE82EFED700F0C2821A0EE82EFED72F
:1014780000D0000ECAB2010E256EB00E00D0E82EC4
:10148800FDD725501200C290CA90050EE82EFED74F
:1014980000F0C2801A0EE82EFED700D0000ECAB0A7
:1014A800010E256EB00E00D0E82EFDD72550120093
:1014B800255027026F00CCFF29F06F00D0FF2AF0DB
:1014C80025502802F3502A2626502702F3502A26B0
:1014D80029C025F02AC026F012000001606F3FC025
:1014E80061F0000E0001626F610E3A6E3B6A000EF9
:1014F8003D6E010E3C6E6051D9EC04F0A00EE82E52
:10150800FED7120033C025F034C026F08EEC04F06C
:1015180025503324296E265034202A6E35C02BF0EE
:1015280036C02CF000EC02F01200286E000E296E76
:1015380028C027F0010E27162750256E266A98EC3A
:1015480006F0D8902832292A070E2964F1D712000C
:10155800286E000E296E28C027F0010E2716275086
:10156800256E266AB7EC06F0D8902832292A070E8D
:101578002964F1D71200286E000E296E28C027F0C2
:10158800010E27162750256E266AD6EC06F0D8904D
:101598002832292A070E2964F1D712006F0060FF4C
:1015A8004DF002017D4B7E2B0101BC81660EB76EAA
:1015B8007C0EB66E3901A39F600037F1D8FF110089
:1015C8006F0060FF55F0000E0201726F010E716F1F
:1015D800400E3D01EA6F39019491A491600057F1E2
:1015E800D8FF1100030E3D017B6F040E736F800E50
:1015F800746F000E756F000E6C6F7599200E6E6F0C
:101608007995739F1200000E266E000E276ED890F3
:1016180026321DEC0AF00009D8A4268E272A070EC8
:101628002764F5D726501200000E266E000E276E8E
:10163800D890263232EC0AF00009D8A4268E272A40
:10164800070E2764F5D726501200000E266E000EEE
:10165800276ED890263247EC0AF00009D8A4268EC7
:10166800272A070E2764F5D72650120000016F6F4E
:101678006BC065F000016F511FECFEF06CC063F0A9
:101688006DC064F06EC065F0DFECF9F0120073BF56
:101698001200000E796F000E7A6F000E766F6C697B
:1016A800510E3A016A6F510E6B6F3D01738F120034
:1016B80002012951FC0B0209296F25052611D8B40E
:1016C8005FECFFF0D88002012235B2EC0CF0040E7A
:1016D8001200010E256E020129B50AD02997226948
:1016E800D6EC0CF0DFEC0BF0C1EC0CF028C225F0C6
:1016F80025501200000E266E000E256E00F0254AB9
:10170800262A26BEFBD7265005E1A00E255CD8B0B8
:101718001200F4D71200286E756C6C2900000000C6
:101728003F0000A042456300436600486700303030
:071738002F30302F3030008C
:101740003D017995600097F06EFD000E6C6F738B14
:1017500079A5FED774BB02D0010E1200000E120054
:101760002A6E0A0E256E2A5008EC0AF0296E0A0E1F
:10177000256E2A50C7EC07F0100DF35029241200F3
:10178000B89E670EB76E440EB66E000E02017E6FF5
:10179000000E7D6F0101BC913901A39FB88E12002C
:1017A000DAEC0CF0F0EC0CF00009D8B406D0000E26
:1017B000B7EC0CF0000EB2EC0CF0000E1200390188
:1017C00093939395929F93913D017A917A957A9F05
:1017D0007A9D7A9376937695769112006D6F6AC0B2
:1017E00065F000016D511FECFEF06BC063F06CC042
:1017F00064F018EC04F012002BC025F02CC026F089
:101800002DC027F02EC028F02FC029F0020E61EC69
:10181000FEF012002BC025F02CC026F02DC027F0C2
:101820002EC028F02FC029F0000E61ECFEF012004F
:101830003901A3B11200A2BF12003D0179B5120017
:1018400079BF120076B91200F3D7020129A912005C
:1018500025C023F226C024F227C025F228C026F294
:10186000299912003901A3A9FDD70D0E3D01EA6F98
:101870003901A3A9FDD70A0E3D01EA6F1200266EB9
:1018800026C025F00F0E251626380F0B0A0DF35033
:1018900025241200256E01D000F03901A3A9FCD740
:1018A000600097F0EAFD12002951FC0B0209296F34
:1018B00022512225B2EC0CF0030E120004D018ECD9
:1018C0000CF019EC03F0020129A51200F8D7BCECCA
:1018D0000CF002012995020E286F0F0E1200BCECCD
:1018E0000CF002012995000E286F0F0E1200DDEC9E
:1018F0000CF0DAEC0CF09AEC0CF01200020125511D
:10190000B7EC0CF05CEC0BF012003D0174AB02D0B4
:10191000010E1200000E12003D0178A102D0010E4E
:101920001200000E12003D0179AF02D0010E12002C
:10193000000E120002012995000E286F0F0E1200F2
:1019400078AB02D0010E1200000E120079A502D071
:10195000010E1200000E120076A902D0010E120034
:10196000000E1200256E600097F06BFD1200256ED0
:10197000600097F06CFD12003D01739F7885738FB6
:101980001200739F000E796F78851200000E6EECC6
:1019900007F01200DDEC0CF0090E1200E0EC0CF088
:1019A000040E1200E0EC0CF0030E1200000E3D01DC
:1019B000796F12003D01739B12003D01748D12007E
:1019C0003D01749D12003D016A5112003D01738D6D
:1019D00012003D01739D1200010E1200020E120052
:1019E0006C511200050E1200010E120079951200C2
:0A19F00076991200799F1200120090
:10D1AE000000000000001B1B0000181818181B1BA5
:10D1BE000000030303031B1B00001B1B1B1B1B1B7D
:10D1CE0000040E1F0404040400040404041F0E04CF
:10D1DE00001112140B110203000E0A0E00000000C3
:10D1EE0000341900B81600A8180032EA0142FE01F8
:10D1FE009E0300BEFE01FC1800DC1900D81900A029
:10D20E0017009C1900A41900EE1800941900DE18DE
:10D21E0000E606001C0500CE18004C754D614D65EC
:10D22E004A655665536144694572004345444D5203
:10D23E00414A505456575A0080C094D40000004BB7
:10D24E0000027F204120696E636C7572653A200D75
:10D25E000A204D414A5F5254435F4D616E75656CB5
:10D26E006C655F323032342D30382E696E632C206F
:10D27E004469616C6F6775655F4F70657261746547
:10D28E0075725F50435F7669615F554152545F32EC
:10D29E003032342D303930340D0A204D454E553153
:10D2AE00305F313233345F323032342D30382E69C4
:10D2BE006E632C204D454E55345F5357345F3230DC
:10D2CE0032342D303931382E696E630D0A0020410B
:10D2DE007574726573203A0D0A202044533138421A
:10D2EE0032305F323032342D30372E682C204F6E74
:10D2FE0065576972655F323032332E680D0A204CE5
:10D30E0043445F34626974735F4932435F32303233
:10D31E00342D30312C2055415254315F46756E6399
:10D32E0074696F6E732E682C205254435F445333CE
:10D33E003233315F323032332D31302E680D0A00E8
:10D34E004346546373670045434F63736700484712
:10D35E004C63736700494E54636F72004E524769B7
:10D36E006E64004E5247636F72004348446D696E9F
:10D37E00004348446D6178004558546D696E00490C
:10D38E004E54687973004558546879730045415579
:10D39E006879730020202020202000204C43445F19
:10D3AE0063686172735F53706563696175785F322C
:10D3BE003032332D303832372E682C202020456500
:10D3CE0070726F6D203A20456570726F6D5F5049B7
:10D3DE00435F323032342E682C2020456570726FD8
:10D3EE006D5F5049435F323032342E632020200D62
:10D3FE000A00204861726477617265203A204361A9
:10D40E007274652050434220436861756469657289
:10D41E00650D0A20536368656D613A205363686534
:10D42E006D615F4368617564696572655F5632311F
:10D43E002E312E342E70646620284B696361642968
:10D44E000D0A0D0A00204469726563746F727920AB
:10D45E003A20433A5C4D504C4142585F50726F6ACD
:10D46E00656374735C4368617564696572655F4377
:10D47E006F6E74726F6C655F31384632374B343273
:10D48E005F323032342E580D0A00205241302C5269
:10D49E0041312C5241323D3378445331384232308F
:10D4AE002C5241343D6C65642C5241333D535141F5
:10D4BE002C5243363D54582055415254312052433C
:10D4CE00373D525820554152540D0A0045434F2EB8
:10D4DE002E2E2E0042415252455F4700424152527B
:10D4EE00455F44004241525245474400464C454335
:10D4FE0048204800464C4543485F4200312F324891
:10D50E00657572004445475245432000204C434404
:10D51E0020347832302063617273202B20525443B2
:10D52E00207375722062757320493243312048573B
:10D53E00203A205243333D53434C2C5243343D53F7
:10D54E0044410D0A002050494331384632374B349E
:10D55E0032202B203378204F57532073656E736F14
:10D56E00722044533138423230207375722052414A
:10D57E00302C5241312C5241320D0A002050726F24
:10D58E006A656374203A2020436861756469657228
:10D59E00655F436F6E74726F6C655F3138463237FC
:10D5AE004B34325F323032340D0A0020524230207A
:10D5BE00696E746572727570742070696E2C20536A
:10D5CE0057302E2E2E535735202B2053573620737F
:10D5DE007572205243350D0A0020536F75726365C4
:10D5EE00203A20206D61696E2E63202C20726576A4
:10D5FE00203A2076657273696F6E3A32343130306C
:10D60E00340D0A002053573020002053573120008C
:10D61E0020535732200020535733200020535734C5
:10D62E00200020535735200020535736200020432A
:10D63E006F6E6669672020496E7465726E616C202C
:10D64E00466F73632036344D487A0D0A0020202031
:10D65E0020202020202020202020202020202020BC
:10D66E0020004572726F722020200044696D616E39
:10D67E006368650053616D65646920200056656EB0
:10D68E006472656469004A65756469202020004DE6
:10D69E0065726372656469004D6172646920202051
:10D6AE00004C756E646920202000446563652E0071
:10D6BE004E6F76652E004F63746F2E005365707437
:10D6CE002E00416F757420004A75696C2E004A75E4
:10D6DE006E6520004D6169202000417672692E0032
:10D6EE004D6172732000466576722E004A616E7629
:10D6FE002E006572722E20002020005002A00050D5
:10D70E0000300020446966303D25332E33662020DC
:10D71E00446966313D25332E336620446966323DB9
:10D72E0025332E336620446966333D25332E32660B
:10D73E000D0A20446966343D25332E32662020447E
:10D74E006966353D25332E326620446966362533AB
:10D75E002E32660D0A4541555F6D696E3D25332E9D
:10D76E003266204541555F6D61782025332E326635
:10D77E00200D0A0020656C6C657320646F697665F8
:10D78E006E7420657472652072656C6965657320B0
:10D79E006D6563616E697175656D656E7420656E1C
:10D7AE0073656D626C657320286D656D652074659B
:10D7BE006D706572617475726520616D6269616EFE
:10D7CE007465290D0A002052657374617572617457
:10D7DE00696F6E206465206C6120636F70696520CF
:10D7EE005573696E65205461626C65732050726763
:10D7FE0020486F726169726520656E204565707292
:10D80E006F6D2050494320617420307830323630AD
:10D81E000D0A0020536F727469206465207465735D
:10D82E0074207061722076616C69646174696F6EC8
:10D83E0020706172205357353E322073656320206D
:10D84E006F752054696D656F757420646520313075
:10D85E00736563206F7520535734200D0A000D0A2F
:10D86E002048617264776172653A207665727369D9
:10D87E006F6E20436172746520504342206368616D
:10D88E00756469657265203A204C434420426C6190
:10D89E006E632061206C276164726573736520303E
:10D8AE0078323020210D0A002053617576652041B3
:10D8BE0066666563746174696F6E5F486562646FF6
:10D8CE0020656E20656570726F6D2040204F726707
:10D8DE005F53617576655F506172616D5F54726101
:10D8EE007661696C2B35362B20696E646963650D24
:10D8FE000A000D0A20417474656E74652072656DA0
:10D90E0069736520656E20706C6163652064657354
:10D91E0020332063617074657572732C65742052A8
:10D92E004553455420706F757220736F727469720F
:10D93E00200D0A000D0A2054657374206D6F646506
:10D94E0020506F6F6C696E672064657320362042BD
:10D95E00502073757220504F525442202C20646513
:10D96E002067617563686520612064726F697465F4
:10D97E00200D0A002052657374697475652050611C
:10D98E0072616D657472657320427974657320647B
:10D99E0065707569732040202530345820736F6987
:10D9AE0074202564202020204261766172643D251A
:10D9BE00640D0A00204C45445F436C69676E6F74BA
:10D9CE00653D3634206F752033322028706F7572A6
:10D9DE00207465737420636C69676E6F7465204C78
:10D9EE0065642045636F206F7520636F6E66292016
:10D9FE000D0A002065783A20553B32383B30383BD3
:10DA0E0032333B31383B31343B30313B23202070B5
:10DA1E006F757220323820416F7574203230323378
:10DA2E00202C2031384831342C4C756E6469200D11
:10DA3E000A002053617576656761726465732063B1
:10DA4E006F7272656374696F6E7320656E204565C3
:10DA5E0070726F6D20656E203078303035302C202E
:10DA6E003078303035342C203078303035380D0A5F
:10DA7E000020436861726765205461626C652050B6
:10DA8E00726F67722073656C656374696F6E6E6515
:10DA9E00652064616E73205461626C652050726FF4
:10DAAE0067722E50726F7669736F6972650D0A0018
:10DABE0020526573746974756520506172616D656D
:10DACE007472657320466C7420646570756973207A
:10DADE0040202530345820736F697420256420202F
:10DAEE0020204261766172643D25640D0A00207328
:10DAFE00617665204574617420696E7020416C6199
:10DB0E00726D6573204036382065742045746174DB
:10DB1E00204F757420416C61726D6520403639203E
:10DB2E00746F20456570726F6D0D0A0020484D3D73
:10DB3E0078783A7979202073657420486575726516
:10DB4E00287878294D696E7574657328797929203E
:10DB5E0053414E53206C69656E2061766563205289
:10DB6E005443202120200D0A003165726520696E14
:10DB7E00697420646573203130205461626C657362
:10DB8E002050726720486F726169726520656E2041
:10DB9E00456570726F6D2050494320617420307856
:10DBAE003130300D0A0020553B32343B30383B319A
:10DBBE00373B31383B33363B30342320706F757230
:10DBCE0020323420416F75742032303137202031AD
:10DBDE00384833362030343D4A657564690D0A0D78
:10DBEE000A002064616E73206C61205461626C6562
:10DBFE0020646520547261766169206574206461C9
:10DC0E006E73206C61205A6F6E65204570726F6D59
:10DC1E00206465207472617661696C0D0A00200DB6
:10DC2E000A526563757065726174696F6E20646502
:10DC3E00732050726F6772616D6D6573206465201D
:10DC4E007472617661696C206465707569732045C4
:10DC5E006570726F6D200D0A002045746174206925
:10DC6E006E697469616C203A20206B3D2535642005
:10DC7E0020736F69742030782530345820206D3D24
:10DC8E00202535642020736F697420307825303458
:10DC9E00580D0A0020546573742053573620706F48
:10DCAE0075722064656D616E6465204567616C698F
:10DCBE00736174696F6E206F752052657374617530
:10DCCE00726174696F6E205573696E650D0A00205E
:10DCDE0052656368617267656D656E7420636F72FD
:10DCEE0072656374696F6E732063617074657572AB
:10DCFE007320445331384232302064657075697335
:10DD0E0020456570726F6D0D0A000D0A0D0A2020F8
:10DD1E004D6F64696669636174696F6E5F50726F8F
:10DD2E006772616D6D6174696F6E5F486F72616964
:10DD3E0072652E203220E02039204F4E4C590D0AAC
:10DD4E000D0A0020526563757065726174696F6E9D
:10DD5E002064657320706172616D657472657320E5
:10DD6E006465207472617661696C20646570756992
:10DD7E007320456570726F6D200D0A0053617665D4
:10DD8E0020746F20656570726F6D204353475F4539
:10DD9E006E5F436F7572732040343420657420209B
:10DDAE0043686F69785F486F72735F47656C204098
:10DDBE0037300D0A002052652D496E69742043706C
:10DDCE0074322054696D657232203130306D5320BB
:10DDDE00706F7572206D65737572652064757265EE
:10DDEE006520646520626F75636C650D0A00696E4F
:10DDFE00646963653D2533642040656570726F6D9F
:10DE0E0020307825303458202050726F672023251B
:10DE1E006420204E616D6520256320203C2D202539
:10DE2E0073200D0A002050726F6772616D6D652050
:10DE3E002325642028256329206166666563746541
:10DE4E002061637475656C6C656D656E74206175AB
:10DE5E00206A6F75723D2025730D0A002050726F77
:10DE6E00672053656C6563743D20253264205072C3
:10DE7E006F677220656E20636F7572733D25326415
:10DE8E002050726F67204E616D65202563200D0A4C
:10DE9E0000205361757665203A204166666563748D
:10DEAE006174696F6E2050726F6772616D6D65205F
:10DEBE002563202D3E206175204A6F7572202573D3
:10DECE0020200D0A0020535735204D656E753D25D7
:10DEDE003264204D414A20686F726C6F6765205224
:10DEEE0054432028656E206D6F64652073706F6FCC
:10DEFE006C696E6729200D0A002E2E2E2046696E43
:10DF0E0020646520726563757020456570726F6D53
:10DF1E002064617461202820756E74696C206F66B0
:10DF2E00666574202B373129202D3E20002050723B
:10DF3E00672E656E20636F757273203A25303264DA
:10DF4E0020736F697420257320204353475F656EDD
:10DF5E005F436F7572733D25332E3266200D0A00B6
:10DF6E00202530326448253032644D2530326473BA
:10DF7E0020204D6F64653D25732020426F75636CC4
:10DF8E006520656E203D3E2025642078203130309E
:10DF9E006D5300204554415420656E7472656520A2
:10DFAE00504F525443203D30782530325820204176
:10DFBE004C313D253032782020414C323D253032D7
:10DFCE0078200D0A00207361766520746F204565F8
:10DFDE006570726F6D2040204F72675F536175766A
:10DFEE00655F506172616D5F5472617661696C201C
:10DFFE002B2037310D0A0045434F5F637367203D79
:10E00E003E25332E316620656E20456570726F6D2C
:10E01E00205472617661696C202B3234202E2E20B2
:10E02E004030253034580D0A004E52475F636F72F0
:10E03E00203D3E25332E316620656E20456570727B
:10E04E006F6D205472617661696C202B3136202EF3
:10E05E002E204030253034580D0A0048474C5F635F
:10E06E007367203D3E25332E316620656E20456553
:10E07E0070726F6D205472617661696C202B32382C
:10E08E00202E2E204030253034580D0A00434844AF
:10E09E005F6D6178203D3E25332E316620656E2002
:10E0AE00456570726F6D205472617661696C202BBC
:10E0BE0030202E2E204030253034580D0A00454198
:10E0CE0055487973203D3E25332E316620656E20EE
:10E0DE00456570726F6D205472617661696C202B8C
:10E0EE003430202E2E204030253034580D0A004575
:10E0FE005854687973203D3E25332E316620656E67
:10E10E0020456570726F6D205472617661696C2066
:10E11E002B3336202E2E204030253034580D0A0059
:10E12E004558545F6D696E203D3E25332E31662075
:10E13E00656E20456570726F6D20547261766169EF
:10E14E006C202B38202E2E204030253034580D0ACE
:10E15E0000494E54687973203D3E25332E3166209A
:10E16E00656E20456570726F6D20547261766169BF
:10E17E006C2B3332202E2E403025303458200D0A91
:10E18E00004348445F6D696E203D3E25332E316657
:10E19E0020656E20456570726F6D205472617661D8
:10E1AE00696C2B34202E2E403025303458200D0A29
:10E1BE0000696E646963653D2533642040203078C4
:10E1CE0025303458202050726F672023256420207C
:10E1DE004E616D65202563203C2D202573200D0A90
:10E1EE00002044656D616E6465204155544F5F6536
:10E1FE0074616C6F6E6E6167652064657320332089
:10E20E00736F6E64657320445331384232300D0A99
:10E21E00000D0A204C656374757265207461626C22
:10E22E00652070726F6772616D6D657320686F72B5
:10E23E006169726520656E20656570726F6D0D0A7D
:10E24E00000D0A2052617070656C20666F726D61F0
:10E25E007420203A2022553B4A4A3B4D4D3B4141CA
:10E26E003B48483B4D4D3B6A533B2322200D0A0051
:10E27E000D0A202D2D2D2044656D616E6465206480
:10E28E006520526573746175726174696F6E2020BA
:10E29E00616374697665202D2D2D2D200D0A0020C9
:10E2AE000D0A53657175656E6365206427496E6945
:10E2BE0074204C43442034783230207669612049F2
:10E2CE0032433120504346383537340D0A004E5212
:10E2DE00475F696E64203D3E256320656E2045656F
:10E2EE0070726F6D205472617661696C202B3635B9
:10E2FE00202E2E204030253034580D0A000D0A20D5
:10E30E002D2D2D2044656D616E6465206427457149
:10E31E0075616C69736174696F6E202061637469D5
:10E32E007665202D2D2D2D200D0A004346545F635A
:10E33E007367203D3E25332E316620656E20456580
:10E34E0070726F6D205472617661696C202E2E4052
:10E35E003025303458200D0A00494E545F636F72D9
:10E36E00203D3E25332E316620656E204565707248
:10E37E006F6D205472617661696C202E2E403025AF
:10E38E00303458200D0A00200D0A20457272657532
:10E39E007220536175766520506172616D6574727D
:10E3AE00657320656E2025345820736F697420259F
:10E3BE0064200D0A002041707075796572207375A6
:10E3CE0072205357362070656E64616E74203E3233
:10E3DE0073656320706F75722076616C6964657207
:10E3EE000D0A00204020646563696D616C20232551
:10E3FE0034752020736F69742040446576696365B7
:10E40E00203762697473203D2030582530325820F1
:10E41E0000205052473D787820202050726F67724E
:10E42E00616D6D6520656E20636F757273207878EF
:10E43E003D203030206120313120200D0A00204552
:10E44E00746174204272756C657572204252553D2E
:10E45E0030206F7520312028706F757220746573AF
:10E46E0074206F6E6C7929200D0A0020417474653A
:10E47E006E74652072656C61636865205357362033
:10E48E002E2E7075697320617070756920737572A8
:10E49E0020535736200D0A000D0A2043686F697805
:10E4AE002064752050726F6772616D6D6520706F9C
:10E4BE007572206C65206A6F75722063686F697360
:10E4CE0069203A2000204368617267656D656E743D
:10E4DE002063617261637465726573205370656346
:10E4EE00696175782020656E20434752414D0D0AB3
:10E4FE000020496E6974206574207465737420540D
:10E50E00696D657236202020382078203530306DC8
:10E51E0053200D0A2053746172740D0A0020436F4C
:10E52E006D70696C656420257320617420257320DD
:10E53E00555443202076657273696F6E20584338A8
:10E54E00203A2564200D0A002063617220466C611A
:10E55E00672052756E204F6E63653D302C20666FBE
:10E56E0072636520656E7375697465206120393933
:10E57E000D0A00204241563D78782020206D6F64B0
:10E58E006520426176617264206176656320783D14
:10E59E003030206120313920200D0A000D0A20462E
:10E5AE006F726365204C65645F436C69676E6F7450
:10E5BE0065313020506F72744120202D3E2025642D
:10E5CE0020200D0A002045727265757220616472FA
:10E5DE006573736520456570726F6D203A20253026
:10E5EE00345820736F6974202564200D0A00535728
:10E5FE00312B53573320202062617363756C652075
:10E60E00486F72732047656C206F75204E6F726D68
:10E61E00616C290D0A002046696E204175746F20C9
:10E62E006574616C6F6E6E616765203320736F6EFB
:10E63E0064657320445331384232300D0A0053570B
:10E64E003220496E637220636F6E7369676E652048
:10E65E00666F72636565202045434F203A2025334F
:10E66E002E32660D0A003C5357314C3E204D6F64DE
:10E67E0069662E2050726F6772616D652023256466
:10E68E00203D3E28256329202025730D0A00496E62
:10E69E00745F6D65733D25332E3166B04320204E79
:10E6AE0052473D256320494E545F636F723D2533BB
:10E6BE002E3166B04300200D0A2053617576652019
:10E6CE00506172616D657472657320656E202534BC
:10E6DE005820736F6974202564200D0A000D0A20DE
:10E6EE00205452414954454D454E542064656D6148
:10E6FE006E646520657175616C69736174696F6EA6
:10E70E00200D0A00535732204445637220636F6E0A
:10E71E007369676E6520666F726365652045434F4A
:10E72E00203A2025332E31660D0A005357332044EC
:10E73E0065637220636F6E7369676E6520666F72B4
:10E74E0063656520434654203A2025332E31660DED
:10E75E000A0053573220496E637220636F6E7369DD
:10E76E00676E6520666F7263656520434654203A76
:10E77E002025332E32660D0A0020546573742070E6
:10E78E00726573656E636520646576696365732073
:10E79E007375722042757320493243310D0A002081
:10E7AE004D65737572657320697373756573206437
:10E7BE0065206C27204567616C69736174696F6EA3
:10E7CE00203A0D0A00204D65737572657320332053
:10E7DE0074656D70657261747572657320436F72C6
:10E7EE00726967656573203A0D0A0020536175766C
:10E7FE006520205461626C652050726F6772616D86
:10E80E006D6174696F6E5F486F7261697265202009
:10E81E00000D0A457272657572204A6F757220532B
:10E82E00656D61696E65206A532E28302061203631
:10E83E002021290D0A000D0A20457272657572207D
:10E84E007361697369652076616C657572206465A4
:10E85E0020426176617264200D0A0020566572694D
:10E86E00662E204E6F7576656C6C652044617465FE
:10E87E00206574204865757265205254430D0A0058
:10E88E0020693D25326420206F6666736574206AA8
:10E89E003D25326420746D705B2532645D3D2530FC
:10E8AE0032580D0A0020693D256420416666656375
:10E8BE00746174696F6E20486562646F20647520A0
:10E8CE00257320203D25640D0A0020496E697420B1
:10E8DE00657420746573742054696D6572362020DA
:10E8EE004E3D30200D0A2053746172740D0A0020C3
:10E8FE005265746F7572204D6F6465204E6F726D28
:10E90E00616C202C466F7263616765204D6F646584
:10E91E00203D20000D0A204E65772074696D65201C
:10E92E0020486F75723D253364204D696E753D2507
:10E93E00336420200D0A0053656C656374696F6E35
:10E94E00206A6F7572203A2025732028706172201C
:10E95E00646566617574290D0A0020536F727469BF
:10E96E0065207669612054696D656F75742031304C
:10E97E00736563206F75205357340D0A00204D6563
:10E98E00737572657320332074656D706572617472
:10E99E007572657320627275746573203A0D0A0084
:10E9AE0020736920484D3D30303A30302020757349
:10E9BE0061676520525443207265616374697665A0
:10E9CE000D0A006E6577205254432025303278258B
:10E9DE00303278253032782530327825303278252D
:10E9EE003032780D0A002054312E494E54455220B3
:10E9FE003D2025352E336625632043202054316378
:10EA0E006F723D25322E3366002054322E455854F7
:10EA1E002020203D2025352E3366256320432020DF
:10EA2E005432636F723D25322E3366002054332EDE
:10EA3E004541552020203D2025352E336625632067
:10EA4E004320205433636F723D25322E33660020EF
:10EA5E0023312041637469766520736F7274696522
:10EA6E0020525443205351573D31487A3A200D0AD3
:10EA7E0000205072673A202573202C4D6F64653D3F
:10EA8E00253264202C2025303264482530324D202A
:10EA9E000D0A0020536F72746965204D656E7520E6
:10EAAE0073757220535730206F752054696D654F02
:10EABE0075740D0A00706F75722025733A204368C5
:10EACE006F69782070726F6772202325642020286A
:10EADE002563290D0A006D6F646966792025303231
:10EAEE00782530327825303278253032782530321C
:10EAFE00782530327820002061647265737365204A
:10EB0E004C43443D20256420736F69742030582592
:10EB1E00303258200D0A0053573461292041666661
:10EB2E006563746174696F6E205072672061752021
:10EB3E006A6F75720D0A0053656C6563742E2050F2
:10EB4E00726F67722E20232564203D3E20256320A0
:10EB5E00202025730D0A00205072673A202573205D
:10EB6E002C4D6F64653D253264202C202530326497
:10EB7E00482530324D20005357346229204D6F64A2
:10EB8E0069662E2050726F6772616D20486F7261D8
:10EB9E006972650D0A006E65772070726F67206569
:10EBAE006E20636F757273202025336420202563D9
:10EBBE00200D0A00202042703D203078253032583A
:10EBCE002C20204475726565203D20253564200D6E
:10EBDE000A0046696E20646520736175766567610B
:10EBEE0072646520656E20656570726F6D0D0A002A
:10EBFE002052656C6563747572652064617461730F
:10EC0E0020656570726F6D203A200D0A0020466CEB
:10EC1E0061672052756E204F6E63652061742040CF
:10EC2E0020307830303030203D002044656D692032
:10EC3E00486575726520656E20636F757273203D31
:10EC4E00202564200D0A005357312B5357322020B4
:10EC5E00436F6E74726F6C6520436861756469658D
:10EC6E0072653D00496E7425332E3166202563256D
:10EC7E00312E31662563253273256325332E316699
:10EC8E00002054656D70203120636F727269676564
:10EC9E00653D2025352E336620200D0A0020546553
:10ECAE006D70203220636F7272696765653D202535
:10ECBE00352E336620200D0A002054656D702033EA
:10ECCE0020636F7272696765653D2025352E336648
:10ECDE0020200D0A00207361766520746F20656513
:10ECEE0070726F6D204036382C36392C37310D0A44
:10ECFE0000204D6F646520656E20636F7572733DE5
:10ED0E0020253264202D3E2025730D0A00316572B8
:10ED1E0065207365726965204D6573757265732024
:10ED2E006272757465730D0A00456570726F6D20A1
:10ED3E0032344C43787878203235366B206F75201C
:10ED4E003531324B0043616C63756C206465732002
:10ED5E00636F7272656374696F6E73203A0D0A0089
:10ED6E000D0A204D454E5531302E3220434F4D5019
:10ED7E00454E534154494F4E0D0A00693D256420BE
:10ED8E0040456570726F6D203078253458202D3EC9
:10ED9E002025640D0A0020436F6E66696720657436
:10EDAE0020496E6974204F6E6520576972650D0A91
:10EDBE00006174203078253458202D3E20202564A3
:10EDCE0020203078253032580D0A000D0A204D458E
:10EDDE004E5531302E33204C696D69746573204366
:10EDEE0048440D0A002053573120546F6F676C65ED
:10EDFE00204368616E6765204D6F64650D0A0020C3
:10EE0E0052414D207A6F6E6520506172616D2054B3
:10EE1E0072617661696C0D0A000D0A2E2E66696E9E
:10EE2E0020646520726573746175726174696F6EAA
:10EE3E000D0A00256325633A2563256320202020D3
:10EE4E00484F52532047454C20202020002050434D
:10EE5E00463837353420666F72204C434420327862
:10EE6E00313663617273000D0A204D454E553130B7
:10EE7E002E3420485953544552455349530D0A00D8
:10EE8E000D0A204D454E5531302E3120434F4E53F5
:10EE9E0049474E45530D0A20002531632025632531
:10EEAE006320202020202020202020202020202011
:10EEBE002000256325633A25632563206D202020DD
:10EECE0020202020202020202020002531632025F6
:10EEDE0063256320616D202020202020202020200B
:10EEEE0020202000256325633A25632563202020FA
:10EEFE00415252455420544F54414C200025316309
:10EF0E0020256325632053544152543D5357314CB1
:10EF1E002B5357324C00204D6F64652025732063B0
:10EF2E006F6E7369676E653D2025332E3166004521
:10EF3E0063726974757265204453333233312E2EE9
:10EF4E002E204F4B0D0A00204D656E753D2025334A
:10EF5E0064204D5061733D20253364200D0A00203E
:10EF6E004574617420616C61726D65732030582533
:10EF7E00303278200D0A002052414D207A6F6E6596
:10EF8E0020506172616D205553494E450D0A000D9A
:10EF9E000A536F727469652053573461204E6F7235
:10EFAE006D616C650D0A0020414C313D25316420A8
:10EFBE0020414C323D25316420202020202000208D
:10EFCE0054656D7065726174757265204453333289
:10EFDE003331203D3E20002042503D305825303206
:10EFEE00582C2020204D656E753D2533642000542D
:10EFFE00312025332E3266256320636F72723D25D4
:10F00E00322E326625630054322025332E32662589
:10F01E006320636F72723D25322E32662563005473
:10F02E00332025332E3266256320636F72723D25A1
:10F03E00322E32662563004578742025332E3166D4
:10F04E00202020456175202532642F253264002052
:10F05E005265736574204D4355203A205265736591
:10F06E007420200D0A000D0A2052657365742076F7
:10F07E006F6C6F6E7461697265200D0A00204172AB
:10F08E006D6520696E74657272757074696F6E73DA
:10F09E00200D0A000D0A2031302073656320656350
:10F0AE006F756C6565202E2E0D0A00204541555F4B
:10F0BE006D6573203D2025352E3266202563430D68
:10F0CE000A0020536F727469652076696120535768
:10F0DE00303E317365630D0A0045787425332E3149
:10F0EE0066202020456175202532642043202000B3
:10F0FE004348446D696E3E25322E316620202053E2
:10F10E00656C2053312000494E54636F723E2025AA
:10F11E00332E3166202053656C2E533120000D0A9C
:10F12E0056657269662030782530345820204E6F2F
:10F13E006D203A20004578742025332E316620202C
:10F14E00204561752025326420432000496E7420CD
:10F15E0025332E31662020204373673D25332E3113
:10F16E006620004E5247636F72202025332E316683
:10F17E00202B2D2053322F5333004558546879736A
:10F18E00202025332E3166202B2D2053322F533342
:10F19E0000436F6E74656E75204C69676E65202333
:10F1AE0033204C4344203A00454155687973202062
:10F1BE0025332E316620536176652053344C00453D
:10F1CE00787425332E316620202045617520253236
:10F1DE00642F25326400414C313D256320414C3271
:10F1EE003D256320646973706172756500206174DA
:10F1FE00203078253458202D3E202025332E32669F
:10F20E000D0A002050726F6772616D6D6520766514
:10F21E007273696F6E203A200020496E6974205413
:10F22E00696D657232203130306D53200D0A000D3C
:10F23E000A2048656C7020436F6D6D616E64657356
:10F24E00203A0D0A0020496E69745F49324328291D
:10F25E00203130304B687A3B0D0A00496E697420BC
:10F26E0054696D6572203420302E357365630D0A36
:10F27E000021414C41524D4520434841554449459A
:10F28E0052452120720A00496E742025332E3166B4
:10F29E002020202020202020202020200020207030
:10F2AE006F75722076616C69646572202020202053
:10F2BE002020002020417070757965722073757260
:10F2CE002053573620202020002056616C6964653B
:10F2DE007220706172205357344C20202020002061
:10F2EE002070656E64616E74203E2032205365631B
:10F2FE0020202020005072673A256320404565701B
:10F30E00726F6D2030782534582000205461626C65
:10F31E0065202325336420707267723A202563209E
:10F32E0000494E546879733E2025332E31662020D5
:10F33E0053656C2053310045434F6373672025326C
:10F34E002E3166202B2D2053322F53330043484449
:10F35E006D61782025322E3166202B2D2053322FD1
:10F36E00533300205431422E494E542E20203D203E
:10F37E0025352E336625634300205432422E4558E0
:10F38E00542E20203D2025352E3366256343002044
:10F39E005433422E45415520202E3D2025352E3307
:10F3AE0066256343004558546D696E202D253264E1
:10F3BE002020536176652053344C004E5247696EBF
:10F3CE006420202563202020736176652053344C01
:10F3DE000048474C6373672025322E3166207361D7
:10F3EE0076652053344C002048657572652025647F
:10F3FE002070726F67723D25640D0A000D0A536FFF
:10F40E00727469652020414E6F726D616C650D0AD4
:10F41E000054312E494E542E202020202020202012
:10F42E0020202020200054322E4558542E202020FB
:10F43E00202020202020202020200054332E454143
:10F44E00552E20202020202020202020202020008B
:10F45E002B2D53322F5333202020202020202020EC
:10F46E0020202020007361766553344C202020200C
:10F47E0020202020202020202000565241492053B9
:10F48E00314C20202020202020202020202000521F
:10F49E00656C6163686572205357362020202020EA
:10F4AE002020200020466F7263616765204D6F64D7
:10F4BE006520202020202020004D414A2052544318
:10F4CE002044533332333120202020202000646129
:10F4DE006E7320456570726F6D2050494320202059
:10F4EE0020200070756973204250205245534554B8
:10F4FE00202E2E2E2020200052656D6574747265AC
:10F50E0020656E20706C61636520202000536F7241
:10F51E007469652070726576656E746976652020F3
:10F52E0020002E2E2E506173206465204D414A20FE
:10F53E005254432120200053617576652020636F5D
:10F54E007272656374696F6E73202000202041749F
:10F55E0074656E7465204250205265736574202068
:10F56E00002021414C41524D4520434841554449CC
:10F57E0045524521200044656D616E6465206176BB
:10F58E006F7274656520212E2E20002046494E2E66
:10F59E002E2E4F4B2E2E2E2E2E2E2E2E2E2E20007B
:10F5AE0056616C696461742E204F4B20706172201D
:10F5BE005357352000536175766567617264652017
:10F5CE0064616E73205254432000736F72746965C8
:10F5DE00204D656E75203462202E2E4F4B20006D0F
:10F5EE006F64656C652041414D4D4A4A78534848D9
:10F5FE004D4E200044656D616E6465204547414C5B
:10F60E0049534154494F4E200065747265206C6910
:10F61E0065657320656E73656D626C652000206490
:10F62E00657320736F6E64657320526571756973AF
:10F63E00652000205265746F7572204D6F646520D1
:10F64E004E6F726D616C20007361766553344C2081
:10F65E002043686F6978204A6F7572200045746187
:10F66E006C6F6E6E616765203320536F6E646573C9
:10F67E00200033204D65737572657320636F72724F
:10F68E0069676565732000204C657320736F6E6427
:10F69E00657320646F6976656E74200043617261D4
:10F6AE006374657265732053706563696175782044
:10F6BE000056657273696F6E2043617274652050D7
:10F6CE004342202021002120506172616D657472C9
:10F6DE006573205553494E452021002120526569FE
:10F6EE006E697469616C69736174696F6E20210053
:10F6FE0052455041524154494F4E2044454D414E82
:10F70E0044454521005645494C4C455553452043EB
:10F71E0048415544494552452100505245535320C6
:10F72E004541552043484155444945524521002DF8
:10F73E002D2D2D2D2D2D2D2D2D2D2D2D2D2D2D2DEB
:10F74E002D2D2D002B2D53322F53332053656C2E20
:10F75E00486575726520202E004C6573203320732A
:10F76E006F6E646573204453313842323000434625
:10F77E00546373673E25322E3166202053656C200C
:10F78E0053310020494E545F6D6573203D20253561
:10F79E002E32662563204300204558545F6D6573F5
:10F7AE00203D2025352E326620256343003130332F
:10F7BE004C696D69746573202065786974205330C7
:10F7CE004C00313032436F6D70656E73202065785A
:10F7DE0069742053304C00313031436F6E7369675A
:10F7EE006E6520657869742053304C003130344892
:10F7FE007973746572657320657869742053304C23
:10F80E00005357322B5357332041435155495420FF
:10F81E00414C41524D004E6F7576656C6C652045BE
:10F82E0047414C49534154494F4E0056616C6964EF
:10F83E00657220706172205357363E3273656300D5
:10F84E0043686F69783D5357312C5357314C3D56B1
:10F85E00616C6964004547414C49534154494F4ED0
:10F86E00207465726D696E6565004D6F64696669B9
:10F87E00652050726F672E486F7261697265002045
:10F88E004D6F6469662050726F67722E486F726199
:10F89E0069726500535720303C20313E20322B20B8
:10F8AE00332D20353D56616C005072672020207339
:10F8BE006176656420746F204570726F6D0020460E
:10F8CE00494E206465207265737461757261746946
:10F8DE006F6E0020526573756C7473204567616C92
:10F8EE0069736174696F6E007361766553344C2071
:10F8FE002053617576652050726F677200535731D1
:10F90E00204368616E67652076616C2050726F6768
:10F91E0072005357314C2076616C69642E53656CBE
:10F92E002050726F6772007361766553344C2020DD
:10F93E0043686F69782050726F6772002B2D5332B7
:10F94E002F5333202053656C65632E50726F677290
:10F95E00003E204166666563742050726F67722D9B
:10F96E003E4A6F75720033204D65732E4453313805
:10F97E00423230204272757465730044656C616961
:10F98E00205357362074726F7020636F7572740037
:10F99E0045786974204D656E7534202F2054696D3D
:10F9AE00654F757400536974756174696F6E20418B
:10F9BE005052455320200D0A0053697475617469C5
:10F9CE006F6E204156414E5420200D0A004166664E
:10F9DE006563746174696F6E5F486562646F0D0A6A
:10F9EE0000204D454E553420766961205357344CD6
:10F9FE002020202000202020526573657420416C49
:10FA0E0061726D65202020200044656D616E646515
:10FA1E00204163636570746565202E2E0020426F51
:10FA2E0075636C6520737572204D656E7531302E61
:10FA3E000073617665206D6F6469662050726F6722
:10FA4E0072616D2E002054312E494E542E203D20D1
:10FA5E0025352E3366256343002054322E455854E7
:10FA6E002E203D2025352E3366256343002054334A
:10FA7E002E4541552E203D2025352E3366256343D8
:10FA8E0000204D4F59454E4E45203D2025352E33F5
:10FA9E006625634300204541555F6D6573203D200B
:10FAAE0025352E33662563430020436F6E736967D9
:10FABE006E653D2025332E32660D0A0020494E54C8
:10FACE005F6D65733D2025352E336625634300201B
:10FADE004558545F6D65733D2025352E336625637D
:10FAEE0043005043463835373441203862697473C9
:10FAFE0020492F4F00204475726565204170707546
:10FB0E0069203A2025356400204D414A2052544345
:10FB1E0020766961203A200D0A00204D656D6F2018
:10FB2E0064616E7320525443200D0A00494E545F97
:10FB3E0063626C3D2025332E3266200D0A00205064
:10FB4E00726573656E746174696F6E203A0D0A008A
:10FB5E0020494E545F6D65733D2025332E31660D61
:10FB6E000A00204475726565203D202564206D5382
:10FB7E00202C2000204465636F646167652054610A
:10FB8E00626C65202300204272756C6575723D2093
:10FB9E004F464620282329004C4344203231313928
:10FBAE00203278313663617273005265736574204A
:10FBBE00416C61726D6573200D0A00205265746F81
:10FBCE007572204D656E753D300D0A00204F6666CC
:10FBDE007365743D2025332E32660D0A0020466F64
:10FBEE007263616765204D6F6465203D2000204281
:10FBFE0072756C6575723D204F4E20282429005079
:10FC0E0043463835373420386269747320494F00C3
:10FC1E0056616C69642E206D6F646966200D0A0052
:10FC2E004572726575722063686F6978200D0A00DF
:10FC3E002063686F69782076616C69642E0D0A0006
:10FC4E00204541555F63626C3D202533640D0A00EB
:10FC5E002050656E74653D2025332E32660D0A00E8
:10FC6E00205431436F723D2025352E33660D0A0028
:10FC7E00205432436F723D2025352E33660D0A0017
:10FC8E00205433436F723D2025352E33660D0A0006
:10FC9E002020415252455420544F54414C202000B4
:10FCAE0050726F6720656E20636F757273203A0015
:10FCBE00454550524F4D203531326279746573008F
:10FCCE000D0A2053746570203D2564200D0A0067CF
:10FCDE006F746F2044656275745F310D0A00676F33
:10FCEE00746F2044656275745F330D0A00676F741C
:10FCFE006F2044656275745F340D0A002043617293
:10FD0E007465205061756C203A2000205245544F86
:10FD1E005552204E4F524D414C000D0A5357312033
:10FD2E006D6F6469662009000D0A204D414A20520C
:10FD3E005443200D0A000D0A54494D45204F555489
:10FD4E00210D0A0053656C6563742E3A2025730DE0
:10FD5E000A00202D2D3E20454550524F4D202000AB
:10FD6E004E5247636F722A2025332E316600494E5C
:10FD7E0054636F722A2025332E316600494E544843
:10FD8E0079732A2025332E316600455854487973ED
:10FD9E002A2025332E3166004541554879732A2095
:10FDAE0025332E3166004558546879732A20253341
:10FDBE002E316600256325633A25632563206D2069
:10FDCE0000536F72746965204D656E75200045583D
:10FDDE00546D696E2A2D2532642E0048474C63738C
:10FDEE00672A2532642E30004F4C4544205353442D
:10FDFE0031333036006E6F6E20726563656E731B25
:10FE0E0039004348446D696E2025322E3166004319
:10FE1E0048446D61782025322E31660045434F638C
:10FE2E0073672A25322E3166004346546373672A60
:10FE3E0025322E3166006465203030682061203016
:10FE4E0031680020204E4F524D414C202020002082
:10FE5E005245544F555220412020004F63742020AC
:10FE6E003420323032340009506C616765203142E3
:10FE7E00203A0009506C616765203242203A000931
:10FE8E00506C616765203342203A0009506C6167FF
:10FE9E0065203148203A0009506C61676520324870
:10FEAE00203A0009506C616765203348203A0025DE
:10FEBE003163202563256320616D00204873656CD6
:10FECE003D25640D0A00203078253032582C202034
:10FEDE000054494D45204F5554212000204D6F644C
:10FEEE00652020257320005254432044533332336F
:10FEFE0031004C45445F436C6931303D004E5247F2
:10FF0E00696E642A202563004A537465703D300D76
:10FF1E000A0048537465703D310D0A004A537465EA
:10FF2E00703D310D0A0050537465703D310D0A005D
:10FF3E004A537465703D320D0A0050537465703D1E
:10FF4E00320D0A004A537465703D330D0A004A5350
:10FF5E007465703D350D0A004A537465703D340961
:10FF6E00002048656C70200D0A0025332E32662065
:10FF7E004320005357312020204D200031313A309C
:10FF8E00383A323300486F72735F47656C00205306
:10FF9E00746F700D0A0025332E3266204300202028
:10FFAE00202020414D007078203A2020002025305E
:10FFBE0035642000323431303034005265637520A0
:10FFCE003A004E6F726D616C0020474F0D0A002093
:10FFDE006F6B0D0A00494E46004E414E00696E662B
:10FFEE00006E616E006C6C7300202E31006C66002A
:01FFFE000002
:020000040001F9
:10000000600E3901D96F000EDB6F000EDD6F080E38
:10001000DF6F000EDE6F290E01016D6F960E6C6FA3
:100020007F0EE82EFED76C2FFCD76D2FFAD7D29E0D
:10003000000E3A01456F000E466F000E476F000E2E
:10004000656F000E666F000E676F000E556F000E35
:10005000566F3901909FD2909191A09FA19101017B
:10006000BC9F87ECF5F0400E3D01EA6F000E0101E8
:10007000D16F000ED06FD1510FE1800ED05DD8B09E
:100080000BD0000ED025D96E050ED121DA6E000EF0
:10009000DF6ED04BD12BEFD7000ED16F000ED06F9B
:1000A000D1510FE1800ED05DD8B00BD0800ED0259D
:1000B000D96E050ED121DA6E000EDF6ED04BD12B3A
:1000C000EFD7000ED16F000ED06FD1510FE17F0E30
:1000D000D05DD8B00BD01E0ED025D96E030ED12125
:1000E000DA6E000EDF6ED04BD12BEFD7000ED16F42
:1000F000000ED06FD1510FE13F0ED05DD8B00BD0C4
:100100009E0ED025D96E030ED121DA6E000EDF6E61
:10011000D04BD12BEFD7000ED16F000ED06FD15145
:100120000FE1090ED05DD8B00BD0AF0ED025D96E3F
:10013000020ED121DA6E000EDF6ED04BD12BEFD73D
:10014000000EA86F050EA96F000E066E000E056E5C
:10015000000EB76F000EB96F010EBB6F000E0201EB
:10016000A66FFEEC04F0290E01016D6F960E6C6F08
:100170007F0EE82EFED76C2FFCD76D2FFAD732EC0E
:100180000CF0A20E2B6EDC0E2C6E78EC06F0000E3E
:100190000101B26F000E066E000E056E260E3D01C7
:1001A000EA6F20D0090E01016D6F1E0E6C6FE40E18
:1001B000E82EFED76C2FFCD76D2FFAD700F005C0C4
:1001C00025F006C026F0000E286E050E276EF6EC10
:1001D00005F025502610D8B4BA7C2E0E4AEC0CF04F
:1001E000054A062A6F0030FF6CF1050E01016D6FA4
:1001F000D8906C336D2FFCD76CB106D0065004E15B
:10020000640E055CD8A0CED7A8C124F1A9C125F100
:10021000030E266FFB0E276F05C028F106C029F1DB
:10022000F0EC03F0A8C125F0A9C126F08EECFBF09C
:1002300032EC0CF0065004E1150E055CD8A00CD091
:1002400006500AE1320E055CD8B006D0450EEA6FC2
:10025000010E0101B26FBA8C000E0201976F0650B9
:1002600004E1330E055CD8A00DD006500BE1500E12
:10027000055CD8B007D0520E3D01EA6F010E0201B5
:10028000976FBA8C000E066E000E056E4C0E2B6E2C
:10029000FB0E2C6E78EC06F0000E0101D16F000E03
:1002A000D06FD15119E1090ED05DD8B015D0D890DA
:1002B000D035D96ED135DA6EE70ED926040EDA22A2
:1002C0006F0078FF2BF06F0074FF2CF078EC06F0D5
:1002D0000101D04BD12BE5D732EC0CF0A8C124F1B1
:1002E000A9C125F12B0E0101266FE50E276F690EBE
:1002F000286FFE0E296F8A0E2A6FFF0E2B6F090ED4
:100300002D6F380E2C6FF0EC03F0A8C125F0A9C1B9
:1003100026F08EECFBF032EC0CF00101B205D8A413
:1003200008D00B0E2B6EE30E2C6E78EC06F032EC40
:100330000CF002019705D8A408D07E0E2B6EE20EB9
:100340002C6E78EC06F032EC0CF0000E01015A6FC6
:10035000000E596FA2ECFEF0116E1E0E256E030EFC
:10036000266EC20E276EFF0E286E39EC01F0000ECD
:10037000266E010E256E1EC327F0EBEC02F0000E78
:10038000266E020E256E1FC327F0EBEC02F0000E66
:10039000266E030E256E20C327F0EBEC02F0000E54
:1003A000266E040E256E21C327F0EBEC02F0000E42
:1003B000266E050E256E22C327F0EBEC02F0000E30
:1003C000266E060E256E23C327F0EBEC02F0000E1E
:1003D000266E070E256E000E276EEBEC02F0630E04
:1003E0001118D8B459D11E0E256E030E266EC20EFA
:1003F000276EFF0E286E39EC01F0000E266E010EFE
:10040000256E1EC327F0EBEC02F0000E266E020EE6
:10041000256E1FC327F0EBEC02F0000E266E030ED4
:10042000256E20C327F0EBEC02F0000E266E040EC2
:10043000256E21C327F0EBEC02F0000E266E050EB0
:10044000256E22C327F0EBEC02F0000E266E060E9E
:10045000256E23C327F0EBEC02F0000E266E070E8C
:10046000256E000E276EEBEC02F0770E2B6EDB0E86
:100470002C6E78EC06F0560E2B6EE50E2C6E78EC9A
:1004800006F0000E0101D16F000ED06FD15105E1D1
:100490000A0ED05DD8B0D7D001D0D5D0000E0A6EEC
:1004A000000E096E0A505FE1180E095CD8B05BD0EF
:1004B000D0C16CF1D1C16DF1050ED89001016C373E
:1004C0006D37E82EFAD709506C270A506D23A00E1D
:1004D0006C25076E000E6D21086ED0C16CF1D1C184
:1004E0006DF1050ED8906C376D37E82EFBD7260ED0
:1004F0006E6F060E6F6F6C516E276D516F23095032
:100500006E25D96E0A506F21DA6EDF50116E07C06A
:1005100025F008C026F011C027F0EBEC02F01150D6
:10052000300F4AEC0CF0D0C16CF1D1C16DF1050E69
:10053000D89001016C376D37E82EFAD709506C2737
:100540000A506D23500E6C25076E020E6D21086E49
:1005500007C025F008C026F011C027F0EBEC02F030
:10056000094A0A2A9FD7200E4AEC0CF0200E4AECCA
:100570000CF0000E0A6E180E096E0A505EE1200E95
:10058000095CD8B05AD0D0C16CF1D1C16DF1050E63
:10059000D89001016C376D37E82EFAD709506C27D7
:1005A0000A506D23A00E6C25076E000E6D21086E9B
:1005B000D0C16CF1D1C16DF1050ED8906C376D379B
:1005C000E82EFBD7260E6E6F060E6F6F6C516E27EE
:1005D0006D516F2309506E25D96E0A506F21DA6E66
:1005E000DF50116E07C025F008C026F011C027F0BB
:1005F000EBEC02F011504AEC0CF0D0C16CF1D1C11F
:100600006DF1050ED89001016C376D37E82EFAD7E1
:1006100009506C270A506D23500E6C25076E020E90
:100620006D21086E07C025F008C026F011C027F024
:10063000EBEC02F0094A0A2AA0D732EC0CF00101D7
:10064000D04BD12B23D7000E5A6F500E596F60EC50
:10065000DDF0020E01015A6F000E596F60ECDDF003
:10066000D5ECFFF0E00E2B6EEB0E2C6E78EC06F066
:10067000000E266E000E256E630E276EEBEC02F068
:10068000030E01016D6F080E6C6F770EE82EFED71A
:100690006C2FFCD76D2FFAD7510E2B6EDD0E2C6E02
:1006A00078EC06F0000E0101686F500E676F29ECC0
:1006B000D8F02C0E2B6EDC0E2C6E78EC06F0A8EC2D
:1006C000F3F0DB0E2B6EF90E2C6E78EC06F0000EBC
:1006D0000101D16F000ED06FD15136E1080ED05D0F
:1006E000D8B032D01E0E246F030E256FB30E266FC6
:1006F000E80E276FD0C128F1D1C129F1D890D035AB
:10070000D96ED135DA6EC50ED926020EDA226F0007
:1007100078FF2AF16F0074FF2BF1D50ED025D96E2A
:10072000020ED121DA6EDF506C6F6C512C6F2D6B85
:10073000F0EC03F01E0E256E030E266E8EECFBF021
:100740000101D04BD12BC8D732EC0CF06C0E2B6EC4
:10075000D80E2C6E78EC06F0530E2B6EF20E2C6E2B
:1007600078EC06F0F6EC0AF0870E2B6EE70E2C6E96
:1007700078EC06F0DDECE5F032EC0CF05D0E2B6E63
:10078000EA0E2C6E78EC06F0D70E2B6EFF0E2C6E58
:1007900078EC06F0400E0201AF6F0E0E3A6EAFC25B
:1007A0003BF0680E5FEC02F0DD0E2B6EFF0E2C6E40
:1007B00078EC06F0090E01016D6F1E0E6C6FE40EF1
:1007C000E82EFED76C2FFCD76D2FFAD700F0020E63
:1007D0006BECF1F0090E01016D6F1E0E6C6FE40EF3
:1007E000E82EFED76C2FFCD76D2FFAD700F0CD0E78
:1007F0002B6EEF0E2C6E78EC06F0000E90ECF7F0FE
:10080000B90E256E020E266E8EECFBF032EC0CF06B
:10081000200E0101CD6F000E586E140E576E1E0E85
:10082000246F030E256F050E266FEB0E276FCDC1CB
:1008300028F1296BCDC12AF12B6BF0EC03F01E0ED1
:10084000256E030E266E8EECFBF03D017589AD0E14
:100850002B6EE20E2C6E78EC06F03D01738F4FECA0
:10086000EEF032EC0CF0010EDDECFBF0010E0001BD
:100870006B6FBF0E6C6FF60E6D6F6C516D11D8A45F
:10088000000E6E6F010E3AEC0BF0020E8EEC05F0CE
:10089000010EDDECFBF0020EDDECFBF0090E0101B8
:1008A0006D6F1E0E6C6FE40EE82EFED76C2FFCD71A
:1008B0006D2FFAD700F0D30E2B6EE40E2C6E78EC71
:1008C00006F0AA0E0001636FF60E646F63516411A7
:1008D000D8A4000E656FDFECF9F0000E0001666F22
:1008E000000E656F23ECF3F0000E0101D16F000ED6
:1008F000D06FD15132E1080ED05DD8B02ED0D0C12A
:100900006CF1D1C16DF1D8906C376D37D8906C37E0
:100910006D37D8906C376D37DA0E6C252B6ED40E90
:100920006D212C6E78EC06F032EC0CF0000E00011C
:10093000666F020E656F010E0101D0250001676F21
:10094000000E0101D1210001686FD0C169F0EAEC0D
:10095000FAF00101D04BD12BCCD7010E8EEC05F073
:1009600032EC0CF0A40E2B6EED0E2C6E78EC06F033
:1009700087EC08F0150E01016D6F4B0E6C6FBE0E0B
:10098000E82EFED76C2FFCD76D2FFAD700F01B0E88
:100990002B6EED0E2C6E78EC06F05AECF8F06DC074
:1009A00094F16EC095F16FC096F170C097F1A8C137
:1009B00024F1A9C125F1710E0101266FF30E276FF5
:1009C00094C128F195C129F196C12AF197C12BF163
:1009D000000E2D6FB00E2C6FF0EC03F0A8C125F0C7
:1009E000A9C126F08EECFBF032EC0CF0F5ECF7F040
:1009F0006DC090F16EC091F16FC092F170C093F133
:100A0000A8C124F1A9C125F1870E0101266FF30EBB
:100A1000276F90C128F191C129F192C12AF193C1A8
:100A20002BF1000E2D6FB00E2C6FF0EC03F0A8C16F
:100A300025F0A9C126F08EECFBF032EC0CF0BFECF7
:100A4000F8F06DC08CF16EC08DF16FC08EF170C08A
:100A50008FF1A8C124F1A9C125F19D0E0101266FD6
:100A6000F30E276F8CC128F18DC129F18EC12AF1B7
:100A70008FC12BF1000E2D6FB00E2C6FF0EC03F038
:100A8000A8C125F0A9C126F08EECFBF032EC0CF0E9
:100A9000010E8EEC05F00101B205D8A408D0EB0ED2
:100AA0002B6EE60E2C6E78EC06F09BECAAF032EC86
:100AB0000CF0DD0E2B6EDC0E2C6E78EC06F0BDEC2F
:100AC00002F01E0E0101246F030E256F6E0E266FBD
:100AD000FC0E276F70C128F171C129F172C12AF192
:100AE00073C12BF1F0EC03F01E0E256E030E266E83
:100AF0008EECFBF01E0E0101246F030E256F7E0E9F
:100B0000266FFC0E276F74C128F175C129F176C1DB
:100B10002AF177C12BF1F0EC03F01E0E256E030EC7
:100B2000266E8EECFBF01E0E0101246F030E256F66
:100B30008E0E266FFC0E276F78C128F179C129F13E
:100B40007AC12AF17BC12BF1F0EC03F01E0E256E69
:100B5000030E266E8EECFBF032EC0CF0010EF0EC86
:100B6000D9F0020E8EEC05F0000E0F6E000E0E6E28
:100B7000000E0D6E000E106E8B0E2B6EF00E2C6E96
:100B800078EC06F047EC03F03901909F000E3A0133
:100B9000866F000E556F7E0E566F000E576F39012F
:100BA000A09F0101BC9F3901A1919181D28E0201C8
:100BB0009705D8A46CD1D40E2B6ED70E2C6E78EC82
:100BC00006F0F00E2B6EDB0E2C6E78EC06F0010EAC
:100BD000DDECFBF0090E01016D6F1E0E6C6FE40E73
:100BE000E82EFED76C2FFCD76D2FFAD700F0010E40
:100BF00000016B6FE90E6C6FF60E6D6F6C516D112D
:100C0000D8A4000E6E6F010E3AEC0BF0010E00013D
:100C10006B6FD40E6C6FF60E6D6F6C516D11D8A4A6
:100C2000000E6E6F020E3AEC0BF0000E00016C6FBE
:100C3000030E6B6FA9ECF4F0090E01016D6F1E0E2F
:100C40006C6FE40EE82EFED76C2FFCD76D2FFAD711
:100C500000F0000E0101D16F000ED06FD1517BE189
:100C60000A0ED05DD8B077D01E0E246F030E256F0C
:100C7000190E266FF30E276FD0C128F1D1C129F1CB
:100C8000390ED025F66ED20ED121F76EF86A000E1D
:100C9000F8220800F5502A6F2B6BF0EC03F01E0EC3
:100CA000256E030E266E8EECFBF032EC0CF0010E7E
:100CB00000016A6F1E0E6B6F030E6C6F030EEEEC7D
:100CC0000BF0000E0A6E000E096E0A5040E1200E75
:100CD000095CD8B03CD0D0C16CF1D1C16DF1050E2A
:100CE000D89001016C376D37E82EFAD709506C2780
:100CF0000A506D23500E6C25076E020E6D21086E92
:100D000007C059F108C05AF1A2ECFEF0116ED0C133
:100D10006CF1D1C16DF1050ED89001016C376D37C2
:100D2000E82EFAD709506C270A506D23A00E6C25C7
:100D3000076E000E6D21086E07C025F008C026F072
:100D400011C027F0EBEC02F0094A0A2ABED70101D4
:100D5000D04BD12B83D732EC0CF0000E0101D16FB8
:100D6000000ED06FD15142E1030ED05DD8B03ED01D
:100D7000000E986F000E996F000E9A6F000E9B6F19
:100D8000700E6C6F010E6D6FD890D035D96ED13565
:100D9000DA6ED890D936DA366C51D9266D51DA220E
:100DA000000EDE6E000EDE6E000EDE6E000EDD6EDC
:100DB000D0C16CF1D1C16DF1D8906C376D37D8903E
:100DC0006C376D37300E6C252B6E000E6D212C6E3E
:100DD00098C12DF099C12EF09AC12FF09BC130F02F
:100DE00046EC05F00101D04BD12BBCD7010E000120
:100DF0006B6FCC0E6C6FF80E6D6F6C516D11D8A4CB
:100E0000000E6E6F010E3AEC0BF0010E00016B6FDD
:100E1000240E6C6FF80E6D6F6C516D11D8A4000E1E
:100E20006E6F020E3AEC0BF0010E00016B6F2C0E90
:100E30006C6FF60E6D6F6C516D11D8A4000E6E6F55
:100E4000030E3AEC0BF0010E00016B6F5A0E6C6F43
:100E5000F50E6D6F6C516D11D8A4000E6E6F040EFF
:100E60003AEC0BF0270E2B6EEE0E2C6E78EC06F0A3
:100E7000BA78090E01016D6F1E0E6C6FE40EE82E3C
:100E8000FED76C2FFCD76D2FFAD700F0F1D732ECDC
:100E90000CF01F0E2B6EE20E2C6E78EC06F0000E9E
:100EA00020ECE2F00101BA51EAECE6F032EC0CF091
:100EB000980E0101C525D96EDA6A040EDA22DF50D8
:100EC000B56FEEEC9DF0010E8EEC05F0690E2B6E09
:100ED000F20E2C6E78EC06F058EC06F032EC0CF0CA
:100EE000A08ED28E32EC0CF0D80E2B6EE80E2C6E4B
:100EF00078EC06F0000E68EC04F00101BCABFDD705
:100F0000BC9B9C0E2B6EFF0E2C6E78EC06F0FF0E39
:100F10002B6EE40E2C6E78EC06F0080E68EC04F0F4
:100F20000101BCABFDD7BC9B9C0E2B6EFF0E2C6E43
:100F300078EC06F0B2EC05F0270E2B6EF20E2C6E5C
:100F400078EC06F0C30E2B6EDD0E2C6E78EC06F0FE
:100F5000B2EC05F0000E0201766F000E756F000E08
:100F60000F6E000E0E6E000E0D6E3901A3AF06D08F
:100F7000A20E2B6EF00E2C6E78EC06F0000E22EC1A
:100F800005F00101C251D8A416D0A8C124F1A9C10D
:100F900025F1BB0E266FFF0E276F87C228F188C28E
:100FA00029F1F0EC03F0A8C125F0A9C126F08EECE0
:100FB000FBF032EC0CF00101BF51D8A408D0C205FF
:100FC000D8A402D0010E01D0000E6BECF1F05AEC67
:100FD000F8F06DC076F06EC077F06FC078F070C03A
:100FE00079F070C17AF071C17BF072C17CF073C18D
:100FF0007DF099ECE0F076C0FAF177C0FBF178C0B3
:10100000FCF179C0FDF1F5ECF7F06DC076F06EC043
:1010100077F06FC078F070C079F074C17AF075C164
:101020007BF076C17CF077C17DF099ECE0F076C082
:10103000F6F177C0F7F178C0F8F179C0F9F1BFECBB
:10104000F8F06DC076F06EC077F06FC078F070C0C9
:1010500079F078C17AF079C17BF07AC17CF07BC1FC
:101060007DF099ECE0F076C0F2F177C0F3F178C052
:10107000F4F179C0F5F1030E0101C219D8A483D0AF
:10108000DAC120F6DBC121F6DCC122F6DDC123F690
:10109000A8C124F1A9C125F1240E266FEF0E276FF8
:1010A000ED0E286F030E296F20C62AF121C62BF101
:1010B00022C62CF123C62DF1F0EC03F0A8C125F0D7
:1010C000A9C126F08EECFBF032EC0CF0A8C124F1A3
:1010D000A9C125F1910E0101266FF70E276FFAC104
:1010E00028F1FBC129F1FCC12AF1FDC12BF1000E51
:1010F0002D6FB00E2C6FF0EC03F0A8C125F0A9C144
:1011000026F08EECFBF032EC0CF0A8C124F1A9C162
:1011100025F1A60E0101266FF70E276FF6C128F103
:10112000F7C129F1F8C12AF1F9C12BF1000E2D6F99
:10113000B00E2C6FF0EC03F0A8C125F0A9C126F089
:101140008EECFBF032EC0CF0A8C124F1A9C125F122
:10115000B90E0101266FF00E276FF2C128F1F3C11D
:1011600029F1F4C12AF1F5C12BF1000E2D6FB00E5B
:101170002C6FF0EC03F0A8C125F0A9C126F08EEC8D
:10118000FBF032EC0CF0000E0101A86F050EA96F08
:101190001050D8B4A3D0A8C124F1A9C125F1700E74
:1011A000266FFB0E276F05C028F106C029F1F0EC71
:1011B00003F0A8C125F0A9C126F08EECFBF0A8C170
:1011C00024F1A9C125F1E50E0101266FEF0E276F6D
:1011D00010C028F1296B0FC02AF12B6BF0EC03F043
:1011E000A8C125F0A9C126F08EECFBF0000E01018C
:1011F000D16F000ED06FD1512BE1060ED05DD8B06B
:1012000027D0D0C16CF1010E6D6F6C2B02D0D8903D
:101210006D376C2FFCD701016D51116E11501018F4
:10122000D8A412D0D0C125F0D1C126F0000E286E6E
:10123000060E276E5CEC0AF0120E25242B6ED60EDD
:1012400026202C6E78EC06F00101D04BD12BD3D7A1
:10125000000E106EBC9F32EC0CF040D01E0E01014F
:10126000246F030E256F550E266FEF0E276F0FC0EC
:1012700028F1296B0EC02AF12B6BF0EC03F01E0E47
:10128000256E030E266E8EECFBF00FD025ECB0F031
:1012900025D0F2ECBFF022D0D3ECBAF01FD095EC01
:1012A000B5F01CD0000E0E6E19D00E5001016C6FFF
:1012B0006D6B6D51000AD8A4F5D76C51000AD8B4F3
:1012C0000DD0010AD8B4E2D7030AD8B4E2D7010A94
:1012D000D8B4E2D7070AD8B4E2D7E4D70A0E0F1879
:1012E000D8B4BCD70101BB05D8A4E1EF8FF00F043F
:1012F000D8A45BD039019191A191000E106EF30E2C
:101300002B6EED0E2C6E78EC06F01E0E256E030E85
:10131000266E8EECFBF00101B751010AB76F000E8B
:10132000B96FB705D8A420D0B605D8A402D0000E56
:10133000FE6FB651D8A402D0010EFE6F010E00015F
:101340006B6FB20E6C6FF40E6D6F6C516D11D8A493
:10135000000E6E6F010E3AEC0BF0EB0E2B6EFB0ED7
:101360002C6E78EC06F015D0010E00016B6F410E6B
:101370006C6FF60E6D6F6C516D11D8A4000E6E6F10
:10138000010E3AEC0BF0FD0E2B6EE80E2C6E78EC95
:1013900006F00101B751300F4AEC0CF032EC0CF0C2
:1013A000020E8EEC05F014EC07F0020E0F18D8A414
:1013B0006ED10101B851D8A46AD139019191A1919E
:1013C000000E106E0101FE05D8A491D02B0E3D0138
:1013D000EA6FD2C186F0D3C187F0D4C188F0D5C1FD
:1013E00089F0000E00018A6F000E8B6FE00E8C6F8B
:1013F000410E8D6FF2ECF5F0D8B01AD0D2C176F074
:10140000D3C177F0D4C178F0D5C179F0000E7A6FEE
:10141000000E7B6F000E7C6F3F0E7D6F99ECE0F04D
:1014200076C0D2F177C0D3F178C0D4F179C0D5F1CC
:101430001E0E0101246F030E256F600E266FE70E4E
:10144000276FD2C128F1D3C129F1D4C12AF1D5C166
:101450002BF1F0EC03F0D2C186F0D3C187F0D4C1F8
:1014600088F0D5C189F0DEC18AF0DFC18BF0E0C120
:101470008CF0E1C18DF06AEC05F086C098F187C070
:1014800099F188C09AF189C09BF1CD0E866FCC0E80
:10149000876FCC0E886F3E0E896F98C18AF099C114
:1014A0008BF09AC18CF09BC18DF0F2ECF5F0D8B0C6
:1014B00003D0040E0201F36F98C186F099C187F042
:1014C0009AC188F09BC189F0CD0E00018A6FCC0EC5
:1014D0008B6FCC0E8C6F3E0E8D6FF2ECF5F0D8B0AA
:1014E00003D0050E0201F36F010E0101B96FFE5129
:1014F000D8A491D02B0E3D01EA6FD2C186F0D3C1A2
:1015000087F0D4C188F0D5C189F0000E00018A6F40
:10151000000E8B6F900E8C6F410E8D6FF2ECF5F01C
:10152000D8B01AD0D2C176F0D3C177F0D4C178F058
:10153000D5C179F0000E7A6F000E7B6F000E7C6FC4
:101540003F0E7D6F99ECE0F076C0D2F177C0D3F119
:1015500078C0D4F179C0D5F11E0E0101246F030EBD
:10156000256F4C0E266FE60E276FD2C128F1D3C12E
:1015700029F1D4C12AF1D5C12BF1F0EC03F0D2C18D
:1015800086F0D3C187F0D4C188F0D5C189F0DAC123
:101590008AF0DBC18BF0DCC18CF0DDC18DF06AEC30
:1015A00005F086C098F187C099F188C09AF189C08A
:1015B0009BF1CD0E866FCC0E876FCC0E886F3E0EE2
:1015C000896F98C18AF099C18BF09AC18CF09BC148
:1015D0008DF0F2ECF5F0D8B003D0040E0201F36FF9
:1015E00098C186F099C187F09AC188F09BC189F0B3
:1015F000CD0E00018A6FCC0E8B6FCC0E8C6F3E0E21
:101600008D6FF2ECF5F0D8B003D0050E0201F36F48
:10161000010E0101B96FD2C125F0D3C126F0D4C1AA
:1016200027F0D5C128F0DEC129F0DFC12AF0E0C1E2
:101630002BF0E1C12CF056ECFDF0D8A006D0000E46
:101640000101B96F200E0201F36FD2C125F0D3C1A1
:1016500026F0D4C127F0D5C128F0DAC129F0DBC1CA
:101660002AF0DCC12BF0DDC12CF056ECFDF0D8A047
:1016700006D0000E0101B96F200E0201F36F1E0E9D
:10168000256E030E266E8EECFBF014EC07F0030EB5
:101690000F18D8A46ED10101B851D8A46AD139016C
:1016A0009191A191000E106E0101FE05D8A491D078
:1016B0002D0E3D01EA6F000E0001866F000E876F50
:1016C000800E886F410E896FD2C18AF0D3C18BF032
:1016D000D4C18CF0D5C18DF0F2ECF5F0D8B01AD0B1
:1016E000D2C176F0D3C177F0D4C178F0D5C179F00A
:1016F000000E7A6F000E7B6F000E7C6FBF0E7D6F49
:1017000099ECE0F076C0D2F177C0D3F178C0D4F193
:1017100079C0D5F11E0E0101246F030E256F390E1D
:10172000266FE70E276FD2C128F1D3C129F1D4C1AA
:101730002AF1D5C12BF1F0EC03F0D2C186F0D3C170
:1017400087F0D4C188F0D5C189F0DEC18AF0DFC14D
:101750008BF0E0C18CF0E1C18DF06AEC05F086C041
:1017600098F187C099F188C09AF189C09BF198C11E
:1017700086F099C187F09AC188F09BC189F0CD0E9F
:101780008A6FCC0E8B6FCC0E8C6F3E0E8D6FF2EC91
:10179000F5F0D8B003D0050E0201F36FCD0E0001B5
:1017A000866FCC0E876FCC0E886F3E0E896F98C106
:1017B0008AF099C18BF09AC18CF09BC18DF0F2EC4C
:1017C000F5F0D8B003D0040E0201F36F010E010151
:1017D000B96FFE51D8A491D02D0E3D01EA6F000ED5
:1017E0000001866F000E876F400E886F410E896F73
:1017F000D2C18AF0D3C18BF0D4C18CF0D5C18DF0A9
:10180000F2ECF5F0D8B01AD0D2C176F0D3C177F0AF
:10181000D4C178F0D5C179F0000E7A6F000E7B6FDD
:10182000000E7C6FBF0E7D6F99ECE0F076C0D2F1B8
:1018300077C0D3F178C0D4F179C0D5F11E0E010183
:10184000246F030E256F120E266FE70E276FD2C18D
:1018500028F1D3C129F1D4C12AF1D5C12BF1F0EC83
:1018600003F0D2C186F0D3C187F0D4C188F0D5C1CE
:1018700089F0DAC18AF0DBC18BF0DCC18CF0DDC10C
:101880008DF06AEC05F086C098F187C099F188C0A8
:101890009AF189C09BF198C186F099C187F09AC1ED
:1018A00088F09BC189F0CD0E8A6FCC0E8B6FCC0E69
:1018B0008C6F3E0E8D6FF2ECF5F0D8B003D0050EB4
:1018C0000201F36FCD0E0001866FCC0E876FCC0E38
:1018D000886F3E0E896F98C18AF099C18BF09AC1CA
:1018E0008CF09BC18DF0F2ECF5F0D8B003D0040E73
:1018F0000201F36F010E0101B96FD2C125F0D3C10E
:1019000026F0D4C127F0D5C128F0DEC129F0DFC10F
:101910002AF0E0C12BF0E1C12CF056ECFDF0D8A08C
:1019200006D0000E0101B96F200E0201F36FD2C183
:1019300025F0D3C126F0D4C127F0D5C128F0DAC1F3
:1019400029F0DBC12AF0DCC12BF0DDC12CF056EC14
:10195000FDF0D8A006D0000E0101B96F200E0201E3
:10196000F36F1E0E256E030E266E8EECFBF014EC4C
:1019700007F0040E0F18D8A478D13901A1919191E4
:10198000000E106E010E0101C06F000EC16F010E3E
:10199000DDECFBF0090E01016D6F1E0E6C6FE40EA5
:1019A000E82EFED76C2FFCD76D2FFAD700F01E0E55
:1019B0000101246F030E256FEF0E266FF90E276FBE
:1019C000F0EC03F01E0E256E030E266E8EECFBF07F
:1019D000010E00016A6F1E0E6B6F030E6C6F010E1D
:1019E000EEEC0BF032EC0CF0010E00016B6F5F0EB1
:1019F0006C6FF90E6D6F6C516D11D8A4000E6E6F87
:101A0000020E3AEC0BF0010E00016B6F8D0E6C6F45
:101A1000F80E6D6F6C516D11D8A4000E6E6F030E31
:101A20003AEC0BF0010E00016B6F4E0E6C6FF80E6E
:101A30006D6F6C516D11D8A4000E6E6F040E3AECF0
:101A40000BF0000E3A01576F000E106E39019181B4
:101A5000020E1018D8A432D0E80E055C030E06580A
:101A6000D8B02CD00101C02B020EC06502D0010EEF
:101A7000C06FC005D8A40AD01E0E246F030E256FB8
:101A8000250E266FEB0E276FF0EC03F0020EC01947
:101A9000D8A40AD01E0E246F030E256F850E266F64
:101AA000EB0E276FF0EC03F01E0E256E030E266E74
:101AB0008EECFBF0000E106EC0EC0BF00101C005C7
:101AC000D8A41AD0000E0001666F020E656F000EDA
:101AD000686F010E676F3E0E696FEAECFAF0000E58
:101AE0000001666F030E656F000E686F010E676F71
:101AF000200E696FEAECFAF0020E0101C019D8A4B9
:101B00001AD0000E0001666F020E656F000E686F3E
:101B1000010E676F200E696FEAECFAF0000E00010B
:101B2000666F030E656F000E686F010E676F3E0EE5
:101B3000696FEAECFAF0190E01016D6F5A0E6C6FC5
:101B4000B10EE82EFED76C2FFCD76D2FFAD700D040
:101B5000000E0001666F020E656F000E686F010EC9
:101B6000676F200E696FEAECFAF0000E0001666FF5
:101B7000030E656F000E686F010E676F200E696FB0
:101B8000EAECFAF0190E01016D6F5A0E6C6FB10E8E
:101B9000E82EFED76C2FFCD76D2FFAD700D0020E9F
:101BA0001018D8A441D0E90E055C030E0658D8A041
:101BB0003BD01E0E0101246F030E256F3E0E266FD3
:101BC000FC0E276FF0EC03F0C0C1C1F1C105D8A431
:101BD00008D0000E00016C6F030E6B6FA9ECF4F0DF
:101BE00007D0000E00016C6F020E6B6FA9ECF4F0D1
:101BF0001E0E256E030E266E8EECFBF0010E00010C
:101C00006B6FD70E6C6FF20E6D6F6C516D11D8A4A7
:101C1000000E6E6F040E3AEC0BF0020E8EEC05F027
:101C2000000E106EC0EC0BF01004D8A406D0E90E24
:101C3000055C030E0658D8B007D00101C151D8A4E5
:101C400003D03901A3AF04D7390191910101C10536
:101C5000D8B47DECA4F0020E0101C119D8B452EC45
:101C600096F0040E0F6E14EC07F0050E0F18D8A4B2
:101C700020D03901A1919191000E3A01576F000EC9
:101C8000106E1E0E0101246F030E256FD30E266FFA
:101C9000DE0E276F0FC028F1296BF0EC03F01E0E4B
:101CA000256E030E266E8EECFBF074ECD2F014EC75
:101CB00007F0060E0F18D8A45CD03901A1919191BC
:101CC000000E106E550E2B6EEC0E2C6E78EC06F09E
:101CD0000101BB05D8A422D0000EBB6F060E000187
:101CE0006B6F9E0E6C6FFC0E6D6F6C516D11D8A4F6
:101CF000000E6E6F030E3AEC0BF0BA9E060E00015A
:101D00006B6F140E6C6FEF0E6D6F6C516D11D8A46C
:101D1000000E6E6F040E3AEC0BF011D0010EBB6F8B
:101D2000060E00016B6F190E6C6FFD0E6D6F6C511E
:101D30006D11D8A4000E6E6F030E3AEC0BF001018A
:101D4000BB51300F4AEC0CF032EC0CF0030E8EEC71
:101D500005F0D30E2B6EDF0E2C6E78EC06F0000E25
:101D6000266E970E256EBBC127F0EBEC02F014EC4B
:101D700007F0070E0F18D8A424D13901A191919131
:101D8000000E106EFC0E2B6EE50E2C6E78EC06F03D
:101D90000101B851D8A49BD0010EB86F0A0EBA6FDA
:101DA000D6C1D2F1D7C1D3F1D8C1D4F1D9C1D5F1BF
:101DB0001E0E246F030E256F5A0E266FF10E276F2D
:101DC000FAC128F1FBC129F1FCC12AF1FDC12BF1B7
:101DD000D2C12CF1D3C12DF1D4C12EF1D5C12FF137
:101DE000F0EC03F0070E0301246F070E2F6F010EB6
:101DF00000016A6F1E0E6B6F030E6C6F020EEEEC2D
:101E00000BF01E0E0101246F030E256F410E266F8D
:101E1000EE0E276FF6C228F1296BF7C22AF12B6B61
:101E2000F9C22CF12D6BFAC22EF12F6BF0EC03F0FE
:101E3000010E00016A6F1E0E6B6F030E6C6F030EB6
:101E4000EEEC0BF01E0E0101246F030E256FA70EA2
:101E5000266FEE0E276F390EBA25F66EF76AD20E90
:101E6000F722F86A000EF8220800F550286F296B57
:101E7000C951020D280EF324F66ED20EF420F76E2F
:101E8000F86A000EF8220800F5502A6F2B6BC95132
:101E9000020D010EF326000EF422280EF324F66E36
:101EA000D20EF420F76EF86A000EF8220800F55002
:101EB0002C6F2D6BF0EC03F0010E00016A6F1E0E0B
:101EC0006B6F030E6C6F040EEEEC0BF036D0000E51
:101ED000B86F1E0E256E030E266E5D0E276EFE0E6B
:101EE000286E39EC01F0090E00016A6F1E0E6B6F4F
:101EF000030E6C6F020EEEEC0BF01E0E256E030E41
:101F0000266E510E276EFE0E286E39EC01F0090E7A
:101F100000016A6F1E0E6B6F030E6C6F030EEEEC0A
:101F20000BF0000E666F040E656F000E686F010EF9
:101F3000676F200E696FEAECFAF00101B851D8B46E
:101F400005D0930E0601246FFF0E04D0D00E0601BB
:101F5000246FFF0E256F1E0E0101246F030E256FE7
:101F6000EA0E266FFE0E276F24C628F125C629F13A
:101F7000F0EC03F01E0E256E030E266E8EECFBF0C9
:101F80008A0E2B6EDD0E2C6E78EC06F0000E2C6E99
:101F90007C0E2B6ED2C12DF0D3C12EF0D4C12FF008
:101FA000D5C130F046EC05F0000E266E960E256E7B
:101FB000B8C127F0EBEC02F0020E8EEC05F014EC49
:101FC00007F0080E0F18D8B4CCB28FD0CCB48DD097
:101FD0003901A1919191000E106EB80E2B6EFB0E7F
:101FE0002C6E78EC06F0010E00016B6F030E6C6F27
:101FF000FA0E6D6F6C516D11D8A4000E6E6F010E4C
:102000003AEC0BF01E0E0101246F030E256FE40E57
:10201000266FF10E276FCCA203D06C6B6C2B02D015
:1020200001016C6BD8906C33300E6C25286F296BD6
:10203000000E2923CCA403D06D6B6D2B02D00101BF
:102040006D6BD8906D33D8906D33300E6D252A6F3F
:102050002B6B000E2B23F0EC03F01E0E256E030EEF
:10206000266E8EECFBF032EC0CF0010E00016A6F74
:102070001E0E6B6F030E6C6F020EEEEC0BF0000E7B
:102080006C6F030E6B6FA9ECF4F0000E00016C6F27
:10209000040E6B6FA9ECF4F0030E8EEC05F0000E4D
:1020A0000101B36FBC80010EBB6FE30E2B6EEC0E13
:1020B0002C6E78EC06F0000E266E940E256EB4C1E0
:1020C00027F0EBEC02F0000E266E950E256EB3C1E4
:1020D00027F0EBEC02F0000E266E970E256EBBC1CA
:1020E00027F0EBEC02F014EC07F06F002CFF11F07E
:1020F00030EC02F07A0E01016D6FC10E6C6F810E33
:10210000E82EFED76C2FFCD76D2FFAD700D0010137
:10211000CF05D8A44DD3C90E2B6EFF0E2C6E78ECD4
:1021200006F0800E256E050E266E8EECFBF032EC6E
:102130000CF0800E0101A66F050EA76F60009BF6E4
:10214000D9FF60009FF6DAFF480EDE18D8A46DD0E4
:1021500020EE01F0A651D926A751DA22650EDE182D
:10216000D8A463D020EE02F0A651D926A751DA22D6
:102170006C0EDE18D8A459D020EE03F0A651D92653
:10218000A751DA22700EDE18D8A44FD03D0E2B6E68
:10219000F20E2C6E78EC06F0160E2B6EFB0E2C6EEB
:1021A00078EC06F0010E2B6EDA0E2C6E78EC06F051
:1021B0001F0E2B6EE40E2C6E78EC06F0810E2B6E4B
:1021C000E50E2C6E78EC06F03A0E2B6EDB0E2C6EC4
:1021D00078EC06F0AE0E2B6EE90E2C6E78EC06F065
:1021E0004C0E2B6EE40E2C6E78EC06F0C20E2B6EAD
:1021F000D90E2C6E78EC06F05D0E2B6EF00E2C6E68
:1022000078EC06F06F0E2B6EFF0E2C6E78EC06F05D
:10221000800E256E050E266E8EECFBF032EC0CF077
:10222000000E0101A66F000EA76F60009BF6D9FF9C
:1022300060009FF6DAFF550EDE18D8A42ED020EEEF
:1022400001F0A651D926A751DA223B0EDE18D8A4F8
:1022500024D020EE13F0A651D926A751DA223B0E46
:10226000DE18D8A41AD0BF51D8A417D0360E2B6EC2
:10227000FD0E2C6E78EC06F0800E256E050E266E97
:102280008EECFBF032EC0CF001ECE9F032EC0CF0EF
:10229000000E0101A66F000EA76F60009BF6D9FF2C
:1022A00060009FF6DAFF420EDE18D8A436D020EE8A
:1022B00001F0A651D926A751DA22520EDE18D8A471
:1022C0002CD020EE02F0A651D926A751DA22550EC5
:1022D000DE18D8A422D020EE03F0A651D926A751AB
:1022E000DA223D0EDE18D8A418D020EE04F0A65154
:1022F000D926A751DA22310EDE18D8B4CA8E20EEC4
:1023000004F0A651D926A751DA22300EDE18D8B42F
:10231000CA9E000EA66F000EA76F60009BF6D9FF45
:1023200060009FF6DAFF420EDE18D8A47DD020EEC2
:1023300001F0A651D926A751DA22410EDE18D8A401
:1023400073D020EE02F0A651D926A751DA22560EFC
:10235000DE18D8A469D020EE03F0A651D926A751E3
:10236000DA223D0EDE18D8A45FD020EE06F0A6518A
:10237000D926A751DA22DF50D8A456D0D00E6C6FE0
:10238000FF0E6D6F20EE04F0A651D926A751DA2278
:10239000DF506E6F6F6B6C516E276D516F236F51F5
:1023A00036E10A0E6E5DD8B032D0D00E6C6FFF0EE3
:1023B0006D6F20EE05F0A651D926A751DA22DF5025
:1023C0006E6F6F6B6C516E276D516F236F511FE1F4
:1023D0000A0E6E5DD8B01BD020EE04F0A651D926AF
:1023E000A751DA22DF50116E1150D00F0A0D6F0085
:1023F000CCFFC2F120EE05F0A651D926A751DA2272
:10240000DF50116EC2511124D00FC26F08D0000EE0
:10241000C26F440E2B6EE80E2C6E78EC06F0000EA8
:102420000101A66F000EA76F60009BF6D9FF600048
:102430009FF6DAFF500EDE18D8A464D020EE01F02B
:10244000A651D926A751DA22520EDE18D8A45AD0A6
:1024500020EE02F0A651D926A751DA22470EDE1847
:10246000D8A450D020EE03F0A651D926A751DA22E5
:102470003D0EDE18D8A446D020EE04F0A651D92691
:10248000A751DA22DF50D00F0A0D6F00CCFF11F0F8
:1024900020EE05F0A651D926A751DA22DF501124EB
:1024A000D00F116E11C06CF17F0E6C170B0E6C61AA
:1024B00025D011C0BAF11E0E246F030E256FA40E95
:1024C000266FEB0E276F11C028F1296B390E1124EE
:1024D000F66EF76AD20EF722F86A000EF8220800AC
:1024E000F5502A6F2B6BF0EC03F01E0E256E030ED9
:1024F000266E8EECFBF01150EAECE6F0000EA66FB3
:10250000000EA76F60009BF6D9FF60009FF6DAFF10
:10251000480EDE18D8A4ABD020EE01F0A651D92683
:10252000A751DA224D0EDE18D8A4A1D020EE02F079
:10253000A651D926A751DA223D0EDE18D8A497D08D
:1025400020EE05F0A651D926A751DA223A0EDE1860
:10255000D8A48DD020EE03F0A651D926A751DA22B7
:10256000DF50116E11C0F6F21150D00F116E1150E4
:102570000A0D6F00CCFF07F06F00D0FF08F020EECF
:1025800004F0A651D926A751DA22DF50116E11C0EE
:10259000F7F21150D00F116E11500724076E000E84
:1025A0000820086E085033E1180E075CD8B02FD011
:1025B00020EE06F0A651D926A751DA22DF50116E7F
:1025C00011C0F9F21150D00F116E11500A0D6F00A9
:1025D000CCFFACF16F00D0FFADF120EE07F0A651BB
:1025E000D926A751DA22DF50116E11C0FAF211502C
:1025F000D00F116E1150AC25AC6F000EAD21AD6F38
:10260000085005E13C0E075CD8A0ACC1C4F10750EE
:102610000810D8A407D0AC51AD11D8A403D0000E37
:10262000BF6F20D007C0C5F1ACC1C4F1010EBF6FB0
:10263000000E0201AD6F1E0E0101246F030E256F07
:10264000220E266FE90E276FC5C128F1296BC4C180
:102650002AF12B6BF0EC03F01E0E256E030E266E96
:102660008EECFBF0000E0101A66F000EA76F60005C
:102670009BF6D9FF60009FF6DAFF520EDE18D8A451
:1026800047D020EE01F0A651D926A751DA22450EF7
:10269000DE18D8A43DD020EE02F0A651D926A751CD
:1026A000DA22530EDE18D8A433D020EE03F0A65160
:1026B000D926A751DA22450EDE18D8A429D020EE5B
:1026C00004F0A651D926A751DA22540EDE18D8A458
:1026D0001FD0A6C125F0A7C126F08EEC04F0050E90
:1026E00025182610D8A40FD0740E2B6EF00E2C6E69
:1026F00078EC06F0000E0101A66F000EA76F040E25
:102700008EEC05F0FF00000E0101A66F000EA76F12
:10271000800E256E050E266E000E276EFF0E286EAB
:10272000000E2A6E0A0E296E94ECF2F02550261047
:10273000D8A43ED0D00E01016C6FFF0E6D6F20EE5D
:102740000BF0A651D926A751DA22DF506E6F6F6BBE
:102750006C516E276D516F236F5125E10A0E6E5D2E
:10276000D8B021D020EE0BF0A651D926A751DA22FD
:10277000DF50D00F116E0F0E116002D011C0BEF1EC
:102780001E0E246F030E256FAA0E266FE50E276F0F
:10279000BEC128F1296BF0EC03F01E0E256E030E6E
:1027A000266E8EECFBF0000E0101A66F000EA76FE7
:1027B00075C267F276C268F2040E0101C219D8A48C
:1027C00027D01E0E246F030E256F6E0E266FDF0EB0
:1027D000276FC5C128F1296BC4C12AF12B6BADC28B
:1027E0002CF12D6BFE51030DED0EF3242E6F030E15
:1027F000F4202F6F67C230F168C231F1F0EC03F0C2
:102800001E0E256E030E266E8EECFBF032EC0CF0E5
:10281000B2EC05F082ECCEF0FAC186F0FBC187F095
:10282000FCC188F0FDC189F07CC18AF07DC18BF0CC
:102830007EC18CF07FC18DF0F2ECF5F0D8B02BD0DA
:10284000F2C186F0F3C187F0F4C188F0F5C189F0D8
:1028500063C225F064C226F0000E26BEFF0E276E6E
:10286000286E010E94ECEFF025C08AF026C08BF0A4
:1028700027C08CF028C08DF0F2ECF5F0D8B00BD06A
:102880000101BB05D8A407D0BABE03D0050E8EEC5B
:1028900005F0BA8E06D0BAAE03D0050E8EEC05F068
:1028A000BA9E0E0E0101C219D8A4F4D01E0E246FD8
:1028B000030E256F6A0E266FDE0E276F000E296F3E
:1028C000000E286FBAC12AF12B6B390EBA25F66EAD
:1028D000F76AD20EF722F86A000EF8220800F550C7
:1028E0002C6F2D6BF0EC03F01E0E256E030E266E82
:1028F0008EECFBF01E0E0101246F030E256FFF0E00
:10290000266FEC0E276FFEC128F1296BFE51030DD7
:10291000ED0EF3242A6F030EF4202B6FF0EC03F07E
:102920001E0E256E030E266E8EECFBF01E0E0101B0
:10293000246F030E256FB70E266FFA0E276FD2C1D4
:1029400028F1D3C129F1D4C12AF1D5C12BF1F0EC82
:1029500003F01E0E256E030E266E8EECFBF01E0E8F
:102960000101246F030E256F5E0E266FFB0E276F8D
:10297000FAC128F1FBC129F1FCC12AF1FDC12BF1FB
:10298000F0EC03F01E0E256E030E266E8EECFBF0AF
:102990001E0E0101246F030E256F5E0E266FFC0EC6
:1029A000276F47C228F148C229F149C22AF14AC219
:1029B0002BF1F0EC03F01E0E256E030E266E8EEC4E
:1029C000FBF01E0E0101246F030E256FDA0E266F39
:1029D000FB0E276F43C228F144C229F145C22AF1F8
:1029E00046C22BF1F0EC03F01E0E256E030E266E90
:1029F0008EECFBF01E0E0101246F030E256F4E0EB0
:102A0000266FFC0E276F63C228F164C229F1F0EC37
:102A100003F01E0E256E030E266E8EECFBF01E0ECE
:102A20000101246F030E256F6D0E266FEF0E276FC9
:102A30006F0030FF6CF1060E6C176C51286F296B1C
:102A4000F0EC03F01E0E256E030E266E8EECFBF0EE
:102A5000CABE0BD01E0E0101246F030E256F940E0B
:102A6000266FFB0E276FF0EC03F0CAAE0BD01E0EE4
:102A70000101246F030E256FFC0E266FFB0E276FDE
:102A8000F0EC03F01E0E256E030E266E8EECFBF0AE
:102A900032EC0CF00C0E0101C219D8A428D01E0E85
:102AA000246F030E256FA10E266FDF0E276F6F00B8
:102AB00030FF28F1296BCCA203D06C6B6C2B02D0B9
:102AC00001016C6B6C512A6F2B6BCCA403D06D6B26
:102AD0006D2B02D001016D6B6D512C6F2D6BF0ECE5
:102AE00003F01E0E256E030E266E8EECFBF0CCA2BC
:102AF000CCB404D00101B351D8B457D00A0E2B6E18
:102B0000FD0E2C6E78EC06F01E0E0101246F030EF4
:102B1000256FB50E266FEF0E276F6F0030FF6CF13B
:102B2000020E6C176C51286F296B6F0030FF6DF12E
:102B3000040E6D176D512A6F2B6BF0EC03F01E0E17
:102B4000256E030E266E8EECFBF032EC0CF0010EBF
:102B500000016B6F1E0E6C6F030E6D6F6C516D116B
:102B6000D8A4200E6E6F020E3AEC0BF0CC50060B80
:102B70000101B46FB351D8A418D0010EB36F000E89
:102B8000266E940E256EB4C127F0EBEC02F0000E19
:102B9000266E950E256EB3C127F0EBEC02F0FC0E0D
:102BA0002B6EDA0E2C6E78EC06F00101B351D8B41E
:102BB00072D0BC90000EBB6F000E02019B6FBA9EDC
:102BC000010E00016B6F6F0E6C6FF50E6D6F6C5127
:102BD0006D11D8A4000E6E6F010E3AEC0BF0010ED1
:102BE00000016B6F3D0E6C6FF70E6D6F6C516D11C8
:102BF000D8A4000E6E6F030E3AEC0BF0010E00012C
:102C00006B6FFE0E6C6FF60E6D6F6C516D11D8A46C
:102C1000000E6E6F040E3AEC0BF0CCA20FD0010E3A
:102C200000016B6F130E6C6FF70E6D6F6C516D11B1
:102C3000D8A4000E6E6F020E3AEC0BF0CCA40FD0AD
:102C4000010E00016B6F280E6C6FF70E6D6F6C51EB
:102C50006D11D8A4000E6E6F020E3AEC0BF0CCA2F0
:102C6000CCB40FD0010E00016B6F0F0E6C6FF80E1D
:102C70006D6F6C516D11D8A4000E6E6F030E3AEC9F
:102C80000BF07F0E2B6EF20E2C6E78EC06F0020E1F
:102C90008EEC05F002D0EEEC9DF00201874B882B04
:102CA000B5EF87F0000E106E000E3A01576F390134
:102CB0009191180E2B6EDD0E2C6E78EC06F0C0ECA8
:102CC0000BF0010E0601006F020E066F340E2B6E24
:102CD000FF0E2C6E78EC06F0000E106E010EDDEC8F
:102CE000FBF0010E00016B6FF60E6C6FF80E6D6F4E
:102CF0006C516D11D8A4000E6E6F010E3AEC0BF002
:102D0000010E00016B6F4A0E6C6FF90E6D6F6C5106
:102D10006D11D8A4000E6E6F020E3AEC0BF0010E8E
:102D200000016B6F200E6C6FF90E6D6F6C516D11A1
:102D3000D8A4000E6E6F030E3AEC0BF0000E0001EB
:102D4000666F040E656F000E686F010E676F3B0EB5
:102D5000F66ED20EF76E000EF86E08006F00D4FF0C
:102D600069F0EAECFAF0020E03ECD6F0040E8EECF9
:102D700005F0010E00016B6F730E6C6FF40E6D6F3A
:102D80006C516D11D8A4000E6E6F010E3AEC0BF071
:102D9000010E00016B6F5E0E6C6FF40E6D6F6C5167
:102DA0006D11D8A4000E6E6F020E3AEC0BF0000EFF
:102DB000106E000E3A01576F39019181C0EC0BF093
:102DC000040E1018D8A414D0E80E055C030E0658A3
:102DD000D8B00ED02B0E3D01EA6F0601062B06512E
:102DE000800A760FD8A002D0020E066F39019191A9
:102DF000080E1018D8A414D0E80E055C030E06586F
:102E0000D8B00ED02D0E3D01EA6F0601060706511F
:102E1000800A7E0FD8B002D0090E066F3901919159
:102E2000040E1018D8B404D0080E1018D8A44DD031
:102E30001E0E0101246F030E256F450E266FEB0E4B
:102E4000276F060106510101286F296B28BF29074A
:102E5000390E06010625F66EF76AD20EF722F86AD9
:102E6000000EF8220800F55001012A6F2B6B0601B5
:102E70000651200D3E0EF324D96E060EF420DA6EB4
:102E8000DF500101666F66512C6F2D6BF0EC03F083
:102E90001E0E256E030E266E8EECFBF0000E106EDD
:102EA0000F0E0101C219D8A404D00601065103EC8B
:102EB000D6F0C0EC0BF09181020E0601006F480EB7
:102EC0002B6EFF0E2C6E78EC06F0000E0001666F84
:102ED000030E656F000E686F070E676F4D0E696F0A
:102EE000EAECFAF0000E0601086F000E076F08BF4B
:102EF00006D0085132E10C0E075DD8B02ED0000E7E
:102F00000001666F030E656F090E060107250001BB
:102F1000676F000E060108210001686F0601065167
:102F2000200D260E0101666F060E676FF3506627AF
:102F3000F45067230601075101016625D96E060189
:102F4000085101016721DA6EDF500001696FEAEC78
:102F5000FAF00601074B082BCAD7060E00016B6F6B
:102F6000B10E6C6FFF0E6D6F6C516D11D8A4000E19
:102F70006E6F040E3AEC0BF0000E0601086F000EA7
:102F8000076F08BF06D0085136E10C0E075DD8B0B8
:102F900032D0000E0001666F040E656F090E060147
:102FA00007250001676F000E060108210001686F08
:102FB00006010651200D260E0101666F060E676F91
:102FC0000C0E6627000E6723F3506627F450672324
:102FD0000601075101016625D96E0601085101015C
:102FE0006721DA6EDF500001696FEAECFAF0060142
:102FF000074B082BC6D7000E0001666F040E656FE5
:10300000000E686F010E676F390E06010625F66E19
:10301000F76AD20EF722F86A000EF82208006F0055
:10302000D4FF69F0EAECFAF0150E0101676F4B0E60
:10303000666FBE0EE82EFED7662FFCD7672FFAD735
:1030400000F0000E0001666F040E656F000E686FE1
:10305000010E676F200E696FEAECFAF0150E0101A0
:10306000676F4B0E666FBE0EE82EFED7662FFCD73D
:10307000672FFAD700F0000E0001666F040E656F2F
:10308000000E686F010E676F390E06010625F66E99
:10309000F76AD20EF722F86A000EF82208006F00D5
:1030A000D4FF69F0EAECFAF0020E1018D8A441D06F
:1030B000E90E055C030E0658D8A03BD0030E0601AE
:1030C000006F1E0E0101246F030E256F740E266F14
:1030D000E60E276F060106510101286F296B28BFF4
:1030E0002907390E06010625F66EF76AD20EF72279
:1030F000F86A000EF8220800F55001012A6F2B6BC8
:1031000006010651200D260EF32401012C6F060E38
:10311000F4202D6FF0EC03F01E0E256E030E266ECC
:103120008EECFBF032EC0CF0000E106EC0EC0BF0ED
:1031300091911004D8A403D0000E0601006F39014C
:10314000A3BF0BD006010051800A7D0FD8B005D077
:103150000051800A7F0FD8B033D639019191000E0B
:10316000106EC0EC0BF07F0E2B6EDA0E2C6E78EC2E
:1031700006F0010EDDECFBF0010E00016B6F780E26
:103180006C6FF80E6D6F6C516D11D8A4000E6E6FE0
:10319000010E3AEC0BF0010E00016B6F520E6C6FDA
:1031A000F70E6D6F6C516D11D8A4000E6E6F020E8C
:1031B0003AEC0BF0010E00016B6F0B0E6C6FF90E09
:1031C0006D6F6C516D11D8A4000E6E6F030E3AEC4A
:1031D0000BF0030E8EEC05F0C0EC0BF0000E0001BE
:1031E000666F040E656F000E686F010E676F390E13
:1031F00006010625F66EF76AD20EF722F86A000E6F
:10320000F82208006F00D4FF69F0EAECFAF006013A
:10321000065103ECD6F0C0EC0BF00C0E00016B6F06
:1032200006010651200D3E0EF324D96E060EF42041
:10323000DA6EDF500101666F676B686B66C16CF018
:1032400067C16DF068C16EF0010E3AEC0BF0090E2B
:1032500000016B6F440E6C6FFE0E6D6F6C516D1143
:10326000D8A4000E6E6F020E3AEC0BF0000E0001B7
:10327000666F030E656F000E686F070E676F4D0E69
:10328000696FEAECFAF0000E0601086F000E076F96
:1032900008BF06D0085142E10C0E075DD8B03ED001
:1032A0000651200D260E0101666F060E676FF35062
:1032B0006627F45067230601075101016625D96E80
:1032C0000601085101016721DA6E000E060107258B
:1032D000E16E040E0821E26E6F007FFFE7FF000E33
:1032E0000001666F030E656F090E060107250001D8
:1032F000676F000E060108210001686F000E0601CD
:103300000725D96E040E0821DA6EDF500001696FBF
:10331000EAECFAF00601074B082BBAD7060E0001BB
:103320006B6FB10E6C6FFF0E6D6F6C516D11D8A489
:10333000000E6E6F040E3AEC0BF0000E0601086FE3
:10334000000E076F08BF06D0085146E10C0E075D5E
:10335000D8B042D00651200D260E0101666F060E30
:10336000676F0C0E6627000E6723F3506627F45034
:1033700067230601075101016625D96E0601085130
:1033800001016721DA6E0C0E06010725E16E040EBD
:103390000821E26E6F007FFFE7FF000E0001666FFD
:1033A000040E656F090E060107250001676F000E08
:1033B000060108210001686F0C0E06010725D96E71
:1033C000040E0821DA6EDF500001696FEAECFAF0B2
:1033D0000601074B082BB6D7000E086F180E076FB3
:1033E00008BF06D0085126E1200E075DD8B022D0D4
:1033F0000651200D260E0101666F060E676FF35011
:103400006627F45067230601075101016625D96E2E
:103410000601085101016721DA6E000E0601072539
:10342000E16E040E0821E26E6F007FFFE7FF074B9D
:10343000082BD6D7030E8EEC05F0010E0601036FA4
:10344000200E2B6EFF0E2C6E78EC06F0000E06019F
:10345000056F000E3A01576F3901A1919181000E5D
:10346000106EC0EC0BF0000E06010525D96EDA6A6D
:10347000040EDA22DF50046F000E0001666F020EA8
:10348000656F000E686F0C0E676F06010551256EA3
:10349000266A25BE2606000E286E0A0E276EDDEC73
:1034A000FDF02550300F0001696FEAECFAF0000ED4
:1034B0000001666F020E656F000E686F0D0E676F7C
:1034C00006010551256E266A25BE2606000E286EC9
:1034D0000A0E276ECBEC00F02550300F0001696F0B
:1034E000EAECFAF0000E0001666F020E656F000E46
:1034F000686F120E676F010E06010525256EE86ADA
:10350000D8B0E82A05BFE806266E000E286E0A0E1F
:10351000276EDDECFDF02550300F0001696FEAECFD
:10352000FAF0000E0001666F020E656F000E686F04
:10353000130E676F010E06010525256EE86AD8B0E7
:10354000E82A05BFE806266E000E286E0A0E276ED2
:10355000CBEC00F02550300F0001696FEAECFAF077
:10356000040E1018D8A414D0E80E055C030E0658FB
:10357000D8B00ED02B0E3D01EA6F0601052B055188
:10358000800A680FD8A002D0000E056F3901919112
:10359000080E1018D8A411D0E80E055C030E0658CA
:1035A000D8B00BD02D0E3D01EA6F0601050705AF1F
:1035B00002D0170E056F39019191040E1018D8B47E
:1035C00004D0080E1018D8A422D0000E106EC0EC43
:1035D0000BF01E0E0101246F030E256FC90E266F1E
:1035E000FE0E276F060105510101286F296B28BFC8
:1035F0002907F0EC03F01E0E256E030E266E8EECEE
:10360000FBF0000E106EC0EC0BF0A1919181060151
:103610000551800A740FD8B064D0000E0525D96E0C
:10362000DA6A040EDA22DF50046F000E0001666FC2
:10363000030E656F090E060105250001676FE86A34
:10364000D8B0E82A060105BFE8060001686F04C685
:1036500069F0EAECFAF0090E0101676F1E0E666F61
:10366000E40EE82EFED7662FFCD7672FFAD700F0BE
:10367000000E0001666F030E656F090E0601052539
:103680000001676FE86AD8B0E82A060105BFE806BE
:103690000001686F200E696FEAECFAF0110E01016B
:1036A000676F3C0E666FCB0EE82EFED7662FFCD7F9
:1036B000672FFAD7000E0001666F030E656F090EC3
:1036C000060105250001676FE86AD8B0E82A0601FF
:1036D00005BFE8060001686F04C669F0EAECFAF07D
:1036E00072D0000E0525D96EDA6A040EDA22DF5098
:1036F000046F000E0001666F040E656FFD0E010180
:10370000666FFF0E676F6651060105250001676F42
:10371000000E060105BFFF0E010167210001686F61
:1037200004C669F0EAECFAF0090E0101676F1E0E9B
:10373000666FE40EE82EFED7662FFCD7672FFAD708
:1037400000F0000E0001666F040E656FFD0E0101B2
:10375000666FFF0E676F6651060105250001676FF2
:10376000000E060105BFFF0E010167210001686F11
:10377000200E696FEAECFAF0110E0101676F3C0E42
:10378000666FCB0EE82EFED7662FFCD7672FFAD7D1
:10379000000E0001666F040E656FFD0E0101666F7D
:1037A000FF0E676F6651060105250001676F000E69
:1037B000060105BFFF0E010167210001686F04C605
:1037C00069F0EAECFAF006010351800A7F0FD8A0F5
:1037D0006AD0020E1018D8A466D0E80E055C030E5D
:1037E0000658D8B060D039019191010E00016B6F7D
:1037F000730E6C6FF40E6D6F6C516D11D8A4000ECA
:103800006E6F010E3AEC0BF0280E2B6EFD0E2C6E37
:1038100078EC06F0010E00016B6F810E6C6FFF0EED
:103820006D6F6C516D11D8A4000E6E6F030E3AECE3
:103830000BF00601042B0451800A7C0FD8A002D0A3
:10384000000E046F000E0525D96EDA6A040EDA2226
:10385000610013F8DFFF1E0E0101246F030E256FB8
:10386000F50E266FF30E276F060105510101286F33
:10387000296B28BF29070601045101012A6F2B6B10
:103880002ABF2B07F0EC03F01E0E256E030E266EEA
:103890008EECFBF0000E106EC0EC0BF0020E060179
:1038A000036F39019181020E06010319D8A442D198
:1038B000100E1018D8A43ED1E90E055C030E065870
:1038C000D8A038D139019191000E106EC0EC0BF0E8
:1038D000010EDDECFBF0010E00016B6F3F0E6C6F13
:1038E000FA0E6D6F6C516D11D8A4000E6E6F010E43
:1038F0003AEC0BF0F90E2B6EE70E2C6E78EC06F01E
:10390000040118510101666F676B66C125F067C13C
:1039100026F08EECFBF032EC0CF006010651016F44
:10392000026B01BF020701C666F102C667F1050E10
:10393000D890010166376737E82EFAD7A00E6625C2
:103940000601016F000E010167210601026F1E0EC4
:103950000101246F030E256F030E266FF30E276FF0
:10396000390E06010625F66EF76AD20EF722F86ABE
:10397000000EF8220800F5500101286F296B01C6DE
:103980002AF102C62BF1F0EC03F01E0E256E030E99
:10399000266E8EECFBF0010E00016A6F1E0E6B6F3F
:1039A000030E6C6F020EEEEC0BF032EC0CF0030E1B
:1039B0008EEC05F0000E0601086F000E076F08BFC1
:1039C00006D008517CE1200E075DD8B078D0000EFB
:1039D0000725D96E040E0821DA6EDF50046F0651F8
:1039E000200D260E0101666F060E676FF3506627E5
:1039F000F45067230601075101016625D96E0601BF
:103A0000085101016721DA6E610013F8DFFF1E0E15
:103A1000246F030E256F890E266FED0E276F07C6E4
:103A200028F108C629F101C62AF102C62BF10601C8
:103A30000651200D260E0101666F060E676FF350CA
:103A40006627F45067230601075101016625D96EE8
:103A50000601085101016721DA6EDF50686F685175
:103A60002C6F2D6BF0EC03F01E0E256E030E266EF0
:103A70008EECFBF0980E06010725D96E040E082186
:103A8000DA6E610013F8DFFF01C625F002C626F0EA
:103A900004C627F0EBEC02F00601014B022B030EEB
:103AA0000101676F080E666F770EE82EFED7662F4E
:103AB000FCD7672FFAD70601074B082B80D7010EDA
:103AC00000016B6FB70E6C6FF80E6D6F6C516D115E
:103AD000D8A4000E6E6F030E3AEC0BF0000E00013E
:103AE000666F030E656F000E686F050E676F390E07
:103AF00006010625F66EF76AD20EF722F86A000E66
:103B0000F82208006F00D4FF69F0EAECFAF0030E27
:103B10008EEC05F0000E106EC0EC0BF006010651A5
:103B200001015D6F5E6B5DBF5E07F2ECEEF0030EB0
:103B30000601036F1004D8A402D0000E036F3901F0
:103B4000A3BF0BD006010351800A7F0FD8A005D078
:103B50000351800A7D0FD8A086D43901A3BF15D0A8
:103B6000030E06010319D8A410D0010E00016B6FDB
:103B7000D80E6C6FF50E6D6F6C516D11D8A4000EE0
:103B80006E6F010E3AEC0BF00FD0010E00016B6F5F
:103B90009E0E6C6FF90E6D6F6C516D11D8A4000EF6
:103BA0006E6F010E3AEC0BF0020E8EEC05F0010E7A
:103BB000DDECFBF0090E0101676F1E0E666FE40E6F
:103BC000E82EFED7662FFCD7672FFAD700F0040E39
:103BD0000F6E000E106EC0EC0BF01200D50EC92552
:103BE000D96EDA6A020EDA22DF50BA6F000ED16F98
:103BF000000ED06FD15120E1200ED05DD8B01CD086
:103C0000BA51200D260E596F060E5A6FF3505927E0
:103C1000F4505A23D0515925D96ED1515A21DA6E18
:103C2000980ED025E16E040ED121E26E6F007FFF69
:103C3000E7FFD04BD12BDED7980EC525D96EDA6AB7
:103C4000040EDA22DF50B56F020EDDECFBF0090E38
:103C500001015A6F1E0E596FE40EE82EFED7592F40
:103C6000FCD75A2FFAD700F0120E0101C219D8A4BE
:103C70001DD01E0E246F030E256F7F0E266FEA0ED9
:103C8000276FB00E286F040E296FFEC12AF12B6B2F
:103C9000C5C12CF12D6BC4C12EF12F6BF0EC03F0DC
:103CA0001E0E256E030E266E8EECFBF00101B85140
:103CB000D8A4E9EFA2F0BB05D8A4E9EFA2F0F9AFD0
:103CC0002AD0F2C1ACF0F3C1ADF0F4C1AEF0F5C151
:103CD000AFF081ECF9F0ACC05DF1ADC05EF11E0E4D
:103CE0000101246F030E256FCD0E266FF10E276F95
:103CF000F6C128F1F7C129F1F8C12AF1F9C12BF178
:103D00005DC12CF15EC12DF163C22EF164C22FF1B1
:103D1000F0EC03F029D0F2C1ACF0F3C1ADF0F4C186
:103D2000AEF0F5C1AFF081ECF9F0ACC05DF1ADC023
:103D30005EF11E0E0101246F030E256F450E266FE6
:103D4000F00E276FF6C128F1F7C129F1F8C12AF169
:103D5000F9C12BF15DC12CF15EC12DF163C22EF1D1
:103D600064C22FF1F0EC03F0070E0301246F070E7D
:103D70002C6F010E00016A6F1E0E6B6F030E6C6FCD
:103D8000010EEEEC0BF0CABE0DD0000E666F010EF8
:103D9000656F000E686F0A0E676F230E696FEAEC9D
:103DA000FAF01ED0020187A10ED0000E0001666F4E
:103DB000010E656F000E686F0A0E676F240E696F43
:103DC000EAECFAF00DD0000E0001666F010E656F8F
:103DD000000E686F0A0E676F200E696FEAECFAF04A
:103DE000000E0101B66F1E0EC46104D0B5A102D051
:103DF000010EB66F1D0EC46504D0B5A302D0010E2E
:103E0000B66F030EB519D8A402D0010EB66FB5C1B6
:103E10005CF1B651FE19D8A407D0B705D8A404D0D8
:103E2000000EB76F000EB96FB751D8A423D0000EA3
:103E3000BE6F200E0201F46FB6C1FEF10101B65152
:103E4000D8A40AD0DAC13FF2DBC140F2DCC141F2B2
:103E5000DDC142F2BA9CBA8AB605D8A430D0DEC120
:103E60003FF2DFC140F2E0C141F2E1C142F2BA8C5F
:103E7000BA9A25D0B605D8A40FD0000EFE6FDAC1CD
:103E80003FF2DBC140F2DCC141F2DDC142F2BA8C4B
:103E9000050EBE6F050E11D0B651D8A410D0010E7C
:103EA000FE6FDEC13FF2DFC140F2E0C141F2E1C18D
:103EB00042F2BA8A060EBE6F040E0201F46F0101CF
:103EC000B951D8A409D03FC2D2F140C2D3F141C206
:103ED000D4F142C2D5F11AD0FE51D8A419D0D2C122
:103EE00025F0D3C126F0D4C127F0D5C128F0DAC11E
:103EF00029F0DBC12AF0DCC12BF0DDC12CF056EC3F
:103F0000FDF0D8A005D0000E0101B96F200E82D0BF
:103F10000101FE05D8A414D0D2C125F0D3C126F0EA
:103F2000D4C127F0D5C128F0DEC129F0DFC12AF0C5
:103F3000E0C12BF0E1C12CF056ECFDF0D8B0E3D796
:103F40000101FE51D8A417D0D2C186F0D3C187F0A9
:103F5000D4C188F0D5C189F0DAC18AF0DBC18BF019
:103F6000DCC18CF0DDC18DF0F2ECF5F0D8B003D0FF
:103F7000050E0201F36F0101FE51D8A417D0DAC17A
:103F800086F0DBC187F0DCC188F0DDC189F0D2C1E9
:103F90008AF0D3C18BF0D4C18CF0D5C18DF0F2EC96
:103FA000F5F0D8B003D0040E0201F36F0101FE0555
:103FB000D8A417D0D2C186F0D3C187F0D4C188F07D
:103FC000D5C189F0DEC18AF0DFC18BF0E0C18CF091
:103FD000E1C18DF0F2ECF5F0D8B003D0050E02018E
:103FE000F36F0101FE05D8A417D0DEC186F0DFC152
:103FF00087F0E0C188F0E1C189F0D2C18AF0D3C175
:104000008BF0D4C18CF0D5C18DF0F2ECF5F0D8B0C6
:1040100003D0040E0201F36F0101C205D8A441D000
:104020001E0E246F030E256F650E266FEB0E276F95
:10403000B00E286F040E296FFEC12AF12B6BC5C18B
:104040002CF12D6BC4C12EF12F6BF0EC03F01E0E82
:10405000256E030E266E8EECFBF01E0E0101246F02
:10406000030E256F3B0E266FDF0E276FB5C128F1BB
:10407000296BFE51030DED0EF3242A6F030EF4207D
:104080002B6FD2C12CF1D3C12DF1D4C12EF1D5C1EA
:104090002FF1F0EC03F01E0E256E030E266E8EEC53
:1040A000FBF0000E03011E6F1E0E0101246F030EB4
:1040B000256F720E266FEC0E276FFAC128F1FBC137
:1040C00029F1FCC12AF1FDC12BF1FFC12CF12D6BAF
:1040D000EEC12EF1EFC12FF1F0C130F1F1C131F19C
:1040E000F4C232F1336BFE51030DED0EF324346F45
:1040F000030EF420356FF3C236F1376BD2C138F1BD
:10410000D3C139F1D4C13AF1D5C13BF1F0EC03F0A0
:10411000070E0301236F070E306FEEC125F0EFC1CC
:1041200026F0F0C127F0F1C128F0000E296E000E34
:104130002A6E000E2B6E000E2C6E56ECFDF0D8A0F1
:1041400007D0200E0301276F200E286F200E296F45
:10415000010E00016A6F1E0E6B6F030E6C6F020E74
:10416000EEEC0BF00C0E0101C219D8A425D01E0EE6
:10417000246F030E256F9C0E266FE60E276FFAC183
:1041800028F1FBC129F1FCC12AF1FDC12BF1FFC1CE
:104190002CF12D6BEEC12EF1EFC12FF1F0C130F1FA
:1041A000F1C131F1F0EC03F01E0E256E030E266E08
:1041B0008EECFBF032EC0CF0000E03011E6F1E0EB5
:1041C0000101246F030E256FC20E266FFD0E276FAF
:1041D000F6C228F1296BF7C22AF12B6BF9C22CF138
:1041E0002D6BFAC22EF12F6BF0EC03F0000E0301E1
:1041F000266F010E00016A6F1E0E6B6F030E6C6F4F
:10420000030EEEEC0BF0000E0101D16F000ED06F2B
:10421000D15136E10C0ED05DD8B032D0980ED025F9
:10422000D96E040ED121DA6EDF505B6F000E0001F3
:10423000666F030E656F090E0101D0250001676FDF
:10424000000E0101D1210001686F5BC169F0EAEC49
:10425000FAF0E40E00D000D0E82EFCD700D000D059
:10426000080E0101C219D8A407D05B51300F4AECE7
:104270000CF02E0E4AEC0CF00101D04BD12BC8D71C
:10428000080EC219D8B432EC0CF0000E03011E6FF8
:104290001E0E0101246F030E256FBD0E266FFE0E4C
:1042A000276F390EBA25F66EF76AD20EF722F86A32
:1042B000000EF8220800F550286F296BC951020D35
:1042C000280EF324F66ED20EF420F76EF86A000E74
:1042D000F8220800F5502A6F2B6BC951020D010E10
:1042E000F326000EF422280EF324F66ED20EF420EC
:1042F000F76EF86A000EF8220800F5502C6F2D6B4F
:10430000F0EC03F0000E0301266F010E00016A6F4E
:104310001E0E6B6F030E6C6F040EEEEC0BF0000EB6
:104320000101D16F000ED06FD15136E10C0ED05D7E
:10433000D8B032D0A40ED025D96E040ED121DA6EB9
:10434000DF505B6F000E0001666F040E656F090E93
:104350000101D0250001676F000E0101D12100018C
:10436000686F5BC169F0EAECFAF0E40E00D000D0AF
:10437000E82EFCD700D000D0080E0101C219D8A445
:1043800007D05B51300F4AEC0CF02E0E4AEC0CF0CB
:104390000101D04BD12BC8D7080EC219D8B432ECCA
:1043A0000CF00101BF51D8A405D0CA513FEC0CF06C
:1043B0000101C56F1E0EC46101D003D0596B592B8A
:1043C00002D00101596BC551020DF350592502016C
:1043D000A26F080E0101C219D8A413D01E0E246FBB
:1043E000030E256F380E266FEC0E276FA2C228F140
:1043F000296BF0EC03F01E0E256E030E266E8EEC7C
:10440000FBF00C0E0101C56172D0000E0001666F59
:10441000040E656F000E686F080E676F200E696FDF
:10442000EAECFAF0000E0001666F030E656F000EF5
:10443000686F080E676F3E0E696FEAECFAF00101D3
:10444000C551090FC36F020187A12ED043D0000EC2
:104450000001666F030E656FC3C167F0686B200EC5
:10446000696FEAECFAF012001E0EC4610CD0000E67
:104470000001666F030E656FC3C167F0686B020EC3
:10448000696FEAECFAF01D0E0101C4651200000E1E
:104490000001666F030E656FC3C167F0686B010EA4
:1044A000696FEAECFAF0120001015C51596F5A6B26
:1044B0005A51000AD8A412005951000AD8B4C7D7DB
:1044C000010AD8B4C4D7030AD8B4C1D7010AD8A402
:1044D0001200CAD7000E0001666F030E656FC3C1DC
:1044E00067F0686B5CC169F0EAECFAF01200000E4C
:1044F0000001666F030E656F000E686F080E676F30
:10450000200E696FEAECFAF0000E0001666F040EEF
:10451000656F000E686F080E676F3E0E696FEAECFC
:10452000FAF00101C551FD0FC36F020187A12ED022
:1045300043D0000E0001666F040E656FC3C167F0C3
:10454000686B200E696FEAECFAF012001E0EC4616F
:104550000CD0000E0001666F040E656FC3C167F0DA
:10456000686B020E696FEAECFAF01D0E0101C4657A
:104570001200000E0001666F040E656FC3C167F084
:10458000686B010E696FEAECFAF0120001015C51F0
:10459000596F5A6B5A51000AD8A412005951000A97
:1045A000D8B4C7D7010AD8B4C4D7030AD8B4C1D77E
:1045B000010AD8A41200CAD7000E0001666F040ECB
:1045C000656FC3C167F0686B5CC169F0EAECFAF033
:1045D0001200000EBE6F000EBD6FBA9ABA9CB805ED
:1045E000D8A498D0D6C1D2F1D7C1D3F1D8C1D4F1D3
:1045F000D9C1D5F11E0E246F030E256F5A0E266FFA
:10460000F10E276FFAC128F1FBC129F1FCC12AF193
:10461000FDC12BF1D2C12CF1D3C12DF1D4C12EF1AA
:10462000D5C12FF1F0EC03F0070E0301246F070E44
:104630002F6F010E00016A6F1E0E6B6F030E6C6F01
:10464000020EEEEC0BF01E0E0101246F030E256F1F
:10465000410E266FEE0E276FF6C228F1296BF7C2C6
:104660002AF12B6BF9C22CF12D6BFAC22EF12F6BB4
:10467000F0EC03F0010E00016A6F1E0E6B6F030E6B
:104680006C6F030EEEEC0BF00A0E0101BA6F1E0EFA
:10469000246F030E256FA70E266FEE0E276F390EBF
:1046A000BA25F66EF76AD20EF722F86A000EF822E3
:1046B0000800F550286F296BC951020D280EF3240C
:1046C000F66ED20EF420F76EF86A000EF82208009B
:1046D000F5502A6F2B6BC951020D010EF326000E07
:1046E000F422280EF324F66ED20EF420F76EF86A48
:1046F000000EF8220800F5502C6F2D6BF0EC03F043
:10470000010E00016A6F1E0E6B6F030E6C6F040EBC
:10471000EEEC0BF00101BB51D8A41200F9AF26D08A
:10472000F2C1ACF0F3C1ADF0F4C1AEF0F5C1AFF041
:1047300081ECF9F0ACC05DF1ADC05EF11E0E01017F
:10474000246F030E256FE70E266FF00E276FF6C15C
:1047500028F1F7C129F1F8C12AF1F9C12BF15DC1A6
:104760002CF15EC12DF1F0EC03F025D0F2C1ACF0DC
:10477000F3C1ADF0F4C1AEF0F5C1AFF081ECF9F0EA
:10478000ACC05DF1ADC05EF11E0E0101246F030EE1
:10479000256F430E266FF10E276FF6C128F1F7C182
:1047A00029F1F8C12AF1F9C12BF15DC12CF15EC1EB
:1047B0002DF1F0EC03F0070E0301246F070E2F6FAD
:1047C000010E00016A6F1E0E6B6F030E6C6F010EFF
:1047D000EEEC0BF0BABE1FD00A0E6A6F230E6B6FA1
:1047E000000E6C6F010EEEEC0BF01E0E0101246F3B
:1047F000030E256F950E266FF20E276FFAC128F172
:10480000FBC129F1FCC12AF1FDC12BF1F0EC03F051
:10481000070E0301246F010E00016A6F1E0E6B6FFD
:10482000030E6C6F020EEEEC0BF01E0E0101246FF6
:10483000030E256FF20E266FEE0E276FF6C228F1DB
:10484000296BF7C22AF12B6BF9C22CF12D6BFAC23E
:104850002EF12F6BF0EC03F0010E00016A6F1E0EBB
:104860006B6F030E6C6F030EEEEC0BF00B0E010181
:10487000BA6F1E0E246F030E256F0B0E266FEF0E00
:10488000276F390EBA25F66EF76AD20EF722F86A4C
:10489000000EF8220800F550286F296BC951020D4F
:1048A000280EF324F66ED20EF420F76EF86A000E8E
:1048B000F8220800F5502A6F2B6BC951020D010E2A
:1048C000F326000EF422280EF324F66ED20EF42006
:1048D000F76EF86A000EF8220800F5502C6F2D6B69
:1048E000F0EC03F0010E00016A6F1E0E6B6F030EF9
:1048F0006C6F040EEEEC0BF01200C70E2B6EF90E6F
:104900002C6E78EC06F0000E0101636F000E626FF2
:104910001E0E246F030E256FFC0E266FDD0E276F13
:1049200062C128F163C129F1800E62252A6F000E51
:1049300063212B6FD50E6225D96E020E6321DA6ECC
:10494000DF50596F59512C6F2D6BD50E6225D96EE2
:10495000020E6321DA6EDF505A6F5B6B390E5A25F7
:10496000F66ED20E5B21F76EF86A000EF822080090
:10497000F5502E6F2F6BD8906235D96E6335DA6E95
:10498000C50ED926020EDA226F0078FF30F16F00D3
:1049900074FF31F1F0EC03F01E0E256E030E266E4F
:1049A0008EECFBF00101624B632B63BFB1D7635107
:1049B00004E1070E625DD8A0ABD73901A191C2C155
:1049C0005CF1000E01015F6F160E2B6EFF0E2C6E58
:1049D00078EC06F0C9C161F1000E106E39019181C9
:1049E000C0EC0BF01E0E0101246F030E256F450E67
:1049F000266FE90E276F6151020DC50EF324D96EA3
:104A0000020EF420DA6E6F0078FF28F16F0074FF59
:104A100029F1F0EC03F01E0E256E030E266E8EECCF
:104A2000FBF0D50E01016125D96EDA6A020EDA2299
:104A3000DF505E6F010EDDECFBF0090E01015A6FD5
:104A40001E0E596FE40EE82EFED7592FFCD75A2FB1
:104A5000FAD700F0010E00016B6F560E6C6FF60E68
:104A60006D6F6C516D11D8A4000E6E6F010E3AEC93
:104A70000BF0010E00016B6F5E0E6C6FF40E6D6F2C
:104A80006C516D11D8A4000E6E6F020E3AEC0BF053
:104A9000010E00016B6F880E6C6FF40E6D6F6C5120
:104AA0006D11D8A4000E6E6F030E3AEC0BF0000EE1
:104AB0000001666F040E656F000E686F010E676F70
:104AC000390E01015E25F66EF76AD20EF722F86AFA
:104AD000000EF82208006F00D4FF69F0EAECFAF04B
:104AE000000E0001666F040E656F000E686F020E07
:104AF000676F3E0E696FEAECFAF0000E0001666F18
:104B0000040E656F000E686F030E676F200E696FED
:104B1000EAECFAF0040E00016B6F01016151020D25
:104B2000C50EF324D96E020EF420DA6E6F0078FF02
:104B300059F16F0074FF5AF159C16CF05AC16DF010
:104B400000016C516D11D8A4000E6E6F040E3AEC8A
:104B50000BF0000E106E39019181040E1018D8A4CC
:104B600014D0E80E055C030E0658D8B00ED02B0EFC
:104B70003D01EA6F0101612B6151800A790FD8A0D4
:104B800002D0000E616F39019191080E1018D8A45F
:104B900011D0E80E055C030E0658D8B00BD02D0ED0
:104BA0003D01EA6F0101610761AF02D0060E616F3E
:104BB00039019191040E1018D8B404D0080E1018C1
:104BC000D8A474D0000E106E1E0E0101246F030EC7
:104BD000256F520E266FFD0E276F6151020DC50E17
:104BE000F324D96E020EF420DA6E6F0078FF28F1FC
:104BF0006F0074FF29F1F0EC03F01E0E256E030E1A
:104C0000266E8EECFBF0D50E01016125D96EDA6AB5
:104C1000020EDA22DF505E6F000E0001666F040E96
:104C2000656F000E686F010E676F390E01015E251A
:104C3000F66EF76AD20EF722F86A000EF822080024
:104C40006F00D4FF69F0EAECFAF0040E00016B6F1C
:104C500001016151020DC50EF324D96E020EF4203C
:104C6000DA6E6F0078FF59F16F0074FF5AF159C185
:104C70006CF05AC16DF000016C516D11D8A4000E9A
:104C80006E6F040E3AEC0BF0010E01015F6F2A0EFD
:104C90002B6EFF0E2C6E78EC06F0000E106EC0EC42
:104CA0000BF0000E3A01576F39019181020E101876
:104CB000D8A4D9D0E90E055C030E0658D8A0D3D0ED
:104CC000000E106E39019191C0EC0BF0D50E010170
:104CD0006125D96EDA6A020EDA22DF505E6F1E0E8F
:104CE000246F030E256F330E266FDE0E276F5E5185
:104CF000286F296B28BF2907390E5E25F66EF76AE3
:104D0000D20EF722F86A000EF8220800F5502A6F3A
:104D10002B6B6151020DC50EF324D96E020EF420E7
:104D2000DA6E6F0078FF2CF16F0074FF2DF1F0EC5C
:104D300003F01E0E256E030E266E8EECFBF0000EA9
:104D40000001666F040E656F000E686F010E676FDD
:104D5000390E01015E25F66EF76AD20EF722F86A67
:104D6000000EF82208006F00D4FF69F0EAECFAF0B8
:104D7000000E0001666F040E656F000E686F020E74
:104D8000676F200E696FEAECFAF0000E0001666FA3
:104D9000040E656F000E686F030E676F200E696F5B
:104DA000EAECFAF001015E5103ECD6F00101615129
:104DB00061255D6F000E0001666F040E656F000EC9
:104DC000686F040E676F280E01015D25F66EF76AA5
:104DD000D20EF722F86A000EF82208006F00D4FF06
:104DE00069F0EAECFAF0000E0001666F040E656FE0
:104DF000000E686F050E676F5DC159F101015A6BB6
:104E000059BF5A07010E5927000E5A23280E59255B
:104E1000F66ED20E5A21F76EF86A000EF8220800DC
:104E20006F00D4FF69F0EAECFAF0000E0001666F43
:104E3000040E656F000E686F060E676F200E696FB7
:104E4000EAECFAF0020E8EEC05F0020E01015F6F43
:104E50003E0E2B6EFF0E2C6E78EC06F0C0EC0BF0C5
:104E6000000E106E91811004D8B484D001015F51FE
:104E7000800A7E0FD8B04FD0000E0001666F040E7E
:104E8000656F000E686F020E676F200E696FEAECA7
:104E9000FAF0000E0001666F020E656F000E686F7B
:104EA000080E676F2A0E696FEAECFAF0190E01011D
:104EB0005A6F5A0E596FB10EE82EFED7592FFCD7F4
:104EC0005A2FFAD700D0000E0001666F020E656FF0
:104ED000000E686F080E676F200E696FEAECFAF03B
:104EE000000E0001666F040E656F000E686F020E03
:104EF000676F3E0E696FEAECFAF0190E01015A6F06
:104F00005A0E596FB10EE82EFED7592FFCD75A2FE3
:104F1000FAD700D026D0000E0001666F020E656F32
:104F2000000E686F080E676F200E696FEAECFAF0EA
:104F3000000E0001666F040E656F000E686F020EB2
:104F4000676F200E696FEAECFAF0290E01015A6FC3
:104F5000960E596F7F0EE82EFED7592FFCD75A2F89
:104F6000FAD73901A3BF06D001015F51800A7E0F35
:104F7000D8A0F3D53901A3BF03D01004D8A416D00C
:104F80000B0E00016B6FDF0E6C6FFE0E6D6F6C51C0
:104F90006D11D8A4000E6E6F020E3AEC0BF0440EA9
:104FA0002B6EFD0E2C6E78EC06F097D2000E106E74
:104FB000C0EC0BF0A60E2B6EE40E2C6E78EC06F017
:104FC00001016151020DC50EF324D96E020EF420C9
:104FD000DA6E6F0078FF2BF06F0074FF2CF078EC26
:104FE00006F032EC0CF0010E00016B6F350E6C6FA9
:104FF000F90E6D6F6C516D11D8A4000E6E6F010E1D
:105000003AEC0BF0010E00016B6F5E0E6C6FF40E4C
:105010006D6F6C516D11D8A4000E6E6F020E3AECDC
:105020000BF00A0E0101C26F000E606F030E5F6F7E
:10503000520E2B6EFF0E2C6E78EC06F0040E10183C
:10504000D8A414D0E80E055C030E0658D8B00ED0D4
:105050002B0E3D01EA6F0101602B6051800A760F33
:10506000D8A002D0000E606F39019191080E10187F
:10507000D8A411D0E80E055C030E0658D8B00BD0AA
:105080002D0E3D01EA6F0101600760AF02D0090EED
:10509000606F39019191040E1018D8B404D0080E35
:1050A0001018D8A429D1000E106E39019191C0ECCE
:1050B0000BF0040E01015F6F660E2B6EFF0E2C6E5F
:1050C00078EC06F01E0E0101246F030E256FC30E4F
:1050D000266FEA0E276F6151020DC50EF324D96EBB
:1050E000020EF420DA6E6F0078FF28F16F0074FF73
:1050F00029F160512A6F2B6B2ABF2B07390E6025CF
:10510000F66EF76AD20EF722F86A000EF82208004F
:10511000F5502C6F2D6BF0EC03F01E0E256E030E78
:10512000266E8EECFBF0000E0001666F030E656FBD
:10513000000E686F070E676F4D0E696FEAECFAF0AC
:105140000101615161255D6F010E00016B6FAC0EB5
:105150006C6FFF0E6D6F6C516D11D8A4000E6E6FE9
:10516000040E3AEC0BF0000E0001666F040E656F42
:10517000000E686F030E676F280E01015D25F66E45
:10518000F76AD20EF722F86A000EF82208006F00C4
:10519000D4FF69F0EAECFAF0000E0001666F040E2D
:1051A000656F000E686F040E676F5DC159F10101F4
:1051B0005A6B59BF5A07010E5927000E5A23280E61
:1051C0005925F66ED20E5A21F76EF86A000EF822B3
:1051D00008006F00D4FF69F0EAECFAF0000E00015D
:1051E000666F040E656F000E686F010E676F390EF3
:1051F00001016025F66EF76AD20EF722F86A000EFA
:10520000F82208006F00D4FF69F0EAECFAF0000E13
:105210000101636F000E626F000E0001666F030EE6
:10522000656F090E010162250001676F000E010123
:1052300063210001686F01016051200D260E596F36
:10524000060E5A6FF3505927F4505A2362515925CC
:10525000D96E63515A21DA6EDF500001696FEAECB2
:10526000FAF0000E0001666F040E656F090E010171
:1052700062250001676F000E010163210001686F64
:1052800001016051200D260E596F060E5A6F0C0E4B
:105290005927000E5A23F3505927F4505A236251CC
:1052A0005925D96E63515A21DA6EDF500001696FBA
:1052B000EAECFAF00101624B632B63BFADD7635197
:1052C00004E10C0E625DD8A0A7D7150E01015A6F3C
:1052D0004B0E596FBE0EE82EFED7592FFCD75A2F12
:1052E000FAD700F0C0EC0BF0000E106E000E3A0181
:1052F000576F390191810CD0290E01015A6F960E1A
:10530000596F7F0EE82EFED7592FFCD75A2FFAD7A8
:10531000100E1018D8A4C7D0E90E055C030E06586D
:10532000D8A0C1D039019191D50E01016125D96E66
:10533000DA6A020EDA22600083F5DFFF1E0E246FA8
:10534000030E256F9F0E266FDE0E276F390E602528
:10535000F66EF76AD20EF722F86A000EF8220800FD
:10536000F550286F296B6151020DC50EF324D96EDB
:10537000020EF420DA6E6F0078FF2AF16F0074FFDE
:105380002BF1F0EC03F01E0E256E030E266E8EEC54
:10539000FBF0000E106E050E01015F6F5C0E2B6EB0
:1053A000FF0E2C6E78EC06F0B60E2B6ED80E2C6E1F
:1053B00078EC06F0B30E2B6EF90E2C6E78EC06F03E
:1053C000000E0101636F000E626F1E0E246F030E4C
:1053D000256FBF0E266FE10E276F62C128F163C1F2
:1053E00029F1880E62252A6F000E63212B6FD50EDE
:1053F0006225D96E020E6321DA6EDF50596F595162
:105400002C6F2D6BD50E6225D96E020E6321DA6EDC
:10541000DF505A6F5B6B390E5A25F66ED20E5B2148
:10542000F76EF86A000EF8220800F5502E6F2F6B09
:10543000D8906235D96E6335DA6EC50ED926020E64
:10544000DA226F0078FF30F16F0074FF31F1F0EC79
:1054500003F01E0E256E030E266E8EECFBF0880EFA
:1054600001016225256E000E6321266ED50E622590
:10547000D96E020E6321DA6EDF50276EEBEC02F07C
:105480000101624B632B63BFA0D7635104E1070E98
:10549000625DD8A09AD732EC0CF039019181000EF0
:1054A000106EC0EC0BF01004D8A409D0E90E055C16
:1054B000030E0658D8A003D0000E01015F6F39011A
:1054C000A3BF0BD001015F51800A7D0FD8A005D08A
:1054D0005F51800A7B0FD8A0B1D53901A3BF0CD092
:1054E000050E01015F19D8A407D09D0E2B6EEF0E9B
:1054F0002C6E78EC06F006D00A0E2B6EF40E2C6E95
:1055000078EC06F05CC1C2F1040E0F6E000E106E56
:10551000C0EC0BF0010EDDECFBF0090E01015A6F3F
:105520001E0E596FE40EE82EFED7592FFCD75A2FC6
:10553000FAD700F01200EF0E2B6EE10E2C6E78EC15
:1055400006F0820E2B6ED70E2C6E78EC06F01E0E37
:105550000101246F030E256F790E266FE40E276F6D
:10556000F0EC03F01E0E256E030E266E8EECFBF0A3
:10557000010EDDECFBF0010E00016B6F9D0E6C6FF8
:10558000F40E6D6F6C516D11D8A4000E6E6F010E8C
:105590003AEC0BF06F0030FF67F1050E0101686F08
:1055A000D8906733682FFCD767A1F4D7010EDDECE4
:1055B000FBF0010E00016B6F020E6C6FF60E6D6F4B
:1055C0006C516D11D8A4000E6E6F010E3AEC0BF009
:1055D000010E00016B6F950E6C6FF60E6D6F6C51C6
:1055E0006D11D8A4000E6E6F020E3AEC0BF0010E96
:1055F00000016B6F170E6C6FF60E6D6F6C516D11B5
:10560000D8A4000E6E6F030E3AEC0BF0010E0001F1
:105610006B6F390E6C6FF80E6D6F6C516D11D8A4F5
:10562000000E6E6F040E3AEC0BF0BA8CBA980FD0E5
:10563000BA7CBA78020E0101686FA00E676F920EF5
:10564000E82EFED7672FFCD7682FFAD700F06F003F
:1056500030FF67F1050E0101686FD8906733682F3E
:10566000FCD767B1E5D7000ED16F000ED06F19D00F
:10567000090E0101686F1E0E676FE40EE82EFED75B
:10568000672FFCD7682FFAD700F00101D04BD12B40
:10569000BA7CBA780101D1510FE1150ED05DD8B0B6
:1056A0000BD06F0030FF67F1050E686FD89067333D
:1056B000682FFCD767A1DCD7D15137E1140ED05D3C
:1056C000D8B033D0000E00016C6F010E6B6FA9ECE7
:1056D000F4F0000E00016C6F020E6B6FA9ECF4F099
:1056E000010E00016B6F890E6C6FF90E6D6F6C51BE
:1056F0006D11D8A4000E6E6F030E3AEC0BF0010E84
:1057000000016B6F840E6C6FF50E6D6F6C516D1137
:10571000D8A4000E6E6F040E3AEC0BF0040E8EEC63
:1057200005F0000E0101B26FFF00010E00016B6F6A
:10573000170E6C6FFA0E6D6F6C516D11D8A4000EC0
:105740006E6F040E3AEC0BF0020E8EEC05F0250E97
:105750002B6EED0E2C6E78EC06F0010EDDECFBF0FE
:105760005AECF8F06DC094F16EC095F16FC096F1EF
:1057700070C097F1A8C124F1A9C125F1530E010110
:10578000266FFA0E276F94C128F195C129F196C1B1
:105790002AF197C12BF1000E2D6FB00E2C6FF0EC9B
:1057A00003F0A8C125F0A9C126F08EECFBF032EC85
:1057B0000CF0010120EE11F0A851D926A951DA22EE
:1057C000070EDF6E010E00016A6FA8C16BF0A9C160
:1057D0006CF0020EEEEC0BF0F5ECF7F06DC090F112
:1057E0006EC091F16FC092F170C093F1A8C124F125
:1057F000A9C125F1670E0101266FFA0E276F90C12E
:1058000028F191C129F192C12AF193C12BF1000E27
:105810002D6FB00E2C6FF0EC03F0A8C125F0A9C1DC
:1058200026F08EECFBF032EC0CF0010120EE11F0D2
:10583000A851D926A951DA22070EDF6E010E000108
:105840006A6FA8C16BF0A9C16CF0030EEEEC0BF00F
:10585000BFECF8F06DC08CF16EC08DF16FC08EF1B1
:1058600070C08FF1A8C124F1A9C125F17B0E0101FF
:10587000266FFA0E276F8CC128F18DC129F18EC1D8
:105880002AF18FC12BF1000E2D6FB00E2C6FF0ECB2
:1058900003F0A8C125F0A9C126F08EECFBF032EC94
:1058A0000CF0010120EE11F0A851D926A951DA22FD
:1058B000070EDF6E010E00016A6FA8C16BF0A9C16F
:1058C0006CF0040EEEEC0BF0020E8EEC05F090C1C5
:1058D0007AF091C17BF092C17CF093C17DF094C1CC
:1058E00076F095C177F096C178F097C179F099EC90
:1058F000E0F076C000F677C001F678C002F679C015
:1059000003F68CC17AF08DC17BF08EC17CF08FC123
:105910007DF000C676F001C677F002C678F003C6C7
:1059200079F099ECE0F076C086F077C087F078C027
:1059300088F079C089F0000E8A6F000E8B6F400EE0
:105940008C6F400E8D6F75ECE3F086C098F187C0C8
:1059500099F188C09AF189C09BF1A8C124F1A9C12D
:1059600025F18F0E0101266FFA0E276F98C128F1DD
:1059700099C129F19AC12AF19BC12BF1000E2D6F1B
:10598000B00E2C6FF0EC03F0A8C125F0A9C126F0F1
:105990008EECFBF032EC0CF0010120EE11F0A8517E
:1059A000D926A951DA22070EDF6E010E00016A6FB7
:1059B000A8C16BF0A9C16CF0010EEEEC0BF0030E68
:1059C0008EEC05F0530E2B6EED0E2C6E78EC06F07F
:1059D00098C186F099C187F09AC188F09BC189F07F
:1059E00094C18AF095C18BF096C18CF097C18DF06F
:1059F0006AEC05F086C070F187C071F188C072F161
:105A000089C073F198C186F099C187F09AC188F076
:105A10009BC189F090C18AF091C18BF092C18CF04A
:105A200093C18DF06AEC05F086C074F187C075F102
:105A300088C076F189C077F198C186F099C187F066
:105A40009AC188F09BC189F08CC18AF08DC18BF01E
:105A50008EC18CF08FC18DF06AEC05F086C078F1B4
:105A600087C079F188C07AF189C07BF1AD0E2B6EC9
:105A7000E70E2C6E78EC06F0010EDDECFBF0010E6B
:105A800000016B6FE10E6C6FF80E6D6F6C516D1154
:105A9000D8A4000E6E6F010E3AEC0BF0000E000160
:105AA0006C6F020E6B6FA9ECF4F01E0E0101246FF7
:105AB000030E256FFD0E266FEF0E276F94C128F1A0
:105AC00095C129F196C12AF197C12BF1000E2D6FD6
:105AD000070E2C6F70C12EF171C12FF172C130F120
:105AE00073C131F1000E336F070E326FF0EC03F02B
:105AF000010E00016A6F1E0E6B6F030E6C6F020EBB
:105B0000EEEC0BF01E0E0101246F030E256F150E37
:105B1000266FF00E276F90C128F191C129F192C133
:105B20002AF193C12BF1000E2D6F070E2C6F74C15B
:105B30002EF175C12FF176C130F177C131F1000E30
:105B4000336F070E326FF0EC03F0010E00016A6F45
:105B50001E0E6B6F030E6C6F030EEEEC0BF01E0E41
:105B60000101246F030E256F2D0E266FF00E276F97
:105B70008CC128F18DC129F18EC12AF18FC12BF181
:105B8000000E2D6F070E2C6F78C12EF179C12FF109
:105B90007AC130F17BC131F1000E336F070E326FE5
:105BA000F0EC03F0010E00016A6F1E0E6B6F030E26
:105BB0006C6F040EEEEC0BF0A8C124F1A9C125F125
:105BC000F40E0101266FE90E276F94C128F195C1EB
:105BD00029F196C12AF197C12BF1000E2D6FB00E5D
:105BE0002C6F70C12EF171C12FF172C130F173C1F0
:105BF00031F1F0EC03F0A8C125F0A9C126F08EEC3C
:105C0000FBF032EC0CF0A8C124F1A9C125F1170E6C
:105C10000101266FEA0E276F90C128F191C129F189
:105C200092C12AF193C12BF1000E2D6FB00E2C6F93
:105C300074C12EF175C12FF176C130F177C131F108
:105C4000F0EC03F0A8C125F0A9C126F08EECFBF022
:105C500032EC0CF0A8C124F1A9C125F13A0E0101E2
:105C6000266FEA0E276F8CC128F18DC129F18EC1F4
:105C70002AF18FC12BF1000E2D6FB00E2C6F78C161
:105C80002EF179C12FF17AC130F17BC131F1F0EC05
:105C900003F0A8C125F0A9C126F08EECFBF032EC90
:105CA0000CF0040E8EEC05F0010EDDECFBF0010EA5
:105CB00000016B6FC10E6C6FF20E6D6F6C516D1148
:105CC000D8A4000E6E6F010E3AEC0BF0010E00012D
:105CD0006B6FED0E6C6FF20E6D6F6C516D11D8A481
:105CE000000E6E6F020E3AEC0BF0010E00016B6FAE
:105CF000AB0E6C6FF20E6D6F6C516D11D8A4000E6F
:105D00006E6F030E3AEC0BF0C30E2B6EE30E2C6E8F
:105D100078EC06F0000E0101D16F000ED06FBA8C46
:105D2000BA980FD0BA7CBA78020E0101686FA00E43
:105D3000676F920EE82EFED7672FFCD7682FFAD731
:105D400000F06F0030FF67F1050E0101686FD89019
:105D50006733682FFCD767B1E5D7000ED16F000E0F
:105D6000D06F19D0090E0101686F1E0E676FE40E27
:105D7000E82EFED7672FFCD7682FFAD700F0010175
:105D8000D04BD12BBA7CBA780101D1510FE1150E5D
:105D9000D05DD8B00BD06F0030FF67F1050E686F93
:105DA000D8906733682FFCD767A1DCD76F0030FF2E
:105DB00067F1050E686FD8906733682FFCD767B11D
:105DC00049D0D15104E1140ED05DD8A043D0BA8C93
:105DD000BA98400E2B6EDA0E2C6E78EC06F0D5ECED
:105DE000FFF0240E2B6EE60E2C6E78EC06F0010E02
:105DF000DDECFBF0010E00016B6F990E6C6FF50E80
:105E00006D6F6C516D11D8A4000E6E6F010E3AECDF
:105E10000BF0010E00016B6F450E6C6FF50E6D6F90
:105E20006C516D11D8A4000E6E6F020E3AEC0BF09F
:105E3000010E00016B6FDC0E6C6FF40E6D6F6C5118
:105E40006D11D8A4000E6E6F030E3AEC0BF0030E2A
:105E50008EEC05F0DD0E2B6EDC0E2C6E78EC06F071
:105E6000BDEC02F070C176F071C177F072C178F0CC
:105E700073C179F094C17AF095C17BF096C17CF042
:105E800097C17DF099ECE0F076C004F677C005F696
:105E900078C006F679C007F61E0E0101246F030EC6
:105EA000256F8F0E266FEC0E276F04C628F105C6EE
:105EB00029F106C62AF107C62BF1F0EC03F01E0EFD
:105EC000256E030E266E8EECFBF074C176F075C164
:105ED00077F076C178F077C179F090C17AF091C10E
:105EE0007BF092C17CF093C17DF099ECE0F076C03C
:105EF00004F677C005F678C006F679C007F61E0EE0
:105F00000101246F030E256FAB0E266FEC0E276F79
:105F100004C628F105C629F106C62AF107C62BF1E9
:105F2000F0EC03F01E0E256E030E266E8EECFBF0D9
:105F300078C176F079C177F07AC178F07BC179F0D9
:105F40008CC17AF08DC17BF08EC17CF08FC17DF069
:105F500099ECE0F076C004F677C005F678C006F656
:105F600079C007F61E0E0101246F030E256FC70EC0
:105F7000266FEC0E276F04C628F105C629F106C668
:105F80002AF107C62BF1F0EC03F01E0E256E030E6E
:105F9000266E8EECFBF0030E8EEC05F032EC0CF06E
:105FA000000E2B6ED90E2C6E78EC06F0BA9C010E0A
:105FB000DDECFBF0010E00016B6F630E6C6FF80EF1
:105FC0006D6F6C516D11D8A4000E6E6F010E3AEC1E
:105FD0000BF0010E00016B6F060E6C6FF50E6D6F0E
:105FE0006C516D11D8A4000E6E6F020E3AEC0BF0DE
:105FF000010E00016B6F670E6C6FF70E6D6F6C51C9
:106000006D11D8A4000E6E6F030E3AEC0BF0010E6A
:1060100000016B6FF10E6C6FF40E6D6F6C516D11B2
:10602000D8A4000E6E6F040E3AEC0BF0BA78090E8D
:106030000101686F1E0E676FE40EE82EFED7672F12
:10604000FCD7682FFAD700F0F1D7010E01015D6F80
:10605000010E0E6E020E0D6E000E106EDEC188F186
:10606000DFC189F1E0C18AF1E1C18BF1DAC184F1CC
:10607000DBC185F1DCC186F1DDC187F1D6C180F1DC
:10608000D7C181F1D8C182F1D9C183F18E0E2B6EB7
:10609000EE0E2C6E78EC06F09E0E256E030E266E2C
:1060A0008EECFBF032EC0CF0010EDDECFBF0090E97
:1060B00001015A6F1E0E596FE40EE82EFED7592FBC
:1060C000FCD75A2FFAD700F09E0E0101246F030E61
:1060D000256FE50E266FF70E276FF0EC03F09E0E8E
:1060E000256E030E266E8EECFBF032EC0CF0010EEA
:1060F00000016A6F9E0E6B6F030E6C6F010EEEEC6B
:106100000BF09E0E0101246F030E256F7C0E266F8F
:10611000F70E276F88C128F189C129F18AC12AF1B8
:106120008BC12BF1F0EC03F09E0E256E030E266E54
:106130008EECFBF032EC0CF0070E0301A76F010EA2
:1061400000016A6F9E0E6B6F030E6C6F020EEEEC19
:106150000BF09E0E0101246F030E256F450E266F76
:10616000F30E276F84C128F185C129F186C12AF178
:1061700087C12BF1F0EC03F09E0E256E030E266E08
:106180008EECFBF032EC0CF0070E0301A76F010E52
:1061900000016A6F9E0E6B6F030E6C6F030EEEECC8
:1061A0000BF09E0E0101246F030E256FDF0E266F8C
:1061B000F30E276F80C128F181C129F182C12AF134
:1061C00083C12BF1F0EC03F09E0E256E030E266EBC
:1061D0008EECFBF032EC0CF0070E0301A76F010E02
:1061E00000016A6F9E0E6B6F030E6C6F040EEEEC77
:1061F0000BF0000E666F020E656F000E686F070EE3
:10620000676F3E0E696FEAECFAF0000E0001666FF0
:10621000020E656F000E686F0C0E676F3E0E696FA1
:10622000EAECFAF0010E8EEC05F0000E106EC0ECF8
:106230000BF01004D8A405D0000E0D6E000E010165
:106240005D6F020E1018D8A49BD0E80E055C030EFB
:106250000658D8B095D00D2A040E0D647BD0020EDE
:106260000D6E78D0000E0001666F020E656F000E95
:10627000686F070E676F3E0E696FEAECFAF0000E6A
:106280000001666F030E656F000E686F070E676F83
:10629000200E696FEAECFAF0000E0001666F040E42
:1062A000656F000E686F070E676F200E696FEAEC6E
:1062B000FAF062D0000E0001666F020E656F000EEC
:1062C000686F070E676F200E696FEAECFAF0000E38
:1062D0000001666F030E656F000E686F070E676F33
:1062E0003E0E696FEAECFAF0000E0001666F040ED4
:1062F000656F000E686F070E676F200E696FEAEC1E
:10630000FAF03AD0000E0001666F020E656F000EC3
:10631000686F070E676F200E696FEAECFAF0000EE7
:106320000001666F030E656F000E686F070E676FE2
:10633000200E696FEAECFAF0000E0001666F040EA1
:10634000656F000E686F070E676F3E0E696FEAECAF
:10635000FAF012D00D500101596F5A6B5A51000AD0
:10636000D8A40AD05951020AD8B47CD7010AD8B4AB
:10637000A1D7070AD8B4C6D7000E106EC0EC0BF038
:10638000020E1018D8A411D0E90E055C030E0658B1
:10639000D8A00BD0000E106EC0EC0BF0010E0D64F7
:1063A00004D00D500A0F01015D6F010E0D6408D07D
:1063B000000E0001716F010E706F22ECF9F003D036
:1063C000010E8EEC05F001015D51D8B406D00A0E25
:1063D0005D6103D03901A3AF2CD73901A3AF02D03F
:1063E000000E0D6E0D50D8B49BD39E0E0101246F8C
:1063F000030E256FCE0E266FFC0E276F5DC128F1B0
:10640000296BF0EC03F09E0E256E030E266E8EECCB
:10641000FBF00DC065F00001666B000E686F070EA3
:10642000676F2A0E696FEAECFAF0110E01015A6FDC
:106430003C0E596FCB0EE82EFED7592FFCD75A2FA2
:10644000FAD7000E106EC0EC0BF0040E1018D8A492
:1064500031D1E80E055C030E0658D8B02BD10C0ED6
:1064600001015D19D8A445D088C186F089C187F0A3
:106470008AC188F08BC189F0000E00018A6F000E7E
:106480008B6FE00E8C6F410E8D6FF2ECF5F0D8B093
:1064900030D088C176F089C177F08AC178F08BC19D
:1064A00079F0000E7A6F000E7B6F000E7C6F3F0E4E
:1064B0007D6F99ECE0F076C088F177C089F178C003
:1064C0008AF179C08BF19E0E0101246F030E256FB6
:1064D000370E266FFE0E276F88C128F189C129F17A
:1064E0008AC12AF18BC12BF1F0EC03F0010E38ECDC
:1064F00006F00D0E01015D19D8A445D084C186F0C7
:1065000085C187F086C188F087C189F0000E00013F
:106510008A6F000E8B6F900E8C6F410E8D6FF2ECB8
:10652000F5F0D8B030D084C176F085C177F086C15F
:1065300078F087C179F0000E7A6F000E7B6F000E45
:106540007C6F3F0E7D6F99ECE0F076C084F177C0F0
:1065500085F178C086F179C087F19E0E0101246F24
:10656000030E256F2A0E266FFE0E276F84C128F1B9
:1065700085C129F186C12AF187C12BF1F0EC03F026
:10658000010E38EC06F00E0E01015D19D8A44FD0B3
:1065900080C186F081C187F082C188F083C189F013
:1065A000000E00018A6F000E8B6F200E8C6F410E63
:1065B0008D6FF2ECF5F0D8B03AD080C176F081C1A1
:1065C00077F082C178F083C179F0000E7A6F000E07
:1065D0007B6F800E7C6F3F0E7D6F99ECE0F076C094
:1065E00080F177C081F178C082F179C083F180C1F8
:1065F000ACF081C1ADF082C1AEF083C1AFF081ECEF
:10660000F9F0ACC05BF1ADC05CF19E0E0101246FEE
:10661000030E256FE90E266FFD0E276F5BC128F173
:106620005CC129F1F0EC03F0010E38EC06F0000E2D
:106630000001666F030E656F000E686F0C0E676FCA
:10664000200E696FEAECFAF0000E0001666F040E8E
:10665000656F000E686F0C0E676F200E696FEAECB5
:10666000FAF0110E01015A6F3C0E596FCB0EE82E55
:10667000FED7592FFCD75A2FFAD7000E0001666FAC
:10668000040E656F000E686F0C0E676F3E0E696F2B
:10669000EAECFAF0110E01015A6F3C0E596FCB0E65
:1066A000E82EFED7592FFCD75A2FFAD7000E106EBE
:1066B000C0EC0BF0080E1018D8A424D1E80E055C2D
:1066C000030E0658D8B01ED10C0E01015D19D8A4D6
:1066D00045D0000E0001866F000E876F800E886F18
:1066E000410E896F88C18AF089C18BF08AC18CF014
:1066F0008BC18DF0F2ECF5F0D8B030D088C176F0D7
:1067000089C177F08AC178F08BC179F0000E7A6F79
:10671000000E7B6F000E7C6FBF0E7D6F99ECE0F07A
:1067200076C088F177C089F178C08AF179C08BF1A1
:106730009E0E0101246F030E256F370E266FFE0E8D
:10674000276F88C128F189C129F18AC12AF18BC13B
:106750002BF1F0EC03F0010E38EC06F00D0E010108
:106760005D19D8A445D0000E0001866F000E876F1A
:10677000400E886F410E896F84C18AF085C18BF00D
:1067800086C18CF087C18DF0F2ECF5F0D8B030D036
:1067900084C176F085C177F086C178F087C179F041
:1067A000000E7A6F000E7B6F000E7C6FBF0E7D6F48
:1067B00099ECE0F076C084F177C085F178C086F17D
:1067C00079C087F19E0E0101246F030E256F2A0EFA
:1067D000266FFE0E276F84C128F185C129F186C17D
:1067E0002AF187C12BF1F0EC03F0010E38EC06F032
:1067F0000E0E01015D19D8A44FD0000E0001866F66
:10680000000E876FA00E886F400E896F80C18AF0DE
:1068100081C18BF082C18CF083C18DF0F2ECF5F078
:10682000D8B03AD080C176F081C177F082C178F0DB
:1068300083C179F0000E7A6F000E7B6F800E7C6F43
:10684000BF0E7D6F99ECE0F076C080F177C081F1EA
:1068500078C082F179C083F180C1ACF081C1ADF024
:1068600082C1AEF083C1AFF081ECF9F0ACC05BF156
:10687000ADC05CF19E0E0101246F030E256FE90E81
:10688000266FFD0E276F5BC128F15CC129F1F0EC8A
:1068900003F0010E38EC06F0000E0001666F030EE7
:1068A000656F000E686F0C0E676F200E696FEAEC63
:1068B000FAF0110E01015A6F3C0E596FCB0EE82E03
:1068C000FED7592FFCD75A2FFAD7000E0001666F5A
:1068D000040E656F000E686F0C0E676F3E0E696FD9
:1068E000EAECFAF0110E01015A6F3C0E596FCB0E13
:1068F000E82EFED7592FFCD75A2FFAD7000E106E6C
:10690000C0EC0BF0100E1018D8A4DFD0E90E055C17
:10691000030E0658D8A0D9D00A0E01015D65D5D066
:10692000C0EC0BF0000E106E01015D510A0F5D6F9F
:10693000160E5D19D8A432D088C1DEF189C1DFF10D
:106940008AC1E0F18BC1E1F19E0E246F030E256F29
:10695000390E266FE30E276FDEC128F1DFC129F162
:10696000E0C12AF1E1C12BF1000E2D6F640E2C6FF6
:10697000F0EC03F0000E2C6E640E2B6EDEC12DF0D9
:10698000DFC12EF0E0C12FF0E1C130F046EC05F0A0
:106990009E0E256E030E266E8EECFBF0170E010187
:1069A0005D19D8A432D084C1DAF185C1DBF186C18A
:1069B000DCF187C1DDF19E0E246F030E256F050EFD
:1069C000266FE00E276FDAC128F1DBC129F1DCC1A7
:1069D0002AF1DDC12BF1000E2D6F680E2C6FF0EC4B
:1069E00003F0000E2C6E680E2B6EDAC12DF0DBC1A9
:1069F0002EF0DCC12FF0DDC130F046EC05F09E0E2C
:106A0000256E030E266E8EECFBF0180E01015D194B
:106A1000D8A432D080C1D6F181C1D7F182C1D8F1DA
:106A200083C1D9F19E0E246F030E256F690E266F68
:106A3000E00E276FD6C128F1D7C129F1D8C12AF1BC
:106A4000D9C12BF1000E2D6F6C0E2C6FF0EC03F002
:106A50009E0E256E030E266E8EECFBF0000E2C6E45
:106A60006C0E2B6EDAC12DF0DBC12EF0DCC12FF0E5
:106A7000DDC130F046EC05F0000E106EC0EC0BF0FE
:106A8000080E00016B6F600E6C6FFD0E6D6F6C5128
:106A90006D11D8A4000E6E6F0D503AEC0BF0030E82
:106AA0008EEC05F0080E00016B6FB20E6C6FEE0EEF
:106AB0006D6F6C516D11D8A4000E6E6F0D503AECD5
:106AC0000BF0000E106EC0EC0BF0140E01015D65B2
:106AD0000AD0000E106EDD0E2B6EFC0E2C6E78ECC4
:106AE00006F025EFB0F0AAEC07F0010E0D640ED011
:106AF00001015D51D8B40AD00A0E5D6107D00EC005
:106B000070F00001716B22ECF9F003D0010E8EECF5
:106B100005F03901A3BF04D0020E01015D6195D4D7
:106B2000010E0E6E3EECFBF01200040E0E6E020E15
:106B30000D6E010E0001FF6F000E106EC0EC0BF029
:106B4000E5C288F1E6C289F1E7C28AF1E8C28BF1B9
:106B5000E1C284F1E2C285F1E3C286F1E4C287F1C9
:106B6000DDC280F1DEC281F1DFC282F1E0C283F1D9
:106B7000750E2B6EEE0E2C6E78EC06F0010EDDEC31
:106B8000FBF0090E01015A6F1E0E596FE40EE82E3C
:106B9000FED7592FFCD75A2FFAD700F09E0E0101CD
:106BA000246F030E256FFA0E266FF70E276FF0EC99
:106BB00003F09E0E256E030E266E8EECFBF032EC7B
:106BC0000CF0010E00016A6F9E0E6B6F030E6C6F6E
:106BD000010EEEEC0BF09E0E0101246F030E256FEB
:106BE0002F0E266FF30E276F88C128F189C129F176
:106BF0008AC12AF18BC12BF1F0EC03F09E0E256EB9
:106C0000030E266E8EECFBF032EC0CF0070E030147
:106C1000A76F010E00016A6F9E0E6B6F030E6C6F03
:106C2000020EEEEC0BF09E0E0101246F030E256F99
:106C3000880E266FF10E276F84C128F185C129F1D6
:106C400086C12AF187C12BF1F0EC03F09E0E256E70
:106C5000030E266E8EECFBF032EC0CF0070E0301F7
:106C6000A76F010E00016A6F9E0E6B6F030E6C6FB3
:106C7000030EEEEC0BF09E0E0101246F030E256F48
:106C8000B60E266FF10E276F80C128F181C129F160
:106C900082C12AF183C12BF1F0EC03F09E0E256E28
:106CA000030E266E8EECFBF032EC0CF0070E0301A7
:106CB000A76F010E00016A6F9E0E6B6F030E6C6F63
:106CC000040EEEEC0BF0000E666F020E656F000E08
:106CD000686F070E676F3E0E696FEAECFAF0000E00
:106CE0000001666F020E656F000E686F0C0E676F15
:106CF0003E0E696FEAECFAF0010E8EEC05F0000E24
:106D0000106EC0EC0BF01004D8A405D0000E0D6E70
:106D1000000E0001FF6F020E1018D8A49BD0E80EE1
:106D2000055C030E0658D8B095D00D2A040E0D64EC
:106D30007BD0020E0D6E78D0000E0001666F020E41
:106D4000656F000E686F070E676F3E0E696FEAECA5
:106D5000FAF0000E0001666F030E656F000E686F9B
:106D6000070E676F200E696FEAECFAF0000E000163
:106D7000666F040E656F000E686F070E676F200E5A
:106D8000696FEAECFAF062D0000E0001666F020E45
:106D9000656F000E686F070E676F200E696FEAEC73
:106DA000FAF0000E0001666F030E656F000E686F4B
:106DB000070E676F3E0E696FEAECFAF0000E0001F5
:106DC000666F040E656F000E686F070E676F200E0A
:106DD000696FEAECFAF03AD0000E0001666F020E1D
:106DE000656F000E686F070E676F200E696FEAEC23
:106DF000FAF0000E0001666F030E656F000E686FFB
:106E0000070E676F200E696FEAECFAF0000E0001C2
:106E1000666F040E656F000E686F070E676F3E0E9B
:106E2000696FEAECFAF012D00D500101596F5A6BFC
:106E30005A51000AD8A40AD05951020AD8B47CD7B2
:106E4000010AD8B4A1D7070AD8B4C6D7000E106E6D
:106E5000C0EC0BF0020E1018D8A411D0E90E055C9E
:106E6000030E0658D8A00BD0000E106EC0EC0BF02D
:106E7000010E0D6404D00D500A0F0001FF6F010ECA
:106E80000D6407D0000E0001716F040E706F22ECCC
:106E9000F9F00001FF51D8B406D00A0EFF6103D00B
:106EA0003901A3AF30D73901A3AF02D0000E0D6E68
:106EB0000D50D8B473D39E0E0101246F030E256FBD
:106EC000CE0E266FFC0E276FFFC028F1296BF0EC69
:106ED00003F09E0E256E030E266E8EECFBF00DC0A9
:106EE00065F00001666B000E686F070E676F2A0E73
:106EF000696FEAECFAF0110E01015A6F3C0E596FFE
:106F0000CB0EE82EFED7592FFCD75A2FFAD7000EFA
:106F1000106EC0EC0BF0040E1018D8A415D1E80EBA
:106F2000055C030E0658D8B00FD10C0E0001FF19F6
:106F3000D8A444D088C186F089C187F08AC188F07E
:106F40008BC189F0000E8A6F000E8B6FC00E8C6FA4
:106F50003F0E8D6FF2ECF5F0D8B030D088C176F0EE
:106F600089C177F08AC178F08BC179F0000E7A6F11
:106F7000000E7B6F000E7C6F3F0E7D6F99ECE0F092
:106F800076C088F177C089F178C08AF179C08BF139
:106F90009E0E0101246F030E256F8A0E266FFD0ED3
:106FA000276F88C128F189C129F18AC12AF18BC1D3
:106FB0002BF1F0EC03F0010E38EC06F00D0EFF198A
:106FC000D8A444D084C186F085C187F086C188F0FA
:106FD00087C189F0000E8A6F000E8B6FC00E8C6F18
:106FE0003F0E8D6FF2ECF5F0D8B030D084C176F062
:106FF00085C177F086C178F087C179F0000E7A6F8D
:10700000000E7B6F000E7C6F3F0E7D6F99ECE0F001
:1070100076C084F177C085F178C086F179C087F1B8
:107020009E0E0101246F030E256FB40E266FFD0E18
:10703000276F84C128F185C129F186C12AF187C152
:107040002BF1F0EC03F0010E38EC06F00E0EFF19F8
:10705000D8A444D080C186F081C187F082C188F075
:1070600083C189F0000E8A6F000E8B6F400E8C6F0B
:10707000400E8D6FF2ECF5F0D8B030D080C176F0D4
:1070800081C177F082C178F083C179F0000E7A6F08
:10709000000E7B6F800E7C6F3F0E7D6F99ECE0F0F1
:1070A00076C080F177C081F178C082F179C083F138
:1070B0009E0E0101246F030E256FA60E266FFD0E96
:1070C000276F80C128F181C129F182C12AF183C1D2
:1070D0002BF1F0EC03F0010E38EC06F0000E666FB9
:1070E000030E656F000E686F0C0E676F200E696FE0
:1070F000EAECFAF0110E01015A6F3C0E596FCB0EFB
:10710000E82EFED7592FFCD75A2FFAD7000E0001D0
:10711000666F030E656F000E686F0C0E676F200EB2
:10712000696FEAECFAF0000E0001666F040E656FFD
:10713000000E686F0C0E676F3E0E696FEAECFAF096
:10714000000E106EC0EC0BF0080E1018D8A415D16C
:10715000E80E055C030E0658D8B00FD10C0E0001E6
:10716000FF19D8A444D0000E866F000E876F000E62
:10717000886F3F0E896F88C18AF089C18BF08AC100
:107180008CF08BC18DF0F2ECF5F0D8B030D088C126
:1071900076F089C177F08AC178F08BC179F0000E62
:1071A0007A6F000E7B6F000E7C6FBF0E7D6F99ECC7
:1071B000E0F076C088F177C089F178C08AF179C0B3
:1071C0008BF19E0E0101246F030E256F8A0E266F30
:1071D000FD0E276F88C128F189C129F18AC12AF1E2
:1071E0008BC12BF1F0EC03F0010E38EC06F00D0E24
:1071F000FF19D8A444D0000E866F000E876F000ED2
:10720000886F3F0E896F84C18AF085C18BF086C17B
:107210008CF087C18DF0F2ECF5F0D8B030D084C19D
:1072200076F085C177F086C178F087C179F0000EDD
:107230007A6F000E7B6F000E7C6FBF0E7D6F99EC36
:10724000E0F076C084F177C085F178C086F179C02E
:1072500087F19E0E0101246F030E256F980E266F95
:10726000FD0E276F84C128F185C129F186C12AF15D
:1072700087C12BF1F0EC03F0010E38EC06F00E0E96
:10728000FF19D8A444D0000E866F000E876F800EC1
:10729000886F3F0E896F80C18AF081C18BF082C1F7
:1072A0008CF083C18DF0F2ECF5F0D8B030D080C115
:1072B00076F081C177F082C178F083C179F0000E59
:1072C0007A6F000E7B6F800E7C6FBF0E7D6F99EC26
:1072D000E0F076C080F177C081F178C082F179C0AA
:1072E00083F19E0E0101246F030E256FA60E266FFB
:1072F000FD0E276F80C128F181C129F182C12AF1D9
:1073000083C12BF1F0EC03F0010E38EC06F0000E17
:10731000666F030E656F000E686F0C0E676F200EB0
:10732000696FEAECFAF0110E01015A6F3C0E596FC9
:10733000CB0EE82EFED7592FFCD75A2FFAD7000EC6
:107340000001666F030E656F000E686F0C0E676FAD
:10735000200E696FEAECFAF0000E0001666F040E71
:10736000656F000E686F0C0E676F3E0E696FEAEC7A
:10737000FAF0000E106EC0EC0BF0100E1018D8A42E
:10738000E2D0E90E055C030E0658D8A0DCD00A0E48
:107390000001FF65D8D0C0EC0BF0000E106E0001AC
:1073A000FF510A0FFF6F160EFF19D8A433D088C102
:1073B000E5F289C1E6F28AC1E7F28BC1E8F29E0EDE
:1073C0000101246F030E256F5F0E266FE10E276FFC
:1073D000E5C228F1E6C229F1E7C22AF1E8C22BF1A1
:1073E000000E2D6F700E2C6FF0EC03F0000E2C6E63
:1073F000700E2B6EE5C22DF0E6C22EF0E7C22FF024
:10740000E8C230F046EC05F09E0E256E030E266EA7
:107410008EECFBF0170E0001FF19D8A433D084C105
:10742000E1F285C1E2F286C1E3F287C1E4F29E0E89
:107430000101246F030E256FFD0E266FE00E276FEE
:10744000E1C228F1E2C229F1E3C22AF1E4C22BF140
:10745000000E2D6F740E2C6FF0EC03F0000E2C6EEE
:10746000740E2B6EE1C22DF0E2C22EF0E3C22FF0BB
:10747000E4C230F046EC05F09E0E256E030E266E3B
:107480008EECFBF0180E0001FF19D8A433D080C198
:10749000DDF281C1DEF282C1DFF283C1E0F29E0E35
:1074A0000101246F030E256FCC0E266FE00E276FAF
:1074B000DDC228F1DEC229F1DFC22AF1E0C22BF1E0
:1074C000000E2D6F780E2C6FF0EC03F09E0E256EE3
:1074D000030E266E8EECFBF0000E2C6E780E2B6EDB
:1074E000DDC22DF0DEC22EF0DFC22FF0E0C230F0A0
:1074F00046EC05F0000E106EC0EC0BF0080E00011B
:107500006B6F600E6C6FFD0E6D6F6C516D11D8A4BA
:10751000000E6E6F0D503AEC0BF0030E8EEC05F082
:10752000080E00016B6FB20E6C6FEE0E6D6F6C513A
:107530006D11D8A4000E6E6F0D503AEC0BF0000EDA
:10754000106EC0EC0BF0140E0001FF650AD0000EA7
:10755000106EFB0E2B6EFC0E2C6E78EC06F095EF89
:10756000B5F0AAEC07F0010E0D640ED00001FF513A
:10757000D8B40AD00A0EFF6107D0000E716F040E56
:10758000706F22ECF9F003D0010E8EEC05F039019A
:10759000A3BF04D0020E0001FF61BDD4040E0E6E25
:1075A0003EECFBF01200000E106EC0EC0BF0030E70
:1075B0000E6E020E0D6E010E01015D6F000E106E5B
:1075C000E2C188F1E3C189F1E4C18AF1E5C18BF13F
:1075D000E6C184F1E7C185F1E8C186F1E9C187F12F
:1075E000E9C2ACF0EAC2ADF0EBC2AEF0ECC2AFF073
:1075F00081ECF9F0ACC0B6F0ADC0B7F0EBEC08F040
:10760000B6C05BF1B7C05CF1D90E2B6EED0E2C6EDF
:1076100078EC06F0010EDDECFBF0090E01015A6F6B
:107620001E0E596FE40EE82EFED7592FFCD75A2FA5
:10763000FAD700F09E0E0101246F030E256FBB0EDA
:10764000266FF70E276FF0EC03F09E0E256E030EEB
:10765000266E8EECFBF032EC0CF0010E00016A6F2E
:107660009E0E6B6F030E6C6F010EEEEC0BF09E0E18
:107670000101246F030E256FFE0E266FF00E276F9B
:1076800088C128F189C129F18AC12AF18BC12BF166
:10769000F0EC03F09E0E256E030E266E8EECFBF0D2
:1076A00032EC0CF0070E0301A76F010E00016A6FA8
:1076B0009E0E6B6F030E6C6F020EEEEC0BF09E0EC7
:1076C0000101246F030E256F5B0E266FF30E276FEB
:1076D00084C128F185C129F186C12AF187C12BF126
:1076E000F0EC03F09E0E256E030E266E8EECFBF082
:1076F00032EC0CF0070E0301A76F010E00016A6F58
:107700009E0E6B6F030E6C6F030EEEEC0BF09E0E75
:107710000101246F030E256FB30E266FF30E276F42
:107720005BC128F15CC129F1F0EC03F09E0E256EDF
:10773000030E266E8EECFBF032EC0CF0070E03010C
:10774000A86F010E00016A6F9E0E6B6F030E6C6FC7
:10775000040EEEEC0BF0000E666F020E656F000E6D
:10776000686F070E676F3E0E696FEAECFAF0000E65
:107770000001666F020E656F000E686F0C0E676F7A
:107780003E0E696FEAECFAF0000E106EC0EC0BF0E2
:107790001004D8A40ED0E80E055C030E0658D8B02D
:1077A00008D0000E0D6E000E01015D6F000E03018A
:1077B0009E6F020E1018D8A49BD0E80E055C030E35
:1077C0000658D8B095D00D2A040E0D647BD0020E59
:1077D0000D6E78D0000E0001666F020E656F000E10
:1077E000686F070E676F3E0E696FEAECFAF0000EE5
:1077F0000001666F030E656F000E686F070E676FFE
:10780000200E696FEAECFAF0000E0001666F040EBC
:10781000656F000E686F070E676F200E696FEAECE8
:10782000FAF062D0000E0001666F020E656F000E66
:10783000686F070E676F200E696FEAECFAF0000EB2
:107840000001666F030E656F000E686F070E676FAD
:107850003E0E696FEAECFAF0000E0001666F040E4E
:10786000656F000E686F070E676F200E696FEAEC98
:10787000FAF03AD0000E0001666F020E656F000E3E
:10788000686F070E676F200E696FEAECFAF0000E62
:107890000001666F030E656F000E686F070E676F5D
:1078A000200E696FEAECFAF0000E0001666F040E1C
:1078B000656F000E686F070E676F3E0E696FEAEC2A
:1078C000FAF012D00D500101596F5A6B5A51000A4B
:1078D000D8A40AD05951020AD8B47CD7010AD8B426
:1078E000A1D7070AD8B4C6D7000E106EC0EC0BF0B3
:1078F000020E1018D8A411D0E90E055C030E06582C
:10790000D8A00BD0000E106EC0EC0BF0010E0D6471
:1079100004D00D500A0F01015D6F010E0D6408D0F7
:10792000000E0001716F030E706F22ECF9F003D0AE
:10793000010E8EEC05F001015D51D8B406D00A0E9F
:107940005D6103D03901A3AF23D73901A3AF02D0C2
:10795000000E0D6E0D50D8B440D39E0E0101246F61
:10796000030E256FCE0E266FFC0E276F5DC128F12A
:10797000296BF0EC03F09E0E256E030E266E8EEC46
:10798000FBF00DC065F00001666B000E686F070E1E
:10799000676F2A0E696FEAECFAF0110E01015A6F57
:1079A0003C0E596FCB0EE82EFED7592FFCD75A2F1D
:1079B000FAD7000E106EC0EC0BF0040E1018D8A40D
:1079C000C9D0E80E055C030E0658D8B0C3D00C0E23
:1079D00001015D19D8A445D088C186F089C187F01E
:1079E0008AC188F08BC189F0000E00018A6F000EF9
:1079F0008B6FF00E8C6F410E8D6FF2ECF5F0D8B0FE
:107A000030D088C176F089C177F08AC178F08BC117
:107A100079F0000E7A6F000E7B6FA00E7C6F400E27
:107A20007D6F99ECE0F076C088F177C089F178C07D
:107A30008AF179C08BF19E0E0101246F030E256F30
:107A4000100E266FFE0E276F88C128F189C129F11B
:107A50008AC12AF18BC12BF1F0EC03F0010E38EC56
:107A600006F00D0E01015D19D8A445D084C186F041
:107A700085C187F086C188F087C189F0000E0001BA
:107A80008A6F000E8B6FAA0E8C6F420E8D6FF2EC18
:107A9000F5F0D8B030D084C176F085C177F086C1DA
:107AA00078F087C179F0000E7A6F000E7B6FA00E20
:107AB0007C6F400E7D6F99ECE0F076C084F177C06A
:107AC00085F178C086F179C087F19E0E0101246F9F
:107AD000030E256F1D0E266FFE0E276F84C128F141
:107AE00085C129F186C12AF187C12BF1F0EC03F0A1
:107AF000010E38EC06F00E0E01015D19D8A426D057
:107B00005CBF06D05C5122E1140E5B5DD8B01ED084
:107B1000050E5B255B6F000E5C215C6F9E0E246F73
:107B2000030E256FDC0E266FFD0E276F5BC128F15B
:107B30005CC129F1F0EC03F05B515C11D8A403D0D7
:107B4000200E0301A56F020E38EC06F0000E106E39
:107B5000C0EC0BF0080E1018D8A4C8D0E80E055CD5
:107B6000030E0658D8B0C2D00C0E01015D19D8A47E
:107B700045D0000E0001866F000E876F700E886F73
:107B8000410E896F88C18AF089C18BF08AC18CF05F
:107B90008BC18DF0F2ECF5F0D8B030D088C176F022
:107BA00089C177F08AC178F08BC179F0000E7A6FC5
:107BB000000E7B6FA00E7C6FC00E7D6F99ECE0F025
:107BC00076C088F177C089F178C08AF179C08BF1ED
:107BD0009E0E0101246F030E256F100E266FFE0E00
:107BE000276F88C128F189C129F18AC12AF18BC187
:107BF0002BF1F0EC03F0010E38EC06F00D0E010154
:107C00005D19D8A445D0000E0001866F000E876F65
:107C1000F00E886F410E896F84C18AF085C18BF0A8
:107C200086C18CF087C18DF0F2ECF5F0D8B030D081
:107C300084C176F085C177F086C178F087C179F08C
:107C4000000E7A6F000E7B6FA00E7C6FC00E7D6FF2
:107C500099ECE0F076C084F177C085F178C086F1C8
:107C600079C087F19E0E0101246F030E256F1D0E52
:107C7000266FFE0E276F84C128F185C129F186C1C8
:107C80002AF187C12BF1F0EC03F0010E38EC06F07D
:107C90000E0E01015D19D8B45CBF24D05C5104E123
:107CA000050E5B5DD8A01ED0FB0E5B255B6FFF0E43
:107CB0005C215C6F9E0E246F030E256FDC0E266F19
:107CC000FD0E276F5BC128F15CC129F1F0EC03F0D8
:107CD0005B515C11D8A403D0200E0301A56F020EE6
:107CE00038EC06F0000E106EC0EC0BF0100E101801
:107CF000D8A4F6D0E90E055C030E0658D8A0F0D043
:107D00000A0E01015D65ECD0C0EC0BF0000E106EA8
:107D100001015D510A0F5D6F160E5D19D8A432D0B6
:107D200088C1E2F189C1E3F18AC1E4F18BC1E5F1D7
:107D30009E0E246F030E256F8F0E266FE10E276FA8
:107D4000E2C128F1E3C129F1E4C12AF1E5C12BF137
:107D5000000E2D6F500E2C6FF0EC03F0000E2C6E09
:107D6000500E2B6EE2C12DF0E3C12EF0E4C12FF0D6
:107D7000E5C130F046EC05F09E0E256E030E266E32
:107D80008EECFBF0170E01015D19D8A432D084C12E
:107D9000E6F185C1E7F186C1E8F187C1E9F19E0E00
:107DA000246F030E256F9B0E266FE00E276FE6C132
:107DB00028F1E7C129F1E8C12AF1E9C12BF1000E50
:107DC0002D6F540E2C6FF0EC03F0000E2C6E540E41
:107DD0002B6EE6C12DF0E7C12EF0E8C12FF0E9C10E
:107DE00030F046EC05F09E0E256E030E266E8EECEE
:107DF000FBF0180E01015D19D8A449D05BC125F034
:107E00005CC126F0000E26BEFF0E276E286E010E06
:107E100094ECEFF025C033F026C034F027C035F0E5
:107E200028C036F0DBEC09F033C0E9F234C0EAF2E6
:107E300035C0EBF236C0ECF29E0E0101246F030E4A
:107E4000256F2E0E266FE10E276FE9C228F1EAC2D8
:107E500029F1EBC22AF1ECC22BF1000E2D6F580E66
:107E60002C6FF0EC03F09E0E256E030E266E8EEC4A
:107E7000FBF0000E2C6E580E2B6EE9C22DF0EAC2FC
:107E80002EF0EBC22FF0ECC230F046EC05F0000E05
:107E9000106EC0EC0BF0080E00016B6F600E6C6F83
:107EA000FD0E6D6F6C516D11D8A4000E6E6F0D50EC
:107EB0003AEC0BF0030E8EEC05F0080E00016B6F30
:107EC000B20E6C6FEE0E6D6F6C516D11D8A4000E7A
:107ED0006E6F0D503AEC0BF0000E106EC0EC0BF014
:107EE000140E01015D650CD0000E106EC0EC0BF09D
:107EF000EC0E2B6EFC0E2C6E78EC06F0D7EFBAF081
:107F0000AAEC07F00A0E0D644CD0000E0001666F5B
:107F1000030E656F000E686F0C0E676F200E696FA1
:107F2000EAECFAF0000E0001666F040E656F000EB9
:107F3000686F0C0E676F200E696FEAECFAF0110E95
:107F400001015A6F3C0E596FCB0EE82EFED7592F08
:107F5000FCD75A2FFAD7000E0001666F030E656F2B
:107F6000000E686F0C0E676F200E696FEAECFAF076
:107F7000000E0001666F040E656F000E686F0C0E38
:107F8000676F3E0E696FEAECFAF0110E01015A6F4D
:107F90003C0E596FCB0EE82EFED7592FFCD75A2F27
:107FA000FAD7010E0D640FD001015D51D8B40BD08A
:107FB000140E5D6108D0000E0001716F030E706F2A
:107FC00022ECF9F003D0010E8EEC05F03901A3BFCD
:107FD00004D0020E01015D61F0D4030E0E6E3EEC82
:107FE000FBF01200020E0E6EEEC188F1EFC189F1B6
:107FF000F0C18AF1F1C18BF1EDC284F1EEC285F1DD
:10800000EFC286F1F0C287F1FFC15BF1010EDDEC3A
:10801000FBF0090E01015A6F1E0E596FE40EE82E97
:10802000FED7592FFCD75A2FFAD700F0010E0101C5
:108030005C6F020E0D6E6E0E2B6EED0E2C6E78ECDC
:1080400006F0010E00016B6FD00E6C6FF70E6D6FB6
:108050006C516D11D8A4000E6E6F010E3AEC0BF04E
:108060009E0E0101246F030E256F150E266FF10E73
:10807000276F88C128F189C129F18AC12AF18BC1F2
:108080002BF1F0EC03F09E0E256E030E266E8EECA7
:10809000FBF032EC0CF0070E0301A76F010E00019C
:1080A0006A6F9E0E6B6F030E6C6F020EEEEC0BF0A0
:1080B0009E0E0101246F030E256F710E266FF10EC7
:1080C000276F84C128F185C129F186C12AF187C1B2
:1080D0002BF1F0EC03F09E0E256E030E266E8EEC57
:1080E000FBF032EC0CF0010E00016A6F9E0E6B6F1C
:1080F000030E6C6F030EEEEC0BF09E0E0101246F6D
:10810000030E256FC90E266FF30E276F5BC128F192
:10811000296BF0EC03F09E0E256E030E266E8EEC9E
:10812000FBF032EC0CF0010E00016A6F9E0E6B6FDB
:10813000030E6C6F040EEEEC0BF0000E666F020E79
:10814000656F000E686F0C0E676F3E0E696FEAEC8C
:10815000FAF0010E8EEC05F0000E106EC0EC0BF084
:108160001004D8A405D0000E0D6E000E01015C6F46
:10817000020E1018D8A49BD0E80E055C030E06581A
:10818000D8B095D00D2A040E0D647BD0020E0D6E72
:1081900078D0000E0001666F020E656F000E686FEA
:1081A000070E676F3E0E696FEAECFAF0000E0001F1
:1081B000666F030E656F000E686F070E676F200E07
:1081C000696FEAECFAF0000E0001666F040E656F4D
:1081D000000E686F070E676F200E696FEAECFAF009
:1081E00062D0000E0001666F020E656F000E686FB0
:1081F000070E676F200E696FEAECFAF0000E0001BF
:10820000666F030E656F000E686F070E676F3E0E98
:10821000696FEAECFAF0000E0001666F040E656FFC
:10822000000E686F070E676F200E696FEAECFAF0B8
:108230003AD0000E0001666F020E656F000E686F87
:10824000070E676F200E696FEAECFAF0000E00016E
:10825000666F030E656F000E686F070E676F200E66
:10826000696FEAECFAF0000E0001666F040E656FAC
:10827000000E686F070E676F3E0E696FEAECFAF04A
:1082800012D00D500101596F5A6B5A51000AD8A4EF
:108290000AD05951020AD8B47CD7010AD8B4A1D760
:1082A000070AD8B4C6D7000E106EC0EC0BF0020E51
:1082B0001018D8A411D0E90E055C030E0658D8A0FA
:1082C0000BD0010E0D6408D00D500A0F01015C6F38
:1082D000000E106EC0EC0BF0010E0D6408D0000E05
:1082E0000001716F020E706F22ECF9F003D0010EE5
:1082F0008EEC05F001015C51D8B406D00A0E5C6129
:1083000003D03901A3AF2CD73901A3AF02D0000E9F
:108310000D6E0D50D8B45ED39E0E0101246F030E76
:10832000256FCE0E266FFC0E276F5CC128F1296BDE
:10833000F0EC03F09E0E256E030E266E8EECFBF025
:10834000000E0001666F020E656F000E686F0C0E66
:10835000676F200E696FEAECFAF0000E0001666F9D
:10836000030E656F000E686F0C0E676F3E0E696F2F
:10837000EAECFAF0C0EC0BF01CD0EEC188F1EFC1D2
:1083800089F1F0C18AF1F1C18BF126D0EDC284F1FF
:10839000EEC285F1EFC286F1F0C287F11DD0FFC1B8
:1083A0005BF11AD02E0E2B6EFC0E2C6E78EC06F0C4
:1083B00013D001015C51596F5A6B5A51000AD8A46D
:1083C000F1D759510C0AD8B4D8D7010AD8B4DED79E
:1083D000030AD8B4E4D7E6D70DC065F00001666B98
:1083E000000E686F070E676F2A0E696FEAECFAF0ED
:1083F000C0EC0BF0000E106E040E1018D8A40ED1B5
:10840000E80E055C030E0658D8B008D12B0E3D01CE
:10841000EA6F0C0E01015C19D8A44ED088C176F029
:1084200089C177F08AC178F08BC179F0000E000124
:108430007A6F000E7B6F000E7C6F3F0E7D6F99ECA4
:10844000E0F076C088F177C089F178C08AF179C010
:108450008BF1000E866F000E876F000E886F400E46
:10846000896F88C18AF089C18BF08AC18CF08BC179
:108470008DF0F2ECF5F0D8B009D0000E0101886F54
:10848000000E896F000E8A6F000E8B6F9E0E010129
:10849000246F030E256F7C0E266FFD0E276F88C19B
:1084A00028F189C129F18AC12AF18BC12BF1F0ECA5
:1084B00003F0010E38EC06F00D0E01015C19D8A492
:1084C0004ED084C176F085C177F086C178F087C13F
:1084D00079F0000E00017A6F000E7B6F000E7C6F4A
:1084E0003F0E7D6F99ECE0F076C084F177C085F1A6
:1084F00078C086F179C087F1000E866F000E876F15
:10850000A00E886F400E896F84C18AF085C18BF000
:1085100086C18CF087C18DF0F2ECF5F0D8B009D0AF
:10852000000E0101846F000E856F000E866F3F0EF6
:10853000876F9E0E0101246F030E256F6E0E266F4E
:10854000FD0E276F84C128F185C129F186C12AF16A
:1085500087C12BF1F0EC03F0020E38EC06F00E0EA2
:1085600001015C19D8A417D05B295B6F480E5B65CD
:1085700002D0410E5B6F9E0E246F030E256F0B0E13
:10858000266FFF0E276F5BC128F1296BF0EC03F01B
:10859000020E38EC06F0000E0001666F030E656FE8
:1085A000000E686F0C0E676F200E696FEAECFAF030
:1085B000000E0001666F040E656F000E686F0C0EF2
:1085C000676F200E696FEAECFAF0110E01015A6F25
:1085D0003C0E596FCB0EE82EFED7592FFCD75A2FE1
:1085E000FAD7000E0001666F040E656F000E686F0B
:1085F0000C0E676F3E0E696FEAECFAF0110E010186
:108600005A6F3C0E596FCB0EE82EFED7592FFCD770
:108610005A2FFAD7000E106EC0EC0BF0080E10188F
:10862000D8A4E8D0E80E055C030E0658D8B0E2D016
:108630002D0E3D01EA6F0C0E01015C19D8A43BD050
:1086400088C176F089C177F08AC178F08BC179F062
:10865000000E00017A6F000E7B6F000E7C6FBF0E64
:108660007D6F99ECE0F076C088F177C089F178C031
:108670008AF179C08BF101018BAF08D0000E886FB1
:10868000000E896F000E8A6F400E8B6F9E0E246F56
:10869000030E256F7C0E266FFD0E276F88C128F113
:1086A00089C129F18AC12AF18BC12BF1F0EC03F0C9
:1086B000010E38EC06F00D0E01015C19D8A43BD078
:1086C00084C176F085C177F086C178F087C179F0F2
:1086D000000E00017A6F000E7B6F000E7C6FBF0EE4
:1086E0007D6F99ECE0F076C084F177C085F178C0B9
:1086F00086F179C087F1010187AF08D0000E846F41
:10870000000E856FA00E866F400E876F9E0E246F41
:10871000030E256F6E0E266FFD0E276F84C128F1A4
:1087200085C129F186C12AF187C12BF1F0EC03F054
:10873000020E38EC06F00E0E01015C19D8A417D019
:108740005B055B6F410E5B6102D0480E5B6F9E0E56
:10875000246F030E256F0B0E266FFF0E276F5BC174
:1087600028F1296BF0EC03F0020E38EC06F0000E55
:108770000001666F030E656F000E686F0C0E676F69
:10878000200E696FEAECFAF0000E0001666F040E2D
:10879000656F000E686F0C0E676F200E696FEAEC54
:1087A000FAF0110E01015A6F3C0E596FCB0EE82EF4
:1087B000FED7592FFCD75A2FFAD7000E0001666F4B
:1087C000040E656F000E686F0C0E676F3E0E696FCA
:1087D000EAECFAF0110E01015A6F3C0E596FCB0E04
:1087E000E82EFED7592FFCD75A2FFAD7000E106E5D
:1087F000C0EC0BF0100E1018D8A4C5D0E90E055C23
:10880000030E0658D8A0BFD00A0E01015C65BBD08C
:108810000D500A0F5C6F1E0E2B6EFC0E2C6E78EC4A
:1088200006F001015C510A0F5C6F000E106EC0EC87
:108830000BF0160E01015C19D8A432D088C1EEF1FC
:1088400089C1EFF18AC1F0F18BC1F1F19E0E246F65
:10885000030E256F670E266FE30E276FEEC128F11A
:10886000EFC129F1F0C12AF1F1C12BF1000E2D6FFA
:108870005C0E2C6FF0EC03F0000E2C6E5C0E2B6E79
:10888000EEC12DF0EFC12EF0F0C12FF0F1C130F0AC
:1088900046EC05F09E0E256E030E266E8EECFBF068
:1088A000170E01015C19D8A432D084C1EDF285C144
:1088B000EEF286C1EFF287C1F0F29E0E246F030E36
:1088C000256F370E266FE00E276FEDC228F1EEC23E
:1088D00029F1EFC22AF1F0C22BF1000E2D6F600ECC
:1088E0002C6FF0EC03F0000E2C6E600E2B6EEDC2C0
:1088F0002DF0EEC22EF0EFC22FF0F0C230F046ECB9
:1089000005F09E0E256E030E266E8EECFBF0180E03
:1089100001015C19D8A421D05BC1FFF19E0E246F28
:10892000030E256FDC0E266FE20E276FFFC128F1C4
:10893000296B000E2B6F910E2A6FF0EC03F09E0E48
:10894000256E030E266E8EECFBF0000E266E910E49
:10895000256E5BC127F0EBEC02F0080E00016B6F97
:10896000600E6C6FFD0E6D6F6C516D11D8A4000E12
:108970006E6F0D503AEC0BF0030E8EEC05F0C0EC70
:108980000BF0000E106E140E01015C6506D0000E97
:10899000106EC0EC0BF0F2EFBFF0AAEC07F0010E86
:1089A0000D640ED001015C51D8B40AD00A0E5C618E
:1089B00007D00EC070F00001716B22ECF9F003D00B
:1089C000010E8EEC05F03901A3BF04D0020E0101A7
:1089D0005C6112D5020E0E6E3EECFBF01200000E32
:1089E000D76F000ED66FB8C0E6F0B9C0E7F0BAC0D6
:1089F000E8F0BBC0E9F0E9AF16D0000ED76F010E6A
:108A0000D66FE6C033F0E7C034F0E8C035F0E9C017
:108A100036F0DBEC09F033C0E6F034C0E7F035C0E7
:108A2000E8F036C0E9F0000E0001EF6F000EEE6FC7
:108A30009CC1DBF09DC1DCF0D651D711D8A402D087
:108A400003A413D0D651D711D8A404D0000EC36FFD
:108A50002B0E03D0000EC36F2D0EC26FC2C048F4A0
:108A6000EE4BEF2BDB07D8A0DC07E6C025F0E7C014
:108A700026F0E8C027F0E9C028F02AECF7F025043A
:108A80002610D8A443D0BF0E0001BD6FFF0EBE6FED
:108A9000BC51BF6FC06BBD51BF27BE51C023C05179
:108AA00011E11A0EBF5DD8B00DD0480EEE25296E2B
:108AB000040EEF212A6EE30E2B6EFF0E2C6E00ECDF
:108AC00002F00CD0480EEE25296E040EEF212A6E1E
:108AD000EB0E2B6EFF0E2C6E00EC02F00001FD0E73
:108AE000DB27FF0EDC23B6C035F0B7C036F0480EEA
:108AF000376E040E386EDBC039F0DCC03AF0C6ECDD
:108B0000FCF035C0B6F036C0B7F01200E6C025F074
:108B1000E7C026F0E8C027F0E9C028F02AECF7F01B
:108B200025502610D8A42CD0BF0E0001BD6FFF0E1B
:108B3000BE6FBC51BF6FC06BBD51BF27BE51C023BC
:108B4000C05111E11A0EBF5DD8B00DD0480EEE2510
:108B5000296E040EEF212A6EE70E2B6EFF0E2C6E8F
:108B600000EC02F0BBD7480EEE25296E040EEF2173
:108B70002A6EEF0E2B6EFF0E2C6E00EC02F0AED7BD
:108B8000000E0001F06F000EF16F800EF26F3F0ECD
:108B9000F36F000EED6F000EEC6FE6C025F0E7C03E
:108BA00026F0E8C027F0E9C028F0000E296E000E7C
:108BB0002A6E000E2B6E000E2C6E56ECFDF0D8A027
:108BC0001DD074D0F0C033F0F1C034F0F2C035F0F5
:108BD000F3C036F0000E376E000E386E200E396E80
:108BE000410E3A6EB7ECDBF033C0F0F034C0F1F078
:108BF00035C0F2F036C0F3F0EC4BED2BE6C086F05A
:108C0000E7C087F0E8C088F0E9C089F0000E376E51
:108C1000000E386E200E396E410E3A6EF0C033F001
:108C2000F1C034F0F2C035F0F3C036F0B7ECDBF051
:108C300033C08AF034C08BF035C08CF036C08DF074
:108C4000F2ECF5F0D8A01ED0BDD7F0C086F0F1C090
:108C500087F0F2C088F0F3C089F0000E8A6F000E32
:108C60008B6F200E8C6F410E8D6F75ECE3F086C01C
:108C7000F0F087C0F1F088C0F2F089C0F3F0EC07A3
:108C8000D8A0ED07E6C086F0E7C087F0E8C088F01E
:108C9000E9C089F0F0C08AF0F1C08BF0F2C08CF02E
:108CA000F3C08DF0F2ECF5F0D8A0CFD7BCC02BF01C
:108CB0002C6AE4EC07F02B500001DD6FDDC0DAF028
:108CC000670EDD19D8A419D001500210D8A404D021
:108CD000000E026E010E016E02BE05D0025008E1C8
:108CE0000104D8B005D0000ED96F060ED86F08D099
:108CF00001C0D8F002C0D9F003D002AEF9D7F3D743
:108D0000670EDD19D8A422D0EDAF06D0FC0EEC5DC5
:108D1000FF0EED59D8A018D0FF0EBD6FFF0EBE6F2D
:108D2000D8C0BFF0D9C0C0F0BD51BF27BE51C023CD
:108D3000EC51BF5DC051800AC16FED51800AC1592D
:108D4000D8A002D0660E01D0650EDA6FD8C0CEF082
:108D5000D9C0CFF0670EDD19D8A405D0660EDA1998
:108D6000D8B4EDAF02D0CE4BCF2B660EDA19D8A413
:108D700016D0EDAF0CD0000EF06F000EF16F800E2C
:108D8000F26F3F0EF36F000EED6F000EEC6F670E8B
:108D9000DD19D8B404D0EC51CE27ED51CF23000E0D
:108DA000EB6F000EEA6FE6C0DEF0E7C0DFF0E8C070
:108DB000E0F0E9C0E1F0F0C0D0F0F1C0D1F0F2C0D5
:108DC000D2F0F3C0D3F07AD0DEC086F0DFC087F0F7
:108DD000E0C088F0E1C089F0F0C08AF0F1C08BF00B
:108DE000F2C08CF0F3C08DF075ECE3F086C09FF01C
:108DF00087C0A0F088C0A1F089C0A2F0BBECEAF067
:108E00009FC0E2F0A0C0E3F0A1C0E4F0A2C0E5F092
:108E1000E2C0ACF0E3C0ADF0E4C0AEF0E5C0AFF04E
:108E200081ECF9F0ACC0D4F0ADC0D5F0DEC086F076
:108E3000DFC087F0E0C088F0E1C089F0F0C037F013
:108E4000F1C038F0F2C039F0F3C03AF0E2C033F0CC
:108E5000E3C034F0E4C035F0E5C036F0B7ECDBF049
:108E600033C08AF034C08BF035C08CF036C08DF042
:108E70006AEC05F086C0DEF087C0DFF088C0E0F065
:108E800089C0E1F0F0C086F0F1C087F0F2C088F050
:108E9000F3C089F0000E8A6F000E8B6F200E8C6F6E
:108EA000410E8D6F75ECE3F086C0F0F087C0F1F0F5
:108EB00088C0F2F089C0F3F0EA4BEB2BCE51EA5DAB
:108EC000EB51800ABD6FCF51800ABD59D8A07CD725
:108ED000F0C033F0F1C034F0F2C035F0F3C036F03A
:108EE000000E376E000E386EA00E396E400E3A6ED0
:108EF000B7ECDBF033C0E2F034C0E3F035C0E4F0AF
:108F000036C0E5F0DEC086F0DFC087F0E0C088F054
:108F1000E1C089F0E2C08AF0E3C08BF0E4C08CF0DD
:108F2000E5C08DF0F2ECF5F0D8A017D0DEC025F04A
:108F3000DFC026F0E0C027F0E1C028F0E2C029F051
:108F4000E3C02AF0E4C02BF0E5C02CF056ECFDF0B5
:108F5000D8A00BD00001D4B108D0000EE26F000EF3
:108F6000E36F000EE46F000EE56FE6C076F0E7C039
:108F700077F0E8C078F0E9C079F0E2C07AF0E3C0B9
:108F80007BF0E4C07CF0E5C07DF099ECE0F076C0C9
:108F9000DEF077C0DFF078C0E0F079C0E1F0DEC04D
:108FA00086F0DFC087F0E0C088F0E1C089F0000EF5
:108FB000376E000E386E200E396E410E3A6ED0C0FC
:108FC00033F0D1C034F0D2C035F0D3C036F0B7ECB6
:108FD000DBF033C08AF034C08BF035C08CF036C083
:108FE0008DF0F2ECF5F0D8A022D0EC4BED2BD0C0F8
:108FF00033F0D1C034F0D2C035F0D3C036F0000E1B
:10900000376E000E386E200E396E410E3A6EB7EC98
:10901000DBF033C0D0F034C0D1F035C0D2F036C070
:10902000D3F0660EDA19D8A402D0CE4BCF2BD0C025
:10903000F0F0D1C0F1F0D2C0F2F0D3C0F3F0650E81
:10904000DA19D8B405D0ECC0CCF0EDC0CDF004D026
:10905000000ECD6F000ECC6F000ECB6F000ECA6FEE
:10906000000EC96F000EC86F000EEB6F000EEA6FA6
:10907000C4D0DEC086F0DFC087F0E0C088F0E1C079
:1090800089F0F0C08AF0F1C08BF0F2C08CF0F3C030
:109090008DF075ECE3F086C09FF087C0A0F088C02B
:1090A000A1F089C0A2F0BBECEAF09FC0E2F0A0C042
:1090B000E3F0A1C0E4F0A2C0E5F0E2C0ACF0E3C090
:1090C000ADF0E4C0AEF0E5C0AFF081ECF9F0ACC0BB
:1090D000D4F0ADC0D5F003B80CD0D451D511D8A47C
:1090E00008D0670EDD19D8B4CDAF03D0C84BC92B5B
:1090F00039D0CA51CB11D8B4CDAF22D0480EEE250D
:10910000D96E040EEF21DA6E2E0EDF6EEE4BEF2BD2
:10911000DB07D8A0DC07000ECB6F010ECA6F10D0A2
:10912000480EEE25D96E040EEF21DA6E300EDF6E9A
:10913000EE4BEF2BDB07D8A0DC07C807D8A0C90788
:10914000C851C911D8A4ECD7480EEE25D96E040E2B
:10915000EF21DA6ED451300FDF6EEE4BEF2BDB07D1
:10916000D8A0DC07DEC086F0DFC087F0E0C088F062
:10917000E1C089F0F0C037F0F1C038F0F2C039F04A
:10918000F3C03AF0E2C033F0E3C034F0E4C035F0AD
:10919000E5C036F0B7ECDBF033C08AF034C08BF0BA
:1091A00035C08CF036C08DF06AEC05F086C0DEF07C
:1091B00087C0DFF088C0E0F089C0E1F0F0C086F041
:1091C000F1C087F0F2C088F0F3C089F0000E8A6F1A
:1091D000000E8B6F200E8C6F410E8D6F75ECE3F0DF
:1091E00086C0F0F087C0F1F088C0F2F089C0F3F0DB
:1091F000CC07D8A0CD07EA4BEB2BCE51EA5DEB5163
:10920000800ABD6FCF51800ABD59D8B008D0EFBFDA
:1092100030D7EF5104E14B0EEE5DD8A02AD7CA51EA
:10922000CB11D8B403A80AD0480EEE25D96E040E8F
:10923000EF21DA6E2E0EDF6EEE4BEF2B480EEE2591
:10924000D96E040EEF21DA6E000EDF6E650EDA19AC
:10925000D8A449D4000EEB6F4F0EEA6F480EEA25F2
:10926000D96E040EEB21DA6E000EDF6E000ED76FA2
:10927000000ED66FEDAF08D0000ED76F010ED66F7F
:10928000EC6DED1FD8B0ED2B000ED96F020ED86F2C
:109290002BD0EA07D8A0EB07480EEA25D96E040EBA
:1092A000EB21DA6EECC025F0EDC026F0000E286E42
:1092B0000A0E276ECBEC00F02550300FDF6EECC0AD
:1092C00025F0EDC026F0000E286E0A0E276EDDECAC
:1092D000FDF025C0ECF026C0EDF00001D807D8A0C5
:1092E000D907DB07D8A0DC07EC51ED11D8A4D1D702
:1092F000D9BF05D0D951CDE1D805D8B0CAD7EA0732
:10930000D8A0EB07D651D711D8A404D0000EC56F52
:109310002B0E03D0000EC56F2D0EC46F480EEA252C
:10932000D96E040EEB21DA6E600013F3DFFFDB076A
:10933000D8A0DC07EA07D8A0EB07BF0EBD6FFF0E71
:10934000BE6FBC51BF6FC06BBD51BF27BE51C023A4
:10935000C05104E11A0EBF5DD8A004D0000EC76F43
:10936000650E03D0000EC76F450EC66F480EEA2586
:10937000D96E040EEB21DA6E60001BF3DFFFDB0712
:10938000D8A0DC07480EEE25296E040EEF212A6EC8
:10939000480EEA252B6E040EEB212C6E00EC02F039
:1093A00073EFC5F0F651D96EDA6A6F007BFFF6FFF6
:1093B0006F0077FFF7FF000EF86E0800F550250AE2
:1093C000D8A465EFCEF0F651D96EDA6ADE2A000E27
:1093D000DD22000E01019D6F000E9C6F9CC103F009
:1093E0009DC104F001680268000E0B6F000E14D0DE
:1093F0000380F651D96EDA6ADE2A000EDD2233D000
:109400000382F7D70384F5D70386F3D70388F1D710
:10941000000E01010B6F010E0A6F25D00001F651FD
:10942000D96EDA6A6F007BFFF6FF6F0077FFF7FFF8
:10943000000EF86E0800F550F96FFA6BFA51000A49
:10944000D8A4E6D7F951200AD8B4DED7030AD8B495
:10945000DDD7080AD8B4D6D7060AD8B4C9D71D0AAA
:10946000D8B4CED7D5D701010A510B11D8B4D6D76D
:1094700003B003920001F651D96EDA6A6F007BFFE8
:10948000F6FF6F0077FFF7FF000EF86E0800F5504B
:109490002A0AD8A42BD0F651D96EDA6ADE2A000E39
:1094A000DD226000DFF3D9FF6000E3F3DAFF6F0035
:1094B0007CFFF9F0020EDE266F007CFFFAF0000E52
:1094C000DD226000E7F3D9FF6000EBF3DAFF6F0005
:1094D00078FF9CF16F0074FF9DF101019DAF3AD0C0
:1094E00003809C6D9D1FD8B09D2B34D0F651D96E52
:1094F000DA6A6F0078FF2CF06F0074FF2DF034EC07
:10950000F0F02CC09CF12DC09DF106D0F651D96E23
:10951000DA6ADE2A000EDD22D00E0001F96FFF0E9E
:10952000FA6FF651D96EDA6A6F007BFFF6FF6F00B3
:1095300077FFF7FF000EF86E0800F550FB6FFC6B2D
:10954000F951FB27FA51FC23FC5104E10A0EFB5DA3
:10955000D8A0DCD70001F651D96EDA6A6F007BFF24
:10956000F6FF6F0077FFF7FF000EF86E0800F5506A
:109570002E0AD8A471D0000E026E000E016EF651B4
:10958000D96EDA6ADE2A000EDD22F651D96EDA6A69
:109590006F007BFFF6FF6F0077FFF7FF000EF86E9E
:1095A0000800F5502A0AD8A423D0F651D96EDA6AF9
:1095B000DE2A000EDD226000DFF3D9FF6000E3F356
:1095C000DAFF6F007CFFF9F0020EDE266F007CFFF1
:1095D000FAF0000EDD226000E7F3D9FF6000EBF344
:1095E000DAFF6F0078FF01F06F0074FF02F034D0F3
:1095F000F651D96EDA6A6F0078FF2CF06F0074FFB5
:109600002DF034ECF0F02CC001F02DC002F006D0AB
:10961000F651D96EDA6ADE2A000EDD22D00E000184
:10962000F96FFF0EFA6FF651D96EDA6A6F007BFFA1
:10963000F6FF6F0077FFF7FF000EF86E0800F55099
:10964000FB6FFC6BF951FB27FA51FC23FC5104E141
:109650000A0EFB5DD8A0DCD7F651D96EDA6A6F002E
:109660007BFFF6FF6F0077FFF7FF000EF86E080034
:10967000F5502B6E2C6AE4EC07F02B5001011A6FA9
:109680001A51D8B441D00001F651D96EDA6A6F0090
:1096900078FFF9F06F0074FFFAF0010EF927000E61
:1096A000FA236000E7F3F6FF6000EBF3F7FF000E2C
:1096B000F86E0800F5502B6E2C6AE4EC07F02B5086
:1096C00001011B6F1B51D8B41FD00001F651D96E98
:1096D000DA6A6F0078FFF9F06F0074FFFAF0020E9B
:1096E000F927000EFA236000E7F3F6FF6000EBF3C2
:1096F000F7FF000EF86E0800F5502B6E2C6AE4ECB4
:1097000007F02B5001011C6F0001F651D96EDA6A87
:109710006F007BFFF6FF6F0077FFF7FF000EF86E1C
:109720000800F550630AD8A42CD0F651D96EDA6A35
:10973000DE2A000EDD226000DFF3D9FF6000E3F3D4
:10974000DAFF6F007CFFF9F0020EDE266F007CFF6F
:10975000FAF0000EDD226000E7F3D9FF6000EBF3C2
:10976000DAFFDF5001011D6FF4C02EF0F5C02FF0BD
:109770001DC130F02CECFCF02EC0F4F02FC0F5F041
:109780001200F651D96EDA6A6F007BFFF6FF6F00A8
:1097900077FFF7FF000EF86E0800F550640AD8B4A2
:1097A00010D0F651D96EDA6A6F007BFFF6FF6F00BA
:1097B00077FFF7FF000EF86E0800F550690AD8A48D
:1097C00047D0F651D96EDA6ADE2A000EDD2260003B
:1097D000DFF3D9FF6000E3F3DAFF6F007CFFF9F0FD
:1097E000020EDE266F007CFFFAF0000EDD22600024
:1097F000E7F3D9FF6000EBF3DAFF6F0078FF00F1C9
:109800006F0074FF01F10101000E01BFFF0E026F36
:10981000036F046F056F066F076FF4C0BAF0F5C0F1
:10982000BBF000C1BCF001C1BDF002C1BEF003C17C
:10983000BFF004C1C0F005C1C1F006C1C2F007C14C
:10984000C3F0B9ECE4F0BAC0F4F0BBC0F5F012001C
:10985000660E01011A19D8A44DD00001F651D96E37
:10986000DA6A6F007BFFF6FF6F0077FFF7FF000EED
:10987000F86E08006F00D4FF1DF1F651D96EDA6A58
:10988000DE2A000EDD226000DFF3D9FF6000E3F383
:10989000DAFF6F007CFFF9F0040EDE266F007CFF1C
:1098A000FAF0000EDD226000E7F3D9FF6000EBF371
:1098B000DAFF6F0078FF16F16F0078FF17F16F0085
:1098C00078FF18F16F0078FF19F1F4C0B6F0F5C019
:1098D000B7F016C1B8F017C1B9F018C1BAF019C184
:1098E000BBF01DC1BCF0EFECC4F0B6C0F4F0B7C0E3
:1098F000F5F012001A0E256E010E266EFB0E276E75
:10990000FF0E286E000E2A6E020E296E94ECF2F005
:1099100025502610D8A45FD00001F651D96EDA6A1E
:109920006F0078FFF9F06F0074FFFAF0010EF9276D
:10993000000EFA236000E7F3F6FF6000EBF3F7FF99
:10994000000EF86E08006F00D4FF1DF1BF0EF96F16
:10995000FF0EFA6FF651D96EDA6A6F007BFFF6FFE1
:109960006F0077FFF7FF000EF86E0800F550FB6FF1
:10997000FC6BF951FB27FA51FC23FC5102E11A0E52
:10998000FB5D6000DFF3D9FF6000E3F3DAFF6F00F7
:109990007CFFF9F0040EDE266F007CFFFAF0000E6B
:1099A000DD226000E7F3D9FF6000EBF3DAFF6F0020
:1099B00078FF16F16F0078FF17F16F0078FF18F14C
:1099C0006F0078FF19F1F651D96EDA6A020EDE26C1
:1099D000000EDD227AD70001F651D96EDA6A6F00E7
:1099E0007BFFF6FF6F0077FFF7FF000EF86E0800B1
:1099F000F550730AD8B417D0F651D96EDA6A6F00F1
:109A000078FF25F06F0074FF26F0F30E276EFF0E2F
:109A1000286E000E2A6E030E296E94ECF2F025508B
:109A20002610D8A44FD00001F651D96EDA6A6F0023
:109A30007BFFF6FF6F0077FFF7FF000EF86E080060
:109A4000F550730AD8B405D0000E01010D6F030E56
:109A500004D0000E01010D6F010E0C6F0001F651D4
:109A6000D96EDA6A01010C51DE260D51DD2260004B
:109A7000DFF3D9FF6000E3F3DAFF6F007CFFF9F05A
:109A8000020EDE266F007CFFFAF0000EDD22600081
:109A9000E7F3D9FF6000EBF3DAFF6F0078FF08F11E
:109AA0006F0074FF09F1F4C02EF0F5C02FF008C16B
:109AB00030F009C131F002ECEDF02EC0F4F02FC00F
:109AC000F5F012000001F651D96EDA6A6F007BFFE3
:109AD000F6FF6F0077FFF7FF000EF86E0800F550F5
:109AE000750AD8A448D0F651D96EDA6ADE2A000E7B
:109AF000DD226000DFF3D9FF6000E3F3DAFF6F00DF
:109B00007CFFF9F0020EDE266F007CFFFAF0000EFB
:109B1000DD226000E7F3D9FF6000EBF3DAFF6F00AE
:109B200078FFFBF06F0074FFFCF0FBC00EF1FCC08F
:109B30000FF10101106B116B126B136B146B156B32
:109B4000F4C060F0F5C061F00EC162F00FC163F0C7
:109B500010C164F011C165F012C166F013C167F065
:109B600014C168F015C169F0E1ECE9F060C0F4F0EF
:109B700061C0F5F01200F651D96EDA6A6F007BFF12
:109B8000F6FF6F0077FFF7FF000EF86E0800F55044
:109B9000780AD8B410D0F651D96EDA6A6F007BFF1C
:109BA000F6FF6F0077FFF7FF000EF86E0800F55024
:109BB000580AD8A459D0F651D96EDA6A6F007BFFE3
:109BC000F6FF6F0077FFF7FF000EF86E08006F00DA
:109BD000D4FF1DF1F651D96EDA6ADE2A000EDD22BD
:109BE0006000DFF3D9FF6000E3F3DAFF6F007CFF72
:109BF000F9F0020EDE266F007CFFFAF0000EDD2287
:109C00006000E7F3D9FF6000EBF3DAFF6F0078FF45
:109C1000FBF06F0074FFFCF0FBC00EF1FCC00FF115
:109C20000101106B116B126B136B146B156BF4C08D
:109C300060F0F5C061F00EC162F00FC163F010C1B9
:109C400064F011C165F012C166F013C167F014C170
:109C500068F015C169F01DC16AF0F7ECE7F060C06B
:109C6000F4F061C0F5F01200F651D96EDA6A6F00B7
:109C70007BFFF6FF6F0077FFF7FF000EF86E08001E
:109C8000F550250AD8A416D0F651D96EDA6ADE2A24
:109C9000000EDD22000E266E250E256EF4C027F084
:109CA000F5C028F093ECFAF0000E0001F56F010EFC
:109CB000F46F1200F651D96EDA6ADE2A000EDD2248
:109CC000000EF56F000EF46F1200F651D96EDA6ACD
:109CD0006F007BFFF6FF6F0077FFF7FF000EF86E57
:109CE0000800F550256E266AF4C027F0F5C028F06C
:109CF00093ECFAF00001F651D96EDA6ADE2A000E12
:109D0000DD22D2D743D2D2C176F0D3C177F0D4C10D
:109D100078F0D5C179F0EEC17AF0EFC17BF0F0C1F7
:109D20007CF0F1C17DF099ECE0F076C07CF177C079
:109D30007DF178C07EF179C07FF1E2C186F0E3C1A8
:109D400087F0E4C188F0E5C189F0000E7A6F000E5B
:109D50007B6F800E7C6F3F0E7D6F7CC176F07DC186
:109D600077F07EC178F07FC179F099ECE0F076C0B1
:109D70008AF077C08BF078C08CF079C08DF0F2EC6F
:109D8000F5F0D8A009D0E2C1EAF1E3C1EBF1E4C1FA
:109D9000ECF1E5C1EDF11AD07CC176F07DC177F030
:109DA0007EC178F07FC179F0000E7A6F000E7B6F74
:109DB000800E7C6F3F0E7D6F99ECE0F076C0EAF18B
:109DC00077C0EBF178C0ECF179C0EDF1000E866F51
:109DD000000E876F000E886F3F0E896FD2C18AF028
:109DE000D3C18BF0D4C18CF0D5C18DF06AEC05F0F5
:109DF00086C01CF687C01DF688C01EF689C01FF6F7
:109E0000E6C186F0E7C187F0E8C188F0E9C189F0D2
:109E1000EAC18AF0EBC18BF0ECC18CF0EDC18DF0A2
:109E20006AEC05F086C018F687C019F688C01AF6E5
:109E300089C01BF618C686F019C687F01AC688F0C6
:109E40001BC689F01CC68AF01DC68BF01EC68CF09E
:109E50001FC68DF06AEC05F086C00CF687C00DF6C3
:109E600088C00EF689C00FF6E6C186F0E7C187F01C
:109E7000E8C188F0E9C189F01CC68AF01DC68BF0E4
:109E80001EC68CF01FC68DF06AEC05F076D1D2C1EB
:109E900076F0D3C177F0D4C178F0D5C179F0EEC1B6
:109EA0007AF0EFC17BF0F0C17CF0F1C17DF099EC6C
:109EB000E0F076C07CF177C07DF178C07EF179C0AA
:109EC0007FF1E2C186F0E3C187F0E4C188F0E5C12B
:109ED00089F0000E7A6F000E7B6F800E7C6F3F0E54
:109EE0007D6F7CC176F07DC177F07EC178F07FC157
:109EF00079F099ECE0F076C08AF077C08BF078C00A
:109F00008CF079C08DF0F2ECF5F0D8A009D0E2C168
:109F1000EAF1E3C1EBF1E4C1ECF1E5C1EDF11AD0F6
:109F20007CC176F07DC177F07EC178F07FC179F099
:109F3000000E7A6F000E7B6F800E7C6F3F0E7D6F80
:109F400099ECE0F076C0EAF177C0EBF178C0ECF183
:109F500079C0EDF1000E866F000E876F000E886FDE
:109F60003F0E896FD2C18AF0D3C18BF0D4C18CF07F
:109F7000D5C18DF06AEC05F086C01CF687C01DF6D1
:109F800088C01EF689C01FF6E6C186F0E7C187F0DB
:109F9000E8C188F0E9C189F0EAC18AF0EBC18BF031
:109FA000ECC18CF0EDC18DF06AEC05F086C018F6BE
:109FB00087C019F688C01AF689C01BF618C686F045
:109FC00019C687F01AC688F01BC689F01CC68AF02D
:109FD0001DC68BF01EC68CF01FC68DF06AEC05F016
:109FE00086C00CF687C00DF688C00EF689C00FF645
:109FF000E6C186F0E7C187F0E8C188F0E9C189F0E1
:10A000001CC68AF01DC68BF01EC68CF01FC68DF0D4
:10A010006AEC05F0B2D0D6C17CF1D7C17DF1D8C1D0
:10A020007EF1D9C17FF1E2C186F0E3C187F0E4C1DE
:10A0300088F0E5C189F0000E00017A6F000E7B6F99
:10A04000800E7C6F3F0E7D6F7CC176F07DC177F016
:10A050007EC178F07FC179F099ECE0F076C08AF0AB
:10A0600077C08BF078C08CF079C08DF0F2ECF5F011
:10A07000D8A009D0E2C1EAF1E3C1EBF1E4C1ECF10F
:10A08000E5C1EDF11AD07CC176F07DC177F07EC1DB
:10A0900078F07FC179F0000E7A6F000E7B6F800E32
:10A0A0007C6F3F0E7D6F99ECE0F076C0EAF177C0EF
:10A0B000EBF178C0ECF179C0EDF1000E866F000E87
:10A0C000876F000E886F3F0E896FD6C18AF0D7C1A7
:10A0D0008BF0D8C18CF0D9C18DF06AEC05F086C048
:10A0E0001CF687C01DF688C01EF689C01FF6E6C1A3
:10A0F00086F0E7C187F0E8C188F0E9C189F0EAC1DC
:10A100008AF0EBC18BF0ECC18CF0EDC18DF06AEC04
:10A1100005F086C018F687C019F688C01AF689C0FF
:10A120001BF618C686F019C687F01AC688F01BC63B
:10A1300089F01CC68AF01DC68BF01EC68CF01FC6A7
:10A140008DF06AEC05F086C00CF687C00DF688C06D
:10A150000EF689C00FF6E6C186F0E7C187F0E8C1C8
:10A1600088F0E9C189F01CC68AF01DC68BF01EC6B6
:10A170008CF01FC68DF06AEC05F086C010F687C023
:10A1800011F688C012F689C013F611D0F1C259F148
:10A19000F2C25AF101015A51000AD8A43CD75951D0
:10A1A000010AD8B4B0D5030AD8B471D634D7E9C2FD
:10A1B00086F0EAC287F0EBC288F0ECC289F07CC17D
:10A1C0008AF07DC18BF07EC18CF07FC18DF06AEC8E
:10A1D00005F086C014F687C015F688C016F689C04B
:10A1E00017F610C686F011C687F012C688F013C69F
:10A1F00089F0E6C18AF0E7C18BF0E8C18CF0E9C1D3
:10A200008DF0F2ECF5F0D8A013D014C686F015C688
:10A2100087F016C688F017C689F018C68AF019C6E6
:10A220008BF01AC68CF01BC68DF075ECE3F012D0E3
:10A2300014C686F015C687F016C688F017C689F0D2
:10A240000CC68AF00DC68BF00EC68CF00FC68DF0D2
:10A2500075ECE3F086C047F287C048F288C049F247
:10A2600089C04AF247C233F048C234F049C235F0DF
:10A270004AC236F0EAC137F0EBC138F0ECC139F030
:10A28000EDC13AF0B7ECDBF033C000F634C001F6B4
:10A2900035C002F636C003F600C686F001C687F068
:10A2A00002C688F003C689F07CC18AF07DC18BF0BC
:10A2B0007EC18CF07FC18DF06AEC05F086C004F69B
:10A2C00087C005F688C006F689C007F604C633F0D5
:10A2D00005C634F006C635F007C636F0DBEC09F0EB
:10A2E00033C043F234C044F235C045F236C046F2C2
:10A2F000F6C186F0F7C187F0F8C188F0F9C189F09E
:10A3000043C28AF044C28BF045C28CF046C28DF045
:10A310006AEC05F086C008F687C009F688C00AF620
:10A3200089C00BF608C686F009C687F00AC688F011
:10A330000BC689F047C28AF048C28BF049C28CF044
:10A340004AC28DF075ECE3F086C094F187C095F1B8
:10A3500088C096F189C097F194C186F095C187F0C5
:10A3600096C188F097C189F0000E8A6F000E8B6F3E
:10A37000A00E8C6F420E8D6FF2ECF5F0D8A006D0D7
:10A38000000E0201646F500E636F37D0EAC186F091
:10A39000EBC187F0ECC188F0EDC189F094C18AF07F
:10A3A00095C18BF096C18CF097C18DF0F2ECF5F071
:10A3B000D8A00BD0EAC1ACF0EBC1ADF0ECC1AEF06F
:10A3C000EDC1AFF081ECF9F014D094C192F095C1D9
:10A3D00093F096C194F097C195F001ECDFF092C034
:10A3E000ACF093C0ADF094C0AEF095C0AFF081EC8E
:10A3F000F9F0ACC063F2ADC064F2090E0101C219FC
:10A40000D8A41200A8C124F1A9C125F13A0E266FE3
:10A41000FB0E276F7CC128F17DC129F17EC12AF195
:10A420007FC12BF1F0EC03F0A8C125F0A9C126F003
:10A430008EECFBF0A8C124F1A9C125F1110E010198
:10A44000266FD70E276F1CC628F11DC629F11EC620
:10A450002AF11FC62BF118C62CF119C62DF11AC608
:10A460002EF11BC62FF10CC630F10DC631F10EC610
:10A4700032F10FC633F110C634F111C635F112C6F0
:10A4800036F113C637F114C638F115C639F116C6C0
:10A490003AF117C63BF104C63CF105C63DF106C6CC
:10A4A0003EF107C63FF108C640F109C641F10AC6B0
:10A4B00042F10BC643F1EAC144F1EBC145F1ECC1F5
:10A4C00046F1EDC147F1000E486F000E496FA00E36
:10A4D0004A6F420E4B6FF0EC03F0A8C125F0A9C102
:10A4E00026F08EECFBF01200010E6BECF1F0010E89
:10A4F000DDECFBF0000E00016B6FC70E6C6FF40E0D
:10A500006D6F6C516D11D8A4000E6E6F010E3AEC98
:10A510000BF0000E00016B6FED0E6C6FF50E6D6FA2
:10A520006C516D11D8A4000E6E6F020E3AEC0BF058
:10A53000000E00016C6F030E6B6FA9ECF4F01E0EA1
:10A540000101246F030E256FE40E266FEA0E276FBC
:10A55000B5C228F1296BB4C22AF12B6BB3C22CF11E
:10A560002D6BB2C22EF12F6BB1C230F1316BB0C284
:10A5700032F1336BF0EC03F0010E00016A6F1E0E36
:10A580006B6F030E6C6F030EEEEC0BF0B80E256EC6
:10A59000040E266E1E0E276E030E286E000E2A6E07
:10A5A000140E296E03EC01F0000E6C6F040E6B6F3D
:10A5B000A9ECF4F0000E00016B6FA20E6C6FF80EA8
:10A5C0006D6F6C516D11D8A4000E6E6F040E3AECD5
:10A5D0000BF0010E8EEC05F0420E2B6ED90E2C6E98
:10A5E00078EC06F0000E22EC05F0000E126E6F0003
:10A5F0002CFF59F17F0E010159175951076E086A56
:10A6000007C0ACF108C0ADF1210E2B6ED80E2C6E38
:10A6100078EC06F01E0E0101246F030E256F670E05
:10A62000266FDC0E276F07C028F108C029F107C08C
:10A630002AF108C02BF1ACC12CF1ADC12DF1ACC198
:10A640002EF1ADC12FF1F0EC03F01E0E256E030EBE
:10A65000266E8EECFBF032EC0CF0080E0C6E000E49
:10A66000126E6F002CFF59F17F0E010159175951DD
:10A67000076E086AB60E00D000D0E82EFCD700D0D6
:10A6800000D000D0CB507F0B7F0AD8B4A5D06F008C
:10A690002CFF59F17F0E010159175951AC6FAD6B69
:10A6A000000E066E000E056E09D0E40E00D000D03C
:10A6B000E82EFCD700D000D0054A062ACB507F0BED
:10A6C0007F0AD8A4F2D705C025F006C026F0000EF8
:10A6D000286E0A0E276E9EEC03F025C005F026C0FA
:10A6E00006F0ACC111F01150FF0A7F0B116ED8902B
:10A6F0001130126E1E0E0101246F030E256FC20E63
:10A70000266FEB0E276F12C028F1296B05C02AF1C6
:10A7100006C02BF1F0EC03F01E0E256E030E266E24
:10A720008EECFBF0000E0101AD6F000EAC6FC0ECC3
:10A730000BF052D0000E0001666F030E656F0CC067
:10A7400067F0686BFF0E696FEAECFAF0110E010119
:10A750005A6F3C0E596FCB0EE82EFED7592FFCD7FF
:10A760005A2FFAD7B70E0C24D96EDA6A040EDA2201
:10A77000DF50116E000E0001666F030E656F0CC096
:10A7800067F0686B11C069F0EAECFAF0110E010194
:10A790005A6F3C0E596FCB0EE82EFED7592FFCD7BF
:10A7A0005A2FFAD72BD00C06070E0C18D8A402D0BB
:10A7B000130E0C6EB70E0C24D96EDA6A040EDA2270
:10A7C000DF50116E000E126E19D00C2A140E0C18E8
:10A7D000D8A4F0D7080EEDD712500101596F5A6B6B
:10A7E0005A51000AD8A40AD05951000AD8B4A2D7A5
:10A7F000010AD8B4D8D7030AD8B4E7D7040E121880
:10A80000D8B404D0080E1218D8A498D0B70E0C24CF
:10A810000101A46FA56B040EA523600093F6D9FF78
:10A82000600097F6DAFFDF50116E4ED0360E256EBF
:10A83000320EB4EC04F074D0390E256E300EB4EC48
:10A8400004F06ED0310E256E300EB4EC04F068D0FA
:10A85000390E256E300EB4EC04F062D0320E256E47
:10A86000300EB4EC04F05CD0390E256E300EB4EC32
:10A8700004F056D0300E116E600093F6D9FF6000E0
:10A8800097F6DAFF600047F0DFFF4AD0360E256EFC
:10A89000300EB4EC04F044D0320E256E300EB4EC21
:10A8A00004F03ED0390E256E300EB4EC04F038D0F2
:10A8B000350E256E300EB4EC04F032D0390E256E14
:10A8C000300EB4EC04F02CD00C50596F5A6B5A5126
:10A8D000000AD8A425D05951080AD8B4A7D7010A2C
:10A8E000D8B4AAD7030AD8B4ADD7010AD8B4B0D720
:10A8F000070AD8B4B3D7010AD8B4B6D7030AD8B474
:10A90000B9D7010AD8B4C2D71F0AD8B4C5D7010A2B
:10A91000D8B4C8D7030AD8B4CBD7010AD8B4CED795
:10A92000010E00016A6FB80E6B6F040E6C6F030EA0
:10A93000EEEC0BF0000E126EC0EC0BF0100E1218C5
:10A94000D8A408D0D10E055C070E0658D8A002D0B6
:10A950003901A38F3901A3BF04D0200E1218D8A447
:10A960007ED6A3BF21D1200E1218D8A41DD1000E6F
:10A9700000016C6F040E6B6FA9ECF4F0000E000187
:10A980006B6FAE0E6C6FF50E6D6F6C516D11D8A4C0
:10A99000000E6E6F040E3AEC0BF0010E8EEC05F01B
:10A9A0009F0E2B6EF10E2C6E78EC06F0B80E256E15
:10A9B000040E266E8EECFBF032EC0CF0BF0E0101A3
:10A9C000A46F040EA56F000E0A6E000E096E000E35
:10A9D000D16F000ED06FD15105E1060ED05DD8B019
:10A9E00084D001D082D0B40E2B6EFF0E2C6E78EC8A
:10A9F00006F0600093F6D9FF600097F6DAFFDF50AB
:10AA00004AEC0CF0010120EE01F0A451D926A55129
:10AA1000DA22DF504AEC0CF0090E4AEC0CF0600030
:10AA200093F6D9FF600097F6DAFFDF50D00F0201EE
:10AA30009E6F9E39F00B116E010120EE01F0A451C2
:10AA4000D926A551DA22DF50D00F02019D6F115097
:10AA50009D25116E0101D051B608D96ED151D8A0F3
:10AA6000E82A0208DA6E600047F0DFFF1E0E246F4E
:10AA7000030E256F8E0E266FE80E276FD051070844
:10AA8000286FD151D8A0E82A0008296F09C02AF1FF
:10AA90000AC02BF1D05107082C6FD151D8A0E82A59
:10AAA00000082D6FD051B608D96ED151D8A0E82A30
:10AAB0000208DA6EDF50596F59512E6F2F6BF0EC90
:10AAC00003F01E0E256E030E266E8EECFBF0020EBA
:10AAD0000924096E000E0A200A6E0101A44BA52B61
:10AAE000A44BA52BD04BD12B76D732EC0CF01E0EFD
:10AAF0000101246F030E256FD10E266FE90E276F1B
:10AB0000B6C228F1296BB5C22AF12B6BB4C22CF165
:10AB10002D6BB3C22EF12F6BB2C230F1316BB1C2CB
:10AB200032F1336BF0EC03F01E0E256E030E266E31
:10AB30008EECFBF0000E0201AF6F010EB06F000E45
:10AB4000B76FAF0E0101A46F020EA56FA4C13AF05A
:10AB5000A5C13BF0000E3D6E080E3C6E680ED9ECB0
:10AB600004F0280E2B6EFB0E2C6E78EC06F032EC07
:10AB70000CF0000E00016B6FC30E6C6FF50E6D6F65
:10AB80006C516D11D8A4000E6E6F040E3AEC0BF0F0
:10AB9000690E2B6EE80E2C6E78EC06F0010E6BEC55
:10ABA000F1F032EC0CF02BD0680E2B6EE90E2C6E0F
:10ABB00078EC06F0000E00016B6F300E6C6FF50E36
:10ABC0006D6F6C516D11D8A4000E6E6F020E3AECD1
:10ABD0000BF0000E00016B6F1B0E6C6FF50E6D6FAE
:10ABE0006C516D11D8A4000E6E6F030E3AEC0BF091
:10ABF000000E00016C6F040E6B6FA9ECF4F0020EF6
:10AC00008EEC05F0120000017C6F7CC07DF0010E1F
:10AC1000DDECFBF0090E0001716F1E0E706FE40E8B
:10AC2000E82EFED7702FFCD7712FFAD700F0720EE6
:10AC3000256E266AB60E276EEE0E286E39EC01F0F0
:10AC4000000E0001726F1E0E256E030E266E7D51E2
:10AC5000200D3E0EF324276E060EF420286E000E03
:10AC60002A6E080E296E03EC01F0010E6A6F1E0EAB
:10AC70006B6F030E6C6F010EEEEC0BF0820E2B6E01
:10AC8000FB0E2C6E78EC06F000017D51300F4AEC83
:10AC90000CF03A0E4AEC0CF01E0E256E030E266EDA
:10ACA0008EECFBF032EC0CF0000E0001666F030E30
:10ACB000656F000E686F070E676F4D0E696FEAECE7
:10ACC000FAF0000E00017F6F000E7E6F000E666FBF
:10ACD000030E656F090E7E25676F000E7F21686F7A
:10ACE0007D51200D260E706F060E716FF350702788
:10ACF000F45071237E517025D96E7F517121DA6E27
:10AD0000DF50696FEAECFAF000017E4B7F2B7FBFCA
:10AD1000DDD77F5104E10C0E7E5DD8A0D7D7060E9B
:10AD20006B6FB10E6C6FFF0E6D6F6C516D11D8A40F
:10AD3000000E6E6F040E3AEC0BF0000E00017F6FF8
:10AD4000000E7E6F000E666F040E656F090E7E2585
:10AD5000676F000E7F21686F7D51200D260E706F8A
:10AD6000060E716F0C0E7027000E7123F3507027C2
:10AD7000F45071237E517025D96E7F517121DA6EA6
:10AD8000DF50696FEAECFAF000017E4B7F2B7FBF4A
:10AD9000D9D77F5104E10C0E7E5DD8A0D3D7000E29
:10ADA000086E000E076E000E0201966F720E010112
:10ADB000A86FA96B000E00016C6F020E6B6FA9ECFF
:10ADC000F4F0000E00017F6F000E7E6F7D51200DAC
:10ADD000260E706F060E716FF3507027F4507123BA
:10ADE0007E517025D96E7F517121DA6EDF500201DC
:10ADF000946F00017E4B7F2B0101BA51200D260E6E
:10AE00000001706F060E716FF3507027F4507123BC
:10AE10007E517025D96E7F517121DA6EDF500201AB
:10AE2000946F00017FBF06D07F5109E1170E7E5D50
:10AE3000D8B005D0020195519419D8B4DAD7200EB4
:10AE40000501006F7EC025F07FC026F0000E286E41
:10AE50000A0E276EDDECFDF02550300F0501016F65
:10AE60007EC025F07FC026F0000E286E0A0E276EE9
:10AE7000CBEC00F02550300F0501026F680E036F18
:10AE80000201962B000E0501046FAAD00A0E0101E3
:10AE9000C219D8A40ED0990E2B6EFE0E2C6E78EC33
:10AEA00006F0000E256E050E266E8EECFBF032ECE1
:10AEB0000CF0090E00016A6F000E6B6F050E6C6FCF
:10AEC000010EEEEC0BF0A8D00A0E0101C219D8A4B5
:10AED0000ED0750E2B6EFE0E2C6E78EC06F0000E6A
:10AEE000256E050E266E8EECFBF032EC0CF0090E92
:10AEF00000016A6F000E6B6F050E6C6F020EEEECB8
:10AF00000BF08AD00A0E0101C219D8A40ED0A50EEA
:10AF10002B6EFE0E2C6E78EC06F0000E256E050EE4
:10AF2000266E8EECFBF032EC0CF00D0E00016A6F19
:10AF3000000E6B6F050E6C6F010EEEEC0BF06CD01B
:10AF40000A0E0101C219D8A40ED0810E2B6EFE0E7E
:10AF50002C6E78EC06F0000E256E050E266E8EEC3B
:10AF6000FBF032EC0CF00D0E00016A6F000E6B6FFF
:10AF7000050E6C6F020EEEEC0BF04ED0110E6A6FE8
:10AF8000000E6B6F050E6C6F010EEEEC0BF00A0EEF
:10AF90000101C219D8A440D0B10E2B6EFE0E2C6E4A
:10AFA00078EC06F0000E256E050E266E8EECFBF09A
:10AFB00032EC0CF031D0110E6A6F000E6B6F050E83
:10AFC0006C6F020EEEEC0BF00A0E0101C219D8A450
:10AFD00023D08D0E2B6EFE0E2C6E78EC06F0E2D791
:10AFE000020196510001706F716B7151000AD8A473
:10AFF00013D07051010AD8B449D7030AD8B464D722
:10B00000010AD8B47FD7070AD8B49AD7010AD8B4AE
:10B01000B5D7030AD8B4CFD794C295F200017E4BBE
:10B020007F2B020E0001716FA00E706F920EE82E42
:10B03000FED7702FFCD7712FFAD700F000017FBF29
:10B04000C5D67F5105E1170E7E5DD8B01200BED681
:10B05000120067C1A0F168C1A1F1500EA019A111A1
:10B06000D8B405D0020EA119A011D8A4A0D1140EF5
:10B07000C26F1E0E246F030E256FBE0E266FDA0EF2
:10B08000276FA0C128F1A1C129F1A0C12AF1A1C156
:10B090002BF1C2C12CF12D6BF0EC03F01E0E256ECE
:10B0A000030E266E8EECFBF0A0C15DF1A1C15EF136
:10B0B00029ECF4F05DC1E2F15EC1E3F15FC1E4F1BE
:10B0C00060C1E5F1040E0101A0255D6F000EA12114
:10B0D0005E6F29ECF4F05DC1E6F15EC1E7F15FC19E
:10B0E000E8F160C1E9F1080E0101A0255D6F000ED5
:10B0F000A1215E6F29ECF4F05DC1E9F25EC1EAF2D4
:10B100005FC1EBF260C1ECF20C0E0101A0255D6F96
:10B11000000EA1215E6F29ECF4F05DC1EEF15EC17D
:10B12000EFF15FC1F0F160C1F1F1100E0101A02556
:10B130005D6F000EA1215E6F29ECF4F05DC1EDF2B0
:10B140005EC1EEF25FC1EFF260C1F0F2140E0101D8
:10B15000A0255D6F000EA1215E6F29ECF4F05DC1AA
:10B16000DEF15EC1DFF15FC1E0F160C1E1F1180E17
:10B170000101A0255D6F000EA1215E6F29ECF4F0A6
:10B180005DC1DAF15EC1DBF15FC1DCF160C1DDF10F
:10B190001C0E0101A0255D6F000EA1215E6F29EC40
:10B1A000F4F05DC1D6F15EC1D7F15FC1D8F160C1E5
:10B1B000D9F1200E0101A0255D6F000EA1215E6F67
:10B1C00029ECF4F05DC1E5F25EC1E6F25FC1E7F2A1
:10B1D00060C1E8F2240E0101A0255D6F000EA121DF
:10B1E0005E6F29ECF4F05DC1E1F25EC1E2F25FC195
:10B1F000E3F260C1E4F2280E0101A0255D6F000EAC
:10B20000A1215E6F29ECF4F05DC1DDF25EC1DEF2DA
:10B210005FC1DFF260C1E0F22C0E0101A0255D6F7D
:10B22000000EA1215E6F29ECF4F05DC1D2F15EC188
:10B23000D3F15FC1D4F160C1D5F1160E0101C26F27
:10B240001E0E246F030E256F820E266FD90E276FF8
:10B25000380EA025286F000EA121296F380EA025D9
:10B260002A6F000EA1212B6FC2C12CF12D6BF0ECC7
:10B2700003F01E0E256E030E266E8EECFBF0000E04
:10B280000101D16F000ED06FD15120E1080ED05DC9
:10B29000D8B01CD0D051A025696FD151A1216A6FBF
:10B2A000380E6925596F000E6A215A6FA2ECFEF024
:10B2B00001016B6FD50ED025D96E020ED121DA6E49
:10B2C0006000AFF5DFFFD04BD12BDED7400EA025BD
:10B2D000596F000EA1215A6FA2ECFEF00101BA6F66
:10B2E000410EA025596F000EA1215A6FA2ECFEF06D
:10B2F0000101FF6F420EA025596F000EA1215A6F68
:10B30000A2ECFEF00101B76F430EA025596F000EAD
:10B31000A1215A6FA2ECFEF00101B96F440EA025E5
:10B32000596F000EA1215A6FA2ECFEF00101B46F1B
:10B33000450EA025596F000EA1215A6FA2ECFEF018
:10B340000101B36F460EA025596F000EA1215A6F5F
:10B35000A2ECFEF00101B86F470EA025596F000E58
:10B36000A1215A6FA2ECFEF00101BB6F000EC26F6B
:10B37000070E2B6EDF0E2C6E78EC06F0500E0101DE
:10B38000A019A111D8A406D00D0E2B6EEE0E2C6EB6
:10B3900078EC06F0020E0101A119A011D8A4120048
:10B3A000850E2B6EEF0E2C6E78EC06F012001E0E42
:10B3B000246F030E256FD30E266FE50E276FA0C1F5
:10B3C00028F1A1C129F1A0C12AF1A1C12BF1F0EC12
:10B3D00003F01E0E256E030E266E8EECFBF012009F
:10B3E0000001FF6F000E00016C6F010E6B6FA9EC86
:10B3F000F4F00001FF51D8A413D08B0E2B6EE90E90
:10B400002C6E78EC06F0740E0001636FF90E646F19
:10B4100063516411D8A4000E656FDFECF9F011D010
:10B42000800E636FF60E646F63516411D8A4000E32
:10B43000656FDFECF9F0D30E2B6EE70E2C6E78EC17
:10B4400006F0000E00016C6F020E6B6FA9ECF4F0B9
:10B450001F0E0001636FF40E646F63516411D8A472
:10B46000000E656FDFECF9F05AECF8F06DC0FAF100
:10B470006EC0FBF16FC0FCF170C0FDF1000E6C6F8F
:10B48000030E6B6FA9ECF4F0F5ECF7F06DC0F6F17C
:10B490006EC0F7F16FC0F8F170C0F9F1340E636F50
:10B4A000F40E646F63516411D8A4000E656FDFEC75
:10B4B000F9F0000E00016C6F040E6B6FA9ECF4F054
:10B4C000490E0001636FF40E646F63516411D8A4D8
:10B4D000000E656FDFECF9F0BFECF8F06DC0F2F133
:10B4E0006EC0F3F16FC0F4F170C0F5F1000E010110
:10B4F000D16F000ED06F0001FF51D8B41AD070C1C7
:10B5000076F071C177F072C178F073C179F0FAC149
:10B510007AF0FBC17BF0FCC17CF0FDC17DF099ECC1
:10B52000E0F076C0FAF177C0FBF178C0FCF179C0A9
:10B53000FDF1A8C124F1A9C125F1CA0E0101266FB0
:10B54000FA0E276FFAC128F1FBC129F1FCC12AF1DB
:10B55000FDC12BF1000E2D6FB00E2C6FF0EC03F03F
:10B56000A8C125F0A9C126F08EECFBF032EC0CF05E
:10B570001E0E0101246F030E256F780E266FFF0E3D
:10B58000276FFAC128F1FBC129F1FCC12AF1FDC1E5
:10B590002BF1F0EC03F00C0E00016A6F1E0E6B6FC6
:10B5A000030E6C6F020EEEEC0BF0000E666F020ED7
:10B5B000656F000E686F110E676F070E696FEAEC1A
:10B5C000FAF00001FF51D8B41AD074C176F075C1F9
:10B5D00077F076C178F077C179F0F6C17AF0F7C1EB
:10B5E0007BF0F8C17CF0F9C17DF099ECE0F076C019
:10B5F000F6F177C0F7F178C0F8F179C0F9F1A8C198
:10B6000024F1A9C125F1DD0E0101266FFA0E276F85
:10B61000F6C128F1F7C129F1F8C12AF1F9C12BF1DE
:10B62000000E2D6FB00E2C6FF0EC03F0A8C125F0CA
:10B63000A9C126F08EECFBF032EC0CF01E0E0101DD
:10B64000246F030E256F780E266FFF0E276FF6C14D
:10B6500028F1F7C129F1F8C12AF1F9C12BF1F0EC79
:10B6600003F00C0E00016A6F1E0E6B6F030E6C6F01
:10B67000030EEEEC0BF0000E666F030E656F000E0E
:10B68000686F110E676F070E696FEAECFAF0BFEC96
:10B69000F8F06DC0F2F16EC0F3F16FC0F4F170C05C
:10B6A000F5F1FF51D8B41AD078C176F079C177F0AE
:10B6B0007AC178F07BC179F0F2C17AF0F3C17BF006
:10B6C000F4C17CF0F5C17DF099ECE0F076C0F2F1C8
:10B6D00077C0F3F178C0F4F179C0F5F1A8C124F195
:10B6E000A9C125F1A30E0101266FFA0E276FF2C141
:10B6F00028F1F3C129F1F4C12AF1F5C12BF1000EB3
:10B700002D6FB00E2C6FF0EC03F0A8C125F0A9C18D
:10B7100026F08EECFBF032EC0CF01E0E0101246FD3
:10B72000030E256FA40E266FFF0E276FF2C128F1BE
:10B73000F3C129F1F4C12AF1F5C12BF1F0EC03F0CA
:10B740000C0E00016A6F1E0E6B6F030E6C6F040E01
:10B75000EEEC0BF0000E666F040E656F000E686F66
:10B76000110E676F070E696FEAECFAF0120036509F
:10B77000800B0001606F36503624626F35BE6281E7
:10B780006251D8B40DD06229D8A408D0000E336E0F
:10B79000000E346E000E356E000E366E358E08D0FB
:10B7A000000E336E000E346E000E356E000E366ED7
:10B7B0003A50800B601B3A503A24616F39BE618168
:10B7C0006151D8B40DD06129D8A408D0000E376ECD
:10B7D000000E386E000E396E000E3A6E398E08D0AB
:10B7E000000E376E000E386E000E396E000E3A6E87
:10B7F0006151D8B403D06251D8A409D0000E336E81
:10B80000000E346E000E356E000E366E120039508A
:10B8100033026F00CCFF6BF06F00D0FF6CF06B5108
:10B82000636F646B656B666B6C51676F686B696B9C
:10B830006A6B385034026F00CCFF6BF06F00D0FFA2
:10B840006CF06B516327000E6423652366236C51F3
:10B850006727000E682369236A23375035026F007B
:10B86000CCFF6BF06F00D0FF6CF06B516327000EC4
:10B870006423652366236C516727000E68236923C0
:10B880006A2365C066F064C065F063C064F0636BF2
:10B89000375034026F00CCFF6BF06F00D0FF6CF0BC
:10B8A0006B5163276C516423000E6523000E6623E1
:10B8B000385033026F00CCFF6BF06F00D0FF6CF09C
:10B8C0006B5163276C516423000E6523000E6623C1
:10B8D00065C066F064C065F063C064F0636B3750A8
:10B8E00033026F00CCFF6BF06F00D0FF6CF06B5138
:10B8F00063276C516423000E6523000E66233950C4
:10B9000034026F00CCFF6BF06F00D0FF6CF06B5116
:10B9100067276C516823000E6923000E6A23385094
:10B9200035026F00CCFF6BF06F00D0FF6CF06B51F5
:10B9300067276C516823000E6923000E6A23395073
:10B9400035026F00CCFF6BF06F00D0FF6CF06B51D5
:10B950003B6E6C513C6E3D6A3E6A3DC03EF03CC061
:10B960003DF03BC03CF03B6A3B5067273C506823AE
:10B970003D5069233E506A2366516727000E6823B5
:10B9800069236A2365C066F064C065F063C064F033
:10B99000636B615162C03BF03C6A3B26000E3C2267
:10B9A000820E3B246B6FFF0E3C206C6F0FD0D89043
:10B9B0006737683769376A3766BF6781D8906337FA
:10B9C0006437653766376B07D8A06C0769AFEFD768
:10B9D000000E616F66AF17D0FF0E63153B6EFF0E52
:10B9E00064153C6EFF0E65153D6E7F0E66153E6E4E
:10B9F0003B503C103D103E10D8B403D0010E616F97
:10BA000002D067B1FBD76151D8B41FD0010E6727B0
:10BA1000000E682369236A236AA117D067C03BF030
:10BA200068C03CF069C03DF06AC03EF03E343E3232
:10BA30003D323C323B323BC067F03CC068F03DC019
:10BA400069F03EC06AF06B4B6C2B6CBF0DD06C5133
:10BA500003E16B29D8A008D0000E676F000E686F55
:10BA6000800E696F7F0E20D06CBF05D06C510EE147
:10BA70006B05D8B00BD0000E676F000E686F000E1C
:10BA8000696F000E6A6F000E606F0FD06BC062F0BE
:10BA9000FF0E6717FF0E68177F0E6917000E6A17F3
:10BAA00062B1698FD89062316A6F60516A1367C062
:10BAB00033F068C034F069C035F06AC036F0120067
:10BAC000500E59195A11D8B405D0020E5A195911ED
:10BAD000D8A47ED11E0E246F030E256FC40E266FD0
:10BAE000E60E276F59C128F15AC129F159C12AF12F
:10BAF0005AC12BF1F0EC03F01E0E256E030E266EDC
:10BB00008EECFBF059C12BF05AC12CF0E2C12DF0A4
:10BB1000E3C12EF0E4C12FF0E5C130F046EC05F0B2
:10BB2000040E010159252B6E000E5A212C6EE6C120
:10BB30002DF0E7C12EF0E8C12FF0E9C130F046EC5E
:10BB400005F0080E010159252B6E000E5A212C6EAE
:10BB5000E9C22DF0EAC22EF0EBC22FF0ECC230F0B9
:10BB600046EC05F00C0E010159252B6E000E5A21F2
:10BB70002C6EEEC12DF0EFC12EF0F0C12FF0F1C10F
:10BB800030F046EC05F0100E010159252B6E000E29
:10BB90005A212C6EEDC22DF0EEC22EF0EFC22FF026
:10BBA000F0C230F046EC05F0140E010159252B6E61
:10BBB000000E5A212C6EDEC12DF0DFC12EF0E0C147
:10BBC0002FF0E1C130F046EC05F0180E01015925C7
:10BBD0002B6E000E5A212C6EDAC12DF0DBC12EF037
:10BBE000DCC12FF0DDC130F046EC05F01C0E010188
:10BBF00059252B6E000E5A212C6ED6C12DF0D7C1BF
:10BC00002EF0D8C12FF0D9C130F046EC05F0200E4F
:10BC1000010159252B6E000E5A212C6EE5C22DF024
:10BC2000E6C22EF0E7C22FF0E8C230F046EC05F095
:10BC3000240E010159252B6E000E5A212C6EE1C2F3
:10BC40002DF0E2C22EF0E3C22FF0E4C230F046EC59
:10BC500005F0280E010159252B6E000E5A212C6E7D
:10BC6000DDC22DF0DEC22EF0DFC22FF0E0C230F0D8
:10BC700046EC05F02C0E010159252B6E000E5A21C1
:10BC80002C6ED2C12DF0D3C12EF0D4C12FF0D5C16E
:10BC900030F046EC05F0000E01015E6F000E5D6FA6
:10BCA00059515D255B6F5A515E215C6F300E5B25EB
:10BCB000256E000E5C21266E000E276EEBEC02F066
:10BCC00001015D4B5E2B5EBFEBD75E5104E1080EB8
:10BCD0005D5DD8A0E5D7000E5E6F000E5D6F595117
:10BCE0005D255B6F5A515E215C6F380E5B25256EBA
:10BCF000000E5C21266ED50E5D25D96E020E5E21EA
:10BD0000DA6EDF50276EEBEC02F001015D4B5E2B2B
:10BD10005EBFE5D75E5104E1080E5D5DD8A0DFD7B8
:10BD2000400E5925256E000E5A21266EBAC127F005
:10BD3000EBEC02F0410E01015925256E000E5A214F
:10BD4000266EFFC127F0EBEC02F0420E01015925EF
:10BD5000256E000E5A21266EB7C127F0EBEC02F0DB
:10BD6000430E01015925256E000E5A21266EB9C1D8
:10BD700027F0EBEC02F0440E01015925256E000E70
:10BD80005A21266EB4C127F0EBEC02F0450E0101FA
:10BD90005925256E000E5A21266EB3C127F0EBEC13
:10BDA00002F0460E01015925256E000E5A21266E1D
:10BDB000B8C127F0EBEC02F0470E01015925256EC2
:10BDC000000E5A21266EBBC127F0EBEC02F01200E8
:10BDD0001E0E246F030E256F950E266FE30E276F40
:10BDE00059C128F15AC129F159C12AF15AC12BF17F
:10BDF000F0EC03F01E0E256E030E266E8EECFBF0AB
:10BE0000120033C2A4F034C2A5F035C2A6F036C287
:10BE1000A7F092C0A4F093C0A5F094C0A6F095C07E
:10BE2000A7F0A4C096F0A5C097F0A6C098F0A7C050
:10BE300099F0180E05D0D8909933983397339633EC
:10BE4000E82EF9D796519E6F9F6B9FBF0FD09F51E1
:10BE500004E1960E9E5DD8A009D092C092F093C0E6
:10BE600093F094C094F095C095F01200A4C096F0A1
:10BE7000A5C097F0A6C098F0A7C099F0200E05D0F5
:10BE8000D8909933983397339633E82EF9D7965153
:10BE9000D8B412D092C033F093C034F094C035F0CF
:10BEA00095C036F0DBEC09F033C092F034C093F06B
:10BEB00035C094F036C095F000019FBF06D09F5169
:10BEC0001FE17E0E9E5DD8B01BD0A4C033F0A5C08C
:10BED00034F0A6C035F0A7C036F0000E376E000E65
:10BEE000386E000E396E000E3A6EB7ECDBF033C0E0
:10BEF00092F034C093F035C094F036C095F0120043
:10BF0000000E7A6F000E7B6F000E7C6F4B0E7D6F04
:10BF100092C076F093C077F094C078F095C079F035
:10BF200099ECE0F076C0A0F077C0A1F078C0A2F064
:10BF300079C0A3F0000E7A6F000E7B6F000E7C6F4D
:10BF4000CB0E7D6FA0C076F0A1C077F0A2C078F0D4
:10BF5000A3C079F099ECE0F076C09AF077C09BF03E
:10BF600078C09CF079C09DF09AC086F09BC087F0A5
:10BF70009CC088F09DC089F092C08AF093C08BF07D
:10BF800094C08CF095C08DF06AEC05F086C0A8F0E6
:10BF900087C0A9F088C0AAF089C0ABF0000E866FF8
:10BFA000000E876F000E886F3F0E896FA8C08AF061
:10BFB000A9C08BF0AAC08CF0ABC08DF0F2ECF5F00C
:10BFC000D8B02DD092C07AF093C07BF094C07CF0B2
:10BFD00095C07DF0A8C076F0A9C077F0AAC078F02F
:10BFE000ABC079F099ECE0F076C0A0F077C0A1F09A
:10BFF00078C0A2F079C0A3F0A0C076F0A1C077F01D
:10C00000A2C078F0A3C079F0000E7A6F000E7B6FAB
:10C01000800E7C6FBF0E7D6F99ECE0F053D0000E68
:10C02000866F000E876F000E886FBF0E896FA8C0E5
:10C030008AF0A9C08BF0AAC08CF0ABC08DF0F2ECF6
:10C04000F5F0D8A02DD092C07AF093C07BF094C0C8
:10C050007CF095C07DF0A8C076F0A9C077F0AAC0AA
:10C0600078F0ABC079F099ECE0F076C0A0F077C042
:10C07000A1F078C0A2F079C0A3F0A0C076F0A1C072
:10C0800077F0A2C078F0A3C079F0000E7A6F000EAE
:10C090007B6F800E7C6F3F0E7D6F99ECE0F012D0CD
:10C0A000A8C076F0A9C077F0AAC078F0ABC079F04C
:10C0B00092C07AF093C07BF094C07CF095C07DF084
:10C0C00099ECE0F076C0A8F077C0A9F078C0AAF0AB
:10C0D00079C0ABF0A4C096F0A5C097F0A6C098F0C8
:10C0E000A7C099F0200E05D0D89099339833973394
:10C0F0009633E82EF9D79651D8B412D0A8C033F0B1
:10C10000A9C034F0AAC035F0ABC036F0DBEC09F0C2
:10C1100033C0A8F034C0A9F035C0AAF036C0ABF0E7
:10C12000A8C092F0A9C093F0AAC094F0ABC095F05B
:10C13000120000017951800B826F79517925846F4B
:10C1400078BF84818451D8B40DD08429D8A408D074
:10C15000000E766F000E776F000E786F000E796F0D
:10C16000788F06D0000E766F000E776F000E786F16
:10C17000000E796F7D51800B836F82518319D8A493
:10C18000828D7D517D25836F7CBF83818351D8B49F
:10C190000DD08329D8A408D0000E7A6F000E7B6FD3
:10C1A000000E7C6F000E7D6F7C8F06D0000E7A6FC4
:10C1B000000E7B6F000E7C6F000E7D6F8451835DDF
:10C1C000D8B022D082AD02D0800E821B84C085F010
:10C1D00083C084F085C083F076C085F07AC076F0A5
:10C1E00085C07AF077C085F07BC077F085C07BF0A2
:10C1F00078C085F07CC078F085C07CF079C085F08F
:10C200007DC079F085C07DF0000E856F845183C0BC
:10C210007EF07F6B7E5F000E7F5B7FBF2CD07F51F7
:10C2200004E11A0E7E5DD8A026D0765177117811E0
:10C230007911D8B402D0010E01D0000E856F000E26
:10C24000766F000E776F000E786F000E796F83C0E7
:10C2500084F015D085A105D0D89085310109856F6E
:10C2600002D0D890853376B1858F7935793378339C
:10C2700077337633842B8351845DD8A0EBD782BD8E
:10C2800028D08451D8A409D0000E766F000E776FA5
:10C29000000E786F000E796F12007A5176277B516D
:10C2A00077237C5178237D51792379A171D085A1A1
:10C2B00005D0D89085310109856F02D0D89085339B
:10C2C00076B1858F79357933783377337633842B2C
:10C2D0005FD07A51765D7B5177597C51785979518D
:10C2E000800A7E6F7D51800A7E59D8B025D0765164
:10C2F0007A5D7E6F77517B597F6F78517C59806F63
:10C3000079517D59816FFF0E7E25766FFF0E7F215B
:10C31000776FFF0E8021786FFF0E8121796F800E7D
:10C32000821B856D8551D8A40FD0010E7627000E93
:10C3300077237823792308D07A51765F7B51775B16
:10C340007C51785B7D51795B765177117811791149
:10C35000D8A41CD08551D8A419D0000E766F000E39
:10C36000776F000E786F000E796F1200D8907637D5
:10C3700077377837793785BF768185A102D0D88025
:10C3800001D0D89085378451D8A4840778AFEED7F0
:10C39000000E836F85AF0BD085C07EF07F0E7E17B9
:10C3A000D8B403D0010E836F02D076B1FBD783518E
:10C3B000D8B420D0010E7627000E77237823792376
:10C3C00079A118D076C07EF077C07FF078C080F079
:10C3D00079C081F08135813380337F337E337EC0F5
:10C3E00076F07FC077F080C078F081C079F0842942
:10C3F000D8A4842B8429D8B403D08451D8A40DD0D8
:10C40000000E766F000E776F000E786F000E796F5A
:10C410008451D8A402D0000E826F84A102D0788FFC
:10C4200001D0789FD8908431796F82BF798F76C0A0
:10C4300076F077C077F078C078F079C079F01200A4
:10C440000001FF6F000E01019F6F000E9E6F000E36
:10C450000201586F000E576F000E566F000E556F99
:10C46000000E01015A6F000E596FA2ECFEF00B6E28
:10C470000BC0A6F20001FF05D8A464D0FE0E2B6EFF
:10C48000EB0E2C6E78EC06F01B0E2B6EEC0E2C6E69
:10C4900078EC06F00A0E256E0B50C7EC07F0300F53
:10C4A0004AEC0CF00A0E256E0B5008EC0AF0300F27
:10C4B0004AEC0CF032EC0CF0110E2B6EF20E2C6EDE
:10C4C00078EC06F0000E01015A6F010E596FA2ECD4
:10C4D000FEF003011E6F000E01015A6F020E596F2C
:10C4E000A2ECFEF003011F6F000E01015A6F030E54
:10C4F000596FA2ECFEF00301206F000E01015A6F8C
:10C50000040E596FA2ECFEF00301216F000E010131
:10C510005A6F050E596FA2ECFEF00301226F000E58
:10C5200001015A6F060E596FA2ECFEF00301236F52
:10C53000000E246F1E0E256E030E266E8EECFBF091
:10C5400032EC0CF0000E0201586F000E576F57C20C
:10C550005DF158C25EF1050ED89001015D375E377E
:10C56000E82EFAD7A00E5D250201556F000E0101DD
:10C570005E210201566F0001FF05D8A435D01E0EC2
:10C580000101246F030E256F330E266FF10E276F06
:10C5900055C228F156C229F1F0EC03F01E0E256EAB
:10C5A000030E266E8EECFBF0000E01019F6F180E3D
:10C5B0009E6F9E51020155250101596F9F51020145
:10C5C000562101015A6FA2ECFEF00B6E0B504AECA3
:10C5D0000CF001019E4B9F2B9F5104E11F0E9E5DAD
:10C5E000D8A0E7D732EC0CF0000E01019F6F000ECF
:10C5F0009E6F9E51020155250101596F9F51020105
:10C60000562101015A6FA2ECFEF00B6E0001FF05EE
:10C61000D8A414D01E0E0101246F030E256FD40E72
:10C62000266FFE0E276F0BC028F1296BF0EC03F08C
:10C630001E0E256E030E266E8EECFBF001019E4B46
:10C640009F2B9F5104E10C0E9E5DD8A0D2D7000114
:10C65000FF05D8B432EC0CF0000E01019F6F000E04
:10C660009E6F9E510201552501015D6F9F51020190
:10C67000562101015E6F0C0E5D25596F000E5E2183
:10C680005A6FA2ECFEF00B6E0001FF05D8A414D087
:10C690001E0E0101246F030E256FD40E266FFE0EB1
:10C6A000276F0BC028F1296BF0EC03F01E0E256EEE
:10C6B000030E266E8EECFBF001019E4B9F2B9F51CB
:10C6C00004E10C0E9E5DD8A0CCD70001FF05D8B4C4
:10C6D00032EC0CF00201574B582B585105E10A0E71
:10C6E000575DD8B0120033D712008951800B966F76
:10C6F000895189259D6F88BF9D819D51D8B40DD0EA
:10C700009D29D8A408D0000E866F000E876F000EFA
:10C71000886F000E896F888F06D0000E866F000E1E
:10C72000876F000E886F000E896F8D51800B961BEE
:10C730008D518D259E6F8CBF9E819E51D8B40DD09A
:10C740009E29D8A408D0000E8A6F000E8B6F000EB1
:10C750008C6F000E8D6F8C8F06D0000E8A6F000ECE
:10C760008B6F000E8C6F000E8D6F8A518B118C11A8
:10C770008D11D8A417D0000E866F000E876F000EA3
:10C78000886F000E896F800E88137F0E8913965173
:10C79000891386C086F087C087F088C088F089C07A
:10C7A00089F012009D51D8A409D0000E866F000EAA
:10C7B000876F000E886F000E896F12009E519DC01A
:10C7C0008EF08F6B8E5F000E8F5B7F0E8E25976FC6
:10C7D000000E8F21986F86C092F087C093F088C0BA
:10C7E00094F089C095F0000E866F000E876F000EE2
:10C7F000886F000E896F000E996F000E9A6F000E01
:10C800009B6F000E9C6F000E9E6F28D09E51D8B477
:10C8100011D0D8909237933794379537D890863780
:10C820008737883789379CBF8681D89099379A3760
:10C830009B379C378A51925D8B5193598C519459F7
:10C840008D519559D8A009D09C8D8A51925F8B51FA
:10C85000935B8C51945B8D51955B9E2B190E9E655D
:10C86000D5D79251931194119511D8B411D09981C3
:10C870000FD0D89086378737883789379CBF868115
:10C88000D89099379A379B379C379707D8A0980745
:10C8900088AFEFD7000E9E6F9CAF17D0FF0E991593
:10C8A0008E6FFF0E9A158F6FFF0E9B15906F7F0E88
:10C8B0009C15916F8E518F1190119111D8B403D0A6
:10C8C000010E9E6F02D086B1FBD79E51D8B41FD007
:10C8D000010E8627000E87238823892389A117D07C
:10C8E00086C08EF087C08FF088C090F089C091F02C
:10C8F0009135913390338F338E338EC086F08FC055
:10C9000087F090C088F091C089F0974B982B98BF22
:10C9100010D0985103E19729D8A00BD0000E986F42
:10C920009769000E866F000E876F000E886F000EED
:10C93000896F98BF05D0985111E19705D8B00ED0F6
:10C94000000E986F000E976F000E866F000E876FB7
:10C95000000E886F000E896F000E966F97C09DF0D5
:10C960009DA102D0888F01D0889FD8909D31896F7A
:10C970000ED7BCC0D4F0BDC0D5F0BEC0D6F0BFC08D
:10C98000D7F0C0C0D8F0C1C0D9F0C2C0DAF0C3C07F
:10C99000DBF00001DBAF02D0010E01D0000ED26F40
:10C9A000D36BD251D311D8B410D0DB1FDA1FD91FEB
:10C9B000D81FD71FD61FD51FD46D000ED523D62361
:10C9C000D723D823D923DA23DB2302AE039202BE76
:10C9D00005D0025008E10104D8B005D0000ECF6F99
:10C9E000010ECE6F04D001C0CEF002C0CFF09CC1CA
:10C9F000D0F09DC1D1F0D251D311D8A402D003A45C
:10CA000003D0D007D8A0D107000EDD6F4F0EDC6F2A
:10CA1000000E0401976F7CD0DC07D8A0DD07480E1C
:10CA2000DC25D96E040EDD21DA6ED4C025F0D5C028
:10CA300026F0D6C027F0D7C028F0D8C029F0D9C03A
:10CA40002AF0DAC02BF0DBC02CF00A0E2D6E000E9F
:10CA50002E6E000E2F6E000E306E000E316E000E28
:10CA6000326E000E336E000E346E02ECF2F025C012
:10CA7000C4F026C0C5F027C0C6F028C0C7F029C042
:10CA8000C8F02AC0C9F02BC0CAF02CC0CBF0C4C07B
:10CA9000B6F0C6C0B7F0EBEC08F0B651300FDF6E61
:10CAA000CE07D8A0CF07D007D8A0D107D4C025F093
:10CAB000D5C026F0D6C027F0D7C028F0D8C029F0BE
:10CAC000D9C02AF0DAC02BF0DBC02CF00A0E2D6E94
:10CAD000000E2E6E000E2F6E000E306E000E316EA8
:10CAE000000E326E000E336E000E346EABECEDF0C5
:10CAF00025C0D4F026C0D5F027C0D6F028C0D7F086
:10CB000029C0D8F02AC0D9F02BC0DAF02CC0DBF055
:10CB10000001DDBF1FD0DD5103E1DC05D8A01AD034
:10CB2000D451D511D611D711D811D911DA11DB1181
:10CB3000D8A472D7CFBF05D0CF5102E1CE05D8B06F
:10CB40006BD7D1BF07D0D15103E1D005D8A002D017
:10CB500003B262D7D251D311D8A402D003A418D003
:10CB6000DC07D8A0DD07D251D311D8A404D0000E21
:10CB7000CD6F2B0E03D0000ECD6F2D0ECC6F480E57
:10CB8000DC25D96E040EDD21DA6E600033F3DFFFA1
:10CB9000BAC035F0BBC036F0480EDC25376E040E47
:10CBA000DD21386ED0C039F0D1C03AF0C6ECFCF0CF
:10CBB00035C0BAF036C0BBF01200000E0101A86FFC
:10CBC000050EA96F6000A3F6D9FF6000A7F6DAFF93
:10CBD000000EDF6E3D017599738F000E01015E6FCF
:10CBE000020E5D6F5DC125F05EC126F0A0EC0BF07A
:10CBF0000009D8B4DAD001015E355E31596F5D317C
:10CC0000076E59C108F0A8C124F1A9C125F1F10EA0
:10CC1000266FE30E276F5DC128F15EC129F107C0C1
:10CC20002AF108C02BF1F0EC03F07AD0A8C133F060
:10CC3000A9C134F05B0E356EEE0E366E86EC0AF04E
:10CC4000ACD01E0E256E030E266E0D0E276EFC0E4A
:10CC5000286E39EC01F0A8C125F0A9C126F08EECB0
:10CC600004F025C05BF126C05CF101015B51A825F1
:10CC7000296E5C51A9212A6E1E0E2B6E030E2C6E9E
:10CC800000EC02F08AD0A8C133F0A9C134F0A60E9E
:10CC9000356EFB0E366E86EC0AF07FD0A8C133F0FD
:10CCA000A9C134F0F00E356EFA0E366E86EC0AF03D
:10CCB00074D0A8C133F0A9C134F0F60E356EFD0E64
:10CCC000366E86EC0AF069D0A8C133F0A9C134F001
:10CCD000BE0E356EFC0E366E86EC0AF05ED0A8C134
:10CCE00033F0A9C134F0F50E356EFE0E366E86ECCB
:10CCF0000AF053D0A8C133F0A9C134F0370E356E15
:10CD0000ED0E366E86EC0AF048D0A8C133F0A9C10A
:10CD100034F0030E356EFE0E366E86EC0AF03DD012
:10CD200007C059F108C05AF15A51000AD8A4EDD7EA
:10CD30005951200AD8B47AD7010AD8B477D7030A50
:10CD4000D8B474D7010AD8B471D7040AD8B46ED74E
:10CD50000F0AD8B476D7010AD8B473D7030AD8B467
:10CD600070D71D0AD8B48FD70F0AD8B497D7010A45
:10CD7000D8B494D7030AD8B491D7010AD8B48ED7BF
:10CD8000070AD8B496D76B0AD8B49ED73F0AD8B44E
:10CD9000A6D7C80AD8B4AED7B8D7A8C125F0A9C1BC
:10CDA00026F08EECFBF032EC0CF0020E01015D255A
:10CDB0005D6F000E5E215E6F5EBF14D75E5104E1B1
:10CDC000FC0E5D5DD8A00ED73D01739F758932ECD6
:10CDD0000CF0120001015B6F0101C2A11CD0AE0E6C
:10CDE0002B6EFC0E2C6E78EC06F001015B51300FBF
:10CDF0004AEC0CF0090E4AEC0CF0390E01015B25EF
:10CE0000F66EF76AD20EF722F86A000EF8220800D2
:10CE1000F5504AEC0CF01E0E0101246F030E256F35
:10CE2000C00E266FEE0E276FF6C228F1296BF7C2EF
:10CE30002AF12B6BF9C22CF12D6BFAC22EF12F6B5C
:10CE4000F0EC03F0000E5D6F000E5C6F5B51200D87
:10CE5000260E596F060E5A6FF3505927F4505A2375
:10CE60005C515925D96E5D515A21DA6E260E5C252A
:10CE7000E16E030E5D21E26E6F007FFFE7FF5C4B0A
:10CE80005D2B5DBFE3D75D5104E10C0E5C5DD8A066
:10CE9000DDD7000E5D6F010E5C6F000E0001666F46
:10CEA000030E656F5CC167F05DC168F01D0E010186
:10CEB0005C25D96E030E5D21DA6EDF500001696FCB
:10CEC000EAECFAF001015C4B5D2B5DBFE6D75D51EA
:10CED00004E1150E5C5DD8A0E0D71E0E246F030E92
:10CEE000256FD90E266FEE0E276F390E5B25F66E75
:10CEF000F76AD20EF722F86A000EF8220800F55001
:10CF0000286F296BC951020D280EF324F66ED20E3C
:10CF1000F420F76EF86A000EF8220800F5502A6F28
:10CF20002B6BC951020D010EF326000EF422280EC0
:10CF3000F324F66ED20EF420F76EF86A000EF82293
:10CF40000800F5502C6F2D6BF0EC03F0000E5D6FB8
:10CF5000000E5C6F5B51200D260E596F060E5A6F46
:10CF60000C0E5927000E5A23F3505927F4505A2318
:10CF70005C515925D96E5D515A21DA6E260E5C2519
:10CF8000E16E030E5D21E26E6F007FFFE7FF5C4BF9
:10CF90005D2B5DBFDFD75D5104E10C0E5C5DD8A059
:10CFA000D9D7000E5D6F010E5C6F000E0001666F39
:10CFB000040E656F5CC167F05DC168F01D0E010174
:10CFC0005C25D96E030E5D21DA6EDF500001696FBA
:10CFD000EAECFAF001015C4B5D2B5DBFE6D75D51D9
:10CFE00005E1150E5C5DD8B01200DFD7120002AE6D
:10CFF000039202BE05D0025009E10104D8B006D068
:10D00000000E0001746F010E736F04D001C073F045
:10D0100002C074F09CC175F09DC176F003A805D0E4
:10D020000001FE0E7527FF0E762362C077F063C005
:10D0300078F064C079F065C07AF066C07BF067C0B4
:10D040007CF068C07DF069C07EF0000E0001806F4A
:10D050004F0E7F6F000E0401976F82D07F07D8A01C
:10D0600080070F0E7715816F826B82BF08D08251C7
:10D0700004E10A0E815DD8A002D0570E01D0300E17
:10D080008125816F000E8221826FBF0E6B6FFF0EB4
:10D090006C6F6A516D6F6E6B6B516D276C516E23A7
:10D0A0006E5122E11A0E6D5DD8B01ED09F0E6B6FCF
:10D0B000FF0E6C6F200E81116D6F000E82116E6F6E
:10D0C0006B516D276C516E236E510EE11A0E6D5D22
:10D0D000D8B00AD081C02BF082C02CF001EC08F04F
:10D0E0002BC081F02CC082F0480E7F25D96E040E33
:10D0F0008021DA6E600007F2DFFF7307D8A07407A3
:10D100007507D8A0760777C06BF078C06CF079C04F
:10D110006DF07AC06EF07BC06FF07CC070F07DC0A7
:10D1200071F07EC072F0050E09D0D8907233713361
:10D1300070336F336E336D336C336B33E82EF5D74A
:10D140006BC077F06CC078F06DC079F06EC07AF08B
:10D150006FC07BF070C07CF071C07DF072C07EF05B
:10D16000000180BF20D0805104E1020E7F5DD8A075
:10D170001AD07751781179117A117B117C117D11B8
:10D180007E11D8A46BD774BF05D0745102E173052A
:10D19000D8B064D776BF07D0765103E17505D8A023
:10D1A00002D003B25BD703A817D07F07D8A08007AF
:10D1B000480E7F25D96E040E8021DA6E6000ABF137
:10D1C000DFFF7F07D8A08007480E7F25D96E040EA9
:10D1D0008021DA6E300EDF6E60C035F061C036F04F
:10D1E000480E7F25376E040E8021386E75C039F0E9
:10D1F00076C03AF0C6ECFCF035C060F036C061F0A5
:10D200001200000E0001616F020E606F000E636F6E
:10D21000000E626F800E0101AE25D96E050EAF21A2
:10D22000DA6E000EDF6EAF5103E1160EAE5DD8B0C0
:10D23000BBD0AF5104E1130EAE5DD8A0B5D0000E47
:10D240000001656F020E646F2DD0800E6425D96ECB
:10D25000050E6521DA6E3B0EDE18D8A421D0800EB3
:10D260006425D96E050E6521DA6E000EDF6E800E24
:10D270006025256E050E6121266E5BECF6F0000E32
:10D280006225D96E030E6321DA6E600097F0DFFF2E
:10D29000624B632B010E6425606F000E6521616F88
:10D2A000644B652B0101AE510001645D0101AF517A
:10D2B00000016559D8A0C9D7800E6025256E050EDE
:10D2C0006121266E5BECF6F0000E6225D96E030E2E
:10D2D0006321DA6E600097F0DFFF00C3C8F103013D
:10D2E00001511F0B0101C76F02C3C6F103C3CAF18D
:10D2F00004C3CBF103010551070B0101C96FC751ED
:10D300003FEC0CF00201AE6F0C0EAE6502D0000EC9
:10D31000AE6F060E0101C96508D0000EC96F1F0E61
:10D320002B6EE80E2C6E78EC06F0000E0201AF6F4B
:10D33000000E0101CC6FCCC1B0F2CB51B0EC0BF0C0
:10D340000201B16F0101CA51B0EC0BF00201B26FE2
:10D35000C9C1B3F20101C851B0EC0BF00201B46FC6
:10D360000101C751B0EC0BF00201B56F0101C651CC
:10D37000B0EC0BF00201B66F000EB76FAF0E856F09
:10D38000020E866F85C23AF086C23BF0000E3D6EFB
:10D39000080E3C6E680ED9EC04F03D0E2B6EEF0EBD
:10D3A0002C6E78EC06F012004F0E2B6EE20E2C6EF7
